:100000000C94ED0C0C941E0D0C941E0D0C941E0DF6
:100010000C941E0D0C94774E0C945F540C9409763E
:100020000C941E0D0C941E0D0C941E0D0C941E0DA4
:100030000C941E0D0C941E0D0C941E0D0C941E0D94
:100040000C941E0D0C942F810C94FB4D0C941E0DE2
:100050000C941E0D0C941E0D0C941E0D0C94177414
:100060000C941E0D0C9467410C943E410C941E0D93
:100070000C941E0D0C941E0D0C941E0D0C941E0D54
:100080000C941A8A0C941E0D0C941E0D0C941E0DCB
:100090000C9415410C94EC400C941E0D0C941E0D08
:1000A0000C941E0D0C941E0D0C941E0D0C941E0D24
:1000B0000C941E0D0C94D4380C941E0D0C941E0D33
:1000C0000C941E0D0C941E0D0C941E0D0C94C3402C
:1000D0000C949A400C941E0D0C9471400C94484062
:1000E0000C941E0D71134E132A138E13E613AD13C9
:1000F000DD13CC139B1478145414B8143C15D71486
:10010000331522150318311868189F187519AE1980
:10011000E719201AFC1AFC1AFC1AFC1AFC1AFC1A21
:10012000FC1AFC1AFC1AFC1AFC1AFC1AFC1AFC1A1F
:10013000FC1AFC1AFC1AFC1AFC1AFC1AFC1AFC1A0F
:10014000FC1AFC1AFC1AFC1AFC1AFC1AFC1AD61827
:1001500009194019591A8E1AC71AF31CF91CFF1CE9
:10016000051D0B1D111D171D1D1D231D291D2F1DD7
:10017000351D471D4D1D531D591D5F1D651D6B1DF3
:10018000711D771D7D1D831D891D8F1D951D9B1D57
:10019000A11DA71DAD1DB91DBF1DC51DCB1DE31D97
:1001A000E91DEF1DF51DFB1D011E4F1E551E5B1E9B
:1001B000671E6D1E731E7F1E851E8B1E911E971E51
:1001C0009D1EAF1EB51EBB1EC11EC71ECD1EE51E49
:1001D000EB1EF11EF71E0F1F151F1B1F211F251FD2
:1001E000291F2D1F331F371F3B1F3F1F431F471F53
:1001F0004B1F511F571F5D1F631F691F6F1F751F07
:100200007B1FD11D071E0D1E131E191E1F1E251E2E
:10021000D31ED91EDF1EFD1E031F091F811F871F4E
:100220008D1FA31EA91E2B1E311E371E3D1E431EF1
:10023000491E611E791EB31D3B1D411DD71DDD1DCD
:10024000931F991F9F1FC232C232DC32C232E93281
:1002500002331D33383301390A3912392639383916
:100260004A395539413D443D333D373D3D3D7B3D68
:10027000483D4C3D523D563D5A3D603D643D683DD4
:100280007B3D6E3D723D763DD142D642DB42E5423A
:10029000EF426843F9420143094313431D43274397
:1002A0003643404368434A4354435E43B076E47662
:1002B000197739776E77A377B377DD782778317838
:1002C00065789A78A878178C2E8C458C5C8C738C0A
:1002D0008A8CA18CB88CD08CEF8C068D1D8D3C8DBA
:1002E000528D212000464143544F525920524553CC
:1002F00045542120003400330032004E6F6E6500FB
:1003000053746F70706564004E65757472616C2013
:100310005475726E004D6F76696E67205265766512
:10032000727365004D6F76696E6720466F727761F4
:100330007264004272616B696E670054414E4B20DB
:10034000524553544F5245440025004865616C7432
:1003500068204C6576656C3A200056454849434C08
:10036000452052455041495220434F4D504C455431
:10037000450054414E4B2044455354524F59454437
:100380000025004865616C7468204C6576656C3AA0
:100390002000290056454849434C452052455041CC
:1003A000495220535441525445442028005245504C
:1003B000414952204F5045524154494F4E204341EC
:1003C0004E43454C4C45440029004D414348494E5D
:1003D000452047554E204849542120280052455079
:1003E000414952204F5045524154494F4E204341BC
:1003F0004E43454C4C454400290043414E4E4F4E20
:100400002048495421202800547572726574207266
:100410006F746174696F6E206973206E6F74206FE2
:1004200066207479706520536572766F2E204E6F4A
:1004300020736574757020617661696C61626C65AA
:100440002E0054757272657420656C6576617469EE
:100450006F6E206973206E6F74206F6620747970E0
:100460006520536572766F2E204E6F20736574750C
:100470007020617661696C61626C652E00546F70EA
:10048000204C65667400546F702043656E7465720D
:1004900000546F70205269676874004D6964646C21
:1004A00065204C656674004D6964646C6520436525
:1004B0006E746572004D6964646C6520526967688A
:1004C0007400426F74746F6D204C65667400426FE7
:1004D00074746F6D2043656E74657200426F74743E
:1004E0006F6D205269676874004649524D574152FA
:1004F000452056455253494F4E3A20006942757384
:1005000000534275730050504D004E6F6E6520448D
:100510006574656374656400417A696D75746820FB
:1005200020202000456C65766174696F6E20200084
:100530005475726E20202020202020005468726F95
:1005400074746C6520202000537469636B20202034
:10055000202020204D696E2020202043656E746588
:10056000722020204D617820202020446561646243
:10057000616E642020526576657273656400524135
:1005800044494F20494E464F202D20004E4F5420C5
:1005900044455445435445440049474E4F52454411
:1005A00000416E616C6F67004469676974616C003B
:1005B000417578204368616E2E2020204D696E20A1
:1005C000202020204D617820202020205479706543
:1005D000004368616E6E656C73207574696C697A2E
:1005E00065643A20004368616E6E656C73206465D3
:1005F0007465637465643A200020284469736162FD
:100600006C656429002028456E61626C6564290070
:100610004D656368616E6963616C207265636F69C3
:100620006C00416972736F6674004D656368616E3A
:100630006963616C2042617272656C3A2000202807
:100640004D31290020284D3229002028422900421E
:10065000617272656C20456C65766174696F6E3A83
:1006600020200020284D30290020284D312900204D
:100670002841290054757272657420526F74617438
:10068000696F6E3A202020004472697665204D6FB4
:10069000746F72733A202020202020004D4F544F59
:1006A000522054595045530054616E6B20285461B8
:1006B0006D69796120444D44290054616E6B202896
:1006C000444B4C4D2047656172626F78290043614D
:1006D000720048616C66747261636B0054616E6B8A
:1006E00000554E4B4E4F574E00596573004E6F00EC
:1006F0002900252C20446563656C65726174696FFF
:100700006E20666163746F72200020284B69636BF2
:100710006261636B2073706565642000547261636D
:100720006B205265636F696C20456E61626C656415
:100730003A202020004E2F4120666F722076656897
:1007400069636C652074797065005475726E204D14
:100750006F64653A202020202020202020202020A7
:100760002020004E2F4120666F72207665686963F5
:100770006C65207479706500596573202854616D2B
:1007800069796129002500202D20004E657574725D
:10079000616C205475726E20416C6C6F7765643AA1
:1007A0002020200020736563005472616E736D69B0
:1007B0007373696F6E2044656C61793A2020202044
:1007C00020002073656300456E67696E6520506187
:1007D0007573652054696D653A2020202020200023
:1007E000207365630053686966742054696D653AC7
:1007F00020202020202020202020202020004175A3
:10080000746F6D61746963004D616E75616C005445
:1008100072616E736D697373696F6E205479706560
:100820003A202020202020002500596573202D200B
:100830000052657665727365205370656564204C5F
:10084000696D697465643A2020002500596573203C
:100850002D2000466F727761726420537065656465
:10086000204C696D697465643A202000206D7329FD
:100870000025207468726F74746C6520666F722036
:10088000002028004D6F746F72204E7564676520DC
:10089000456E61626C65643A202020200029004E7C
:1008A0006F6E65004E6F6E65002C2050726573652B
:1008B000743A20002900202841646A7573746564C5
:1008C00020746F200020284C6576656C3A20004427
:1008D0006563656C2052616D7020456E61626C6568
:1008E000643A20202020200029004E6F6E65004EC3
:1008F0006F6E65002C205072657365743A20002974
:1009000000202841646A757374656420746F200048
:1009100020284C6576656C3A2000416363656C2045
:1009200052616D7020456E61626C65643A202020D2
:100930002020004163746976652044726976696E8F
:10094000672050726F66696C653A20005665686969
:10095000636C6520547970653A2020202020202087
:1009600020202020004452495645205345545449E4
:100970004E47530020736563005265636F696C20B6
:1009800064656C61793A20202020202020202020DE
:1009900020202020202020202000250059657320C1
:1009A0002D200042617272656C20456C6576617421
:1009B000696F6E205370656564204C696D6974655C
:1009C000643A20002500596573202D20005475726B
:1009D00072657420526F746174696F6E2053706514
:1009E0006564204C696D697465643A202000545533
:1009F000525245542053455454494E475300556E66
:100A00006B6E6F776E004865617679004D6564693D
:100A1000756D004C6967687400437573746F6D0081
:100A2000556E6B6E6F776E004F70656E2050616E05
:100A30007A65720054616D69796120537065630055
:100A400020736563207265636F7665727929002073
:100A50007365632072656C6F61642C2000204D47C4
:100A600020686974732C20002063616E6E6F6E20A5
:100A7000686974732C2000280057656967687420C2
:100A8000436C6173733A20202020200044616D6123
:100A900067652050726F66696C653A2020200059A6
:100AA0006573202800416363657074204D472044BE
:100AB000616D6167653A20005965732028005365B0
:100AC0006E64204D4720495220436F64653A2020D0
:100AD000004E2F4100526570616972656420627931
:100AE0003A202020202020004E2F41004869742009
:100AF00050726F746F636F6C20323A20202000298F
:100B00000020285465616D2000466972652050728E
:100B10006F746F636F6C3A20202020004669726505
:100B20002050726F746F636F6C3A20202020004950
:100B300073205265706169722054616E6B3F202092
:100B40002000495220262054616E6B20426174744B
:100B50006C696E672044697361626C656400424130
:100B600054544C4520494E464F00554E4B4E4F571E
:100B70004E0042656E6564696E6920544253204D93
:100B80006963726F0042656965722055534D2D523D
:100B9000432D320054616967656E20536F756E6432
:100BA0002043617264004F70656E2050616E7A65FB
:100BB0007220536F756E6420436172640042656EEB
:100BC0006564696E6920544253204D696E69005313
:100BD0006F756E6420636172643A2000534F554E06
:100BE0004420434152440048696C6C20506879733A
:100BF00069637320456E61626C65643A2020202031
:100C000020202020200042617272656C20537461A4
:100C100062696C697A6174696F6E20456E61626C9D
:100C200065643A200053656E736F72206465746565
:100C3000637465643A20202020202020202020207A
:100C40002020205965730053656E736F72206E6F9C
:100C5000742064657465637465642100494E45526F
:100C60005449414C204D4541535552454D454E54F4
:100C700020554E495400556E6B6E6F776E00566569
:100C80006869636C6520537065656400456E6769CB
:100C90006E65205370656564005468726F74746C7F
:100CA0006520436F6D6D616E6400537065656420EF
:100CB0006465637265617365732062656C6F77202C
:100CC00000537065656420696E6372656173657356
:100CD0002061626F7665200056656869636C6520E7
:100CE00044657374726F7965640043616E6E6F6EF4
:100CF00020486974004272616B6573204170706CAA
:100D0000696564005661726961626C650020286FD4
:100D100066203529003320286F66203329003220D1
:100D2000286F66203329003120286F662033290080
:100D30003220286F66203229003120286F66203249
:100D40002900506F732000417578204368616E6EF2
:100D5000656C20005661726961626C65004F6E00BF
:100D60004F6666004200410045787465726E616CA2
:100D700020496E7075742000070809090B0C0C0BD4
:100D80000C0C54757272657420537469636B202D5A
:100D9000200046756E6374696F6E202300202D3E1F
:100DA00020002073656300547572726574206D6F46
:100DB00076656D656E742064656C61793A202000FB
:100DC0004E6F6E65005965730054757272657420BC
:100DD000737469636B2066756E6374696F6E733AC2
:100DE000200046554E4354494F4E205452494747E0
:100DF0004552530076206375746F6666290020287B
:100E0000004C564320456E61626C65643A20202098
:100E1000202020007600566F6C746167653A2020B0
:100E2000202020202020202000596573004E6F00D4
:100E30004261747465727920446574656374656495
:100E40003A20004241545445525900536572696139
:100E50006C203320547820426175643A2020004190
:100E600075782053657269616C20426175643A201F
:100E70002020004D6F746F722053657269616C2081
:100E8000426175643A20005553422053657269618E
:100E90006C20426175643A20202000424155442074
:100EA00052415445530000002100240027002A002D
:100EB0002D003000330001010000040107010A0188
:100EC00000002200250028002B002E0031003400F5
:100ED00002010000050108010B01000020002300B1
:100EE000260029002C002F00320000010000030121
:100EF000060109010505050507050808080802029D
:100F000002020A0A080804040404010101010101A3
:100F100001010303030303030303040707070C0C86
:100F20000C0C0C0C0C0C020202020606060606064D
:100F300006060B0B0B0B0B0B0B0B010210202008F2
:100F40000810204010204080020102010804020124
:100F50000102040810204080804020100804020193
:100F600080040201804020100804020108040201EC
:100F70000102040810204080010204081020408073
:100F800000000A0B02090C0D0E0807030401000003
:100F90000000000000000000000000000000000051
:100FA000000000000000000000000000121110000E
:100FB0000000000000000000000000000000000031
:100FC00000000000000042617272656C2053746181
:100FD00062696C697A6174696F6E3A205475726ED9
:100FE0006564204F4E0042617272656C20537461DB
:100FF00062696C697A6174696F6E3A205475726EB9
:101000006564204F46460048696C6C2050687973CF
:101010006963733A205475726E6564204F4E0048C0
:10102000696C6C20506879736963733A20547572E7
:101030006E6564204F464600494F20506F72742001
:1010400041204F7574707574202D204F6E00494FEC
:1010500020506F72742041204F7574707574202D6C
:10106000204F666600494F20506F72742042204F17
:101070007574707574202D204F6E00494F20506F8D
:1010800072742042204F7574707574202D204F6645
:1010900066004C56432045786974202D20566F6CAD
:1010A0007461676520526573746F72656400762998
:1010B000004C5643207468726573686F6C642072CC
:1010C000656163686564212028004C696768742045
:1010D00031204F6E004C696768742031204F66667E
:1010E000004C696768742032204F6E004C69676855
:1010F000742032204F666600326E64204D472053C4
:10110000746F7000326E64204D47205374617274A6
:101110000052756E6E696E67204C69676874732043
:101120004F6E0052756E6E696E67204C6967687409
:1011300073204F666600417578204F757470757422
:10114000204F6E00417578204F7574707574204F74
:1011500066660053746F70205265766F6C76696EA8
:101160006720417578204C696768740053746F700C
:1011700020417578204F757470757420426C696ECB
:101180006B696E6700537461727420417578204FEB
:10119000757470757420426C696E6B696E6700556A
:1011A0006E6B6E6F776E0044657461636865642F63
:1011B0004E41005265636F696C20536572766F0013
:1011C00050616E20536572766F00536572766F2F93
:1011D000455343004F6E626F617264204D6F746FB0
:1011E0007220447269766572004F70656E2050619E
:1011F0006E7A65722053636F7574205365726961EE
:101200006C20455343005361626572746F6F74685C
:101210002053657269616C00506F6C6F6C75205360
:10122000657269616C00536572766F203100536599
:1012300072766F203200536572766F2033005365EB
:1012400072766F203400536572766F2035005365D7
:1012500072766F203600536572766F2037005365C3
:1012600072766F203800524144494F204641494C24
:101270005341464500526164696F2052656164794B
:10128000202D200052657665727365643A20200037
:101290004D61782050756C73653A20004D696E2061
:1012A00050756C73653A2000456E642056616C750C
:1012B000657300456E64205265636F696C205365E9
:1012C00072766F20536574757000456E6420526F9E
:1012D000746174696F6E20536572766F2053657404
:1012E000757000456E6420456C65766174696F6E3B
:1012F00020536572766F2053657475700053657264
:10130000766F20756E2D7265766572736564005315
:101310006572766F207265766572736564005265DA
:101320007665727365643A2020004D6178205075AF
:101330006C73653A20004D696E2050756C73653A88
:10134000200053746172742056616C756573004996
:101350004E56414C494420534552564F2E204E4F35
:101360002053455455502E005365747570205265B6
:10137000636F696C20536572766F00536574757086
:101380002054757272657420526F746174696F6E47
:101390002050616E20536572766F005365747570CE
:1013A0002054757272657420456C65766174696F3E
:1013B0006E2050616E20536572766F0055736572B2
:1013C0002046756E6374696F6E20310055736572C7
:1013D0002046756E6374696F6E203200466F7277B7
:1013E0006172642047656172004E65757472616C4C
:1013F00020476561720052657665727365204765A6
:1014000061720053657420416363656C2052616DA5
:1014100070204C6576656C3A2000536574204465F5
:1014200063656C2052616D70204C6576656C3A2066
:10143000005365742042617272656C2053656E734F
:10144000697469766974793A200053657420486933
:101450006C6C2053656E73697469766974793A208F
:1014600000416E616C6F6720557365722046756E22
:101470006374696F6E2031202D2000416E616C6FA6
:101480006720557365722046756E6374696F6E20B0
:1014900032202D20002D00202D20002000545255F8
:1014A000450046414C534500250057616974696EFB
:1014B0006720666F7220726164696F2E2E2E200085
:1014C000536D6F6B657220656E61626C656400536D
:1014D0006D6F6B65722064697361626C6564005343
:1014E000657420766F6C756D653A20005573657272
:1014F00020536F756E642000466972652043616EEB
:101500006E6F6E0046697265205265706169722067
:101510005369676E616C00416972736F6674202D48
:10152000204D616E75616C20547269676765720049
:101530004D656368616E6963616C205265636F69B4
:101540006C202D204D616E75616C20547269676747
:10155000657200536572766F205265636F696C2007
:101560002D204D616E75616C2054726967676572DC
:10157000004869676820496E74656E7369747920E4
:10158000466C61736820556E6974202D204D616E24
:1015900075616C2054726967676572004D4720530E
:1015A00074617274004D472053746F7000417578F8
:1015B000204F757470757420507265736574204483
:1015C000696D00417578204F757470757420466C94
:1015D000617368656400417578204F757470757427
:1015E00020496E766572736520466C617368656428
:1015F0000053746F7020417578204F757470757446
:1016000020426C696E6B696E670053746F70205274
:1016100065766F6C76696E6720417578204C6967D6
:10162000687400310031202D20537461727420528F
:101630006570656174696E670031202D2053746F89
:101640007000320032202D20537461727420526574
:1016500070656174696E670032202D2053746F705D
:1016600000330033202D2053746172742052657052
:10167000656174696E670033202D2053746F7000AC
:10168000340034202D2053746172742052657065CB
:101690006174696E670034202D2053746F700035BB
:1016A0000035202D2053746172742052657065617D
:1016B00074696E670035202D2053746F70003600FA
:1016C00036202D20537461727420526570656174E8
:1016D000696E670036202D2053746F7000401F70B4
:1016E00017D007A00FA00FDC05D007C4091027886A
:1016F00013983A10276C023A026C023A026C023AD2
:10170000026C02B036384A5C121C255C125C121C5A
:10171000255C12BC7FC7F2C07887A5B7C5A00F882B
:1017200013B80B401FB80BB80B7017401F416972FC
:10173000736F6674202D20456E61626C6564004D88
:10174000656368616E6963616C205265636F696C83
:10175000202D20456E61626C656400416972736F73
:101760006674202D2044697361626C6564004D6568
:101770006368616E6963616C205265636F696C2098
:101780002D2044697361626C656400436F6D6D73F5
:10179000206368616E67656420746F205553420052
:1017A000436F6D6D73206368616E67656420746F4D
:1017B0002053657269616C20310044726976696EEC
:1017C000672050726F66696C652073657420746F52
:1017D0002023005475726E20456E67696E65204F38
:1017E0006E004D616E75616C207472616E736D690F
:1017F0007373696F6E202D2070757420696E206E72
:1018000065757472616C2067656172206265666FD0
:101810007265207374617274696E6720656E6769A2
:101820006E6521005475726E20456E67696E652085
:101830004F666600456E67696E65204175746F205E
:1018400053687574646F776E00456E6761676520D5
:101850005472616E736D697373696F6E004469735E
:10186000656E67616765205472616E736D6973732D
:10187000696F6E00536574205475726E204D6F64ED
:10188000653A203100536574205475726E204D6F97
:1018900064653A203200536574205475726E204D91
:1018A0006F64653A203300456E61626C65204E6559
:1018B000757472616C205475726E73004469736143
:1018C000626C65204E65757472616C205475726E21
:1018D00073002900202D2041646A757374656420AB
:1018E000746F2000202853656E736974697669747B
:1018F0007920002900202D2041646A757374656485
:1019000020746F2000202853656E736974697669AE
:10191000747920005374617274205265766F6C760E
:10192000696E6720417578204C6967687400536F51
:101930006E790052435441204D616368696E6520A1
:1019400047756E00436C61726B204D616368696E10
:10195000652047756E00524354412052657061699D
:1019600072004942552052657061697200436C6192
:10197000726B20526570616972004F70656E5061C4
:101980006E7A657200567354616E6B00464F560056
:1019900054616967656E0048656E67204C6F6E67BD
:1019A0000054616D69796120312F33350054616DC8
:1019B00069796120322D53686F740054616D6979C3
:1019C0006100556E6B6E6F776E003A20004269744D
:1019D00020004761703A20009CA111241FBECFEF68
:1019E000D1E2DEBFCDBF00E00CBF15E0A0E0B2E069
:1019F000EFE8FFE701E00BBF02C007900D92A43BA8
:101A0000B107D9F722E1A4EBB5E001C01D92AE3CCD
:101A1000B207E1F71CE0CDEEDCE000E006C0219764
:101A20000109802FFE010E9498ACCC3ED10780E0D6
:101A30000807A9F70E94D6900C9458B20C940000A5
:101A40002F923F924F925F926F927F928F929F92CE
:101A5000AF92BF92CF92DF92EF92FF920F931F93BC
:101A6000CF93DF93CDB7DEB7A9970FB6F894DEBF5B
:101A70000FBECDBF85EC91E00E94E3B16A327F4496
:101A80008105910519F00E94B78608C049EC51E024
:101A900060E070E087E69EE00E94CBB140E052EC4F
:101AA00061E070E083E998E00E94356340910D1099
:101AB00050910E1060910F107091101086EF97E00A
:101AC0000E943563409111105091121060911310D3
:101AD0007091141089E597E00E94356340911510CC
:101AE0005091161060911710709118108CEB96E0C1
:101AF0000E94356385EF9CE09093B7058093B6050F
:101B000086EB9AE09093B5058093B40583E998E05D
:101B10009093C9128093C81210922D0D1092FA0C56
:101B20001092F70C1092F90C1092F80C11E010932F
:101B3000850D0E94117F80912B108093600610927A
:101B40005F061092800082E0809381008FE286BB66
:101B500010926F0010928500109284009BE2909387
:101B6000A0009AE09093A10089BB1092720010929D
:101B7000A5001092A4001092A9001092A800109243
:101B8000AB001092AA001092AD001092AC0099EA3E
:101B900090932001109321018ABB10927300109240
:101BA000250110922401109229011092280110920F
:101BB0002B0110922A0110922D0110922C0180917C
:101BC000040F9091050F8093F0059093F1058130FB
:101BD00071F461E08FE30E946E428091F1058823E9
:101BE00019F00E9492450FC00E947D450CC0809163
:101BF000F105882311F062E001C060E08FE30E94EC
:101C00006E420E94A4478091060F9091070F809327
:101C1000F7059093F805813071F461E08EE30E943E
:101C20006E428091F805882319F00E9467450FC025
:101C30000E9452450CC08091F805882311F062E0A3
:101C400001C060E08EE30E946E420E94734760E034
:101C500085E40E946E4262E08CE30E946E4262E084
:101C60008BE30E946E4262E080E40E946E4262E07A
:101C700081E40E946E4262E082E40E946E4262E071
:101C800081E20E946E4262E084E40E946E4261E062
:101C900089E30E946E4261E08AE30E946E420E94E4
:101CA00004460E94364661E085E30E946E4261E090
:101CB00085E00E946E4261E070E085E00E94AA42E9
:101CC00061E084E00E946E4261E087E00E946E4223
:101CD00061E089E20E943F4261E089E20E946E4237
:101CE0006A9A60E085E30E943F4260E085E00E94DE
:101CF0003F4260E084E00E943F4260E087E00E9453
:101D00003F42729861E088E00E946E4280E090E07D
:101D10009C012959314FF901ED55FF4F40814F3654
:101D200029F4329720813181232B31F403968837AF
:101D3000910571F760E001C061E088E00E943F42D8
:101D400061E08BE20E946E4260E08BE20E943F42C3
:101D50000E9436460E94D2798091A60A813009F00D
:101D60006CC08091A90A9091AA0AA091AB0AB09187
:101D7000AC0A4091AD0A5091AE0A6091AF0A7091E1
:101D8000B00A841B950BA60BB70B84379E40A105A8
:101D9000B10500F30E94B78680915D0690915E06C2
:101DA0000E94254080915D0690915E060E9425402C
:101DB0000E94906665EE72E080915D0690915E06ED
:101DC0000E94C73E01E010E00E9407460E9436468E
:101DD0006EEE72E080E090E00E94B54362EE72E049
:101DE00080915D0690915E060E94C73E0E94044667
:101DF0000E9433460530110531F064EF71E080E058
:101E000090E00E94B5430F5F1F4F06301105E1F6C9
:101E100080915D0690915E060E9425400E9490662A
:101E200080915D0690915E060E94254080915D063E
:101E300090915E060E94254002C081118BCF809157
:101E40006F00826080936F00809184009091850084
:101E50008056904F909389008093880081E0809312
:101E6000F60D8093F90D8093FC0D8093FF0D809308
:101E70000B0E80930E0E9091BC0F9150953040F058
:101E80008093BC0F61E070E085E591E00E943879B5
:101E90009091BC0F2DEF290F8091800F233008F017
:101EA00012C28A3079F03CF4883009F45DC0893080
:101EB00009F4C1C1B7C18B3009F49EC08C3009F45C
:101EC000E0C0B0C183E290E00E94B2ADFC0188E0C6
:101ED00090E0938382838824839499249A949582B2
:101EE0008482AA24AA94B12CB782A6821186108675
:101EF000108E03E8702E718E89E5C82E87E0D82EEB
:101F0000D38EC28E9AE6E92E92E0F92EF182E0821B
:101F100001E110E111A300A312A2F0934F06E09398
:101F20004E06CF010E94B54983E290E00E94B2AD17
:101F3000FC0189E090E09383828395828482B7825A
:101F4000A68211861086108E718ED38EC28EF1827B
:101F5000E08211A300A312A2F0934D06E0934C0679
:101F6000CF010E94B54934C380E290E00E94B2AD37
:101F7000FC0188E090E093838283882483949924F1
:101F80009A9495828482AA24AA94B12CB782A682BC
:101F900011861086108E7AE0D72ED18EA9E5EA2E12
:101FA000A7E0FA2EF38EE28E02E512E011830083A1
:101FB000F0934F06E0934E06CF010E94835E80E2CD
:101FC00090E00E94B2ADFC0189E090E093838283AF
:101FD00095828482B782A68211861086108ED18E59
:101FE000F38EE28E11830083F0934D06E0934C064E
:101FF000CF010E94835EECC289E190E00E94B2AD05
:10200000FC0188E090E093838283CC24C394DD2498
:10201000DA94D582C482EE24EA94F12CF782E68227
:1020200011861086108E06E412E011830083F0936F
:102030004F06E0934E06CF010E94C95D10920B0E31
:102040008091BC0F843009F0C3C289E190E00E9406
:10205000B2ADFC0189E090E093838283D582C48293
:10206000F782E68211861086108E11830083F0932A
:102070004D06E0934C06CF010E94C95D10920E0EF2
:10208000A7C2943009F063C089E190E00E94B2AD2C
:102090008C01B6E88B2EB5E09B2EDC0111969C924C
:1020A0008E9287E090E013969C938E931297AA24C9
:1020B000A394BB24BA941596BC92AE921497CC24E8
:1020C000CA94D12C1796DC92CE92169719961C9230
:1020D0001E92189758961C92C8010E94FE8126EE07
:1020E000E22E23E0F22EF801F182E08210934F06F7
:1020F00000934E06C8010E94615C1092F60D89E1C2
:1021000090E00E94B2AD8C01DC0111969C928E92FF
:1021100086E090E013969C938E9312971596BC924E
:10212000AE9214971796DC92CE92169719961C923F
:102130001E92189758961C92C8010E94FE81F801C1
:10214000F182E08210934D0600934C0665C085E055
:102150008093BC0F89E190E00E94B2AD8C0176E8DB
:10216000872E75E0972EDC0111969C928E9287E067
:1021700090E013969C938E931297AA24A394BB2469
:10218000BA941596BC92AE921497CC24CA94D12CD2
:102190001796DC92CE92169719961C921E9218975B
:1021A00058961C92C8010E94FE81A6EEEA2EA3E07A
:1021B000FA2EF801F182E08210934D0600934C064E
:1021C000C8010E94615C1092F60D89E190E00E94C6
:1021D000B2AD8C01DC0111969C928E9286E090E06B
:1021E00013969C938E9312971596BC92AE92149769
:1021F0001796DC92CE92169719961C921E921897FB
:1022000058961C92C8010E94FE81F801F182E0827A
:1022100010934F0600934E06C8010E94615C109215
:10222000F90DD6C189E08093800F69E070E089E103
:1022300091E00E94387980E290E00E94B2ADFC010A
:1022400088E090E0938382838824839499249A94ED
:1022500095828482AA24AA94B12CB782A682118680
:102260001086108E50E8D52ED18E69E5E62E67E0F7
:10227000F62EF38EE28E0EE512E011830083F093CA
:102280004F06E0934E06CF010E94614980E290E044
:102290000E94B2ADFC0189E090E093838283958235
:1022A0008482B782A68211861086108ED18EF38E1C
:1022B000E28E11830083F0934D06E0934C06CF012C
:1022C0000E94614985C18A3079F03CF4883009F474
:1022D00055C0893009F425C11BC18B3009F471C088
:1022E0008C3009F4A8C014C183E290E00E94B2AD22
:1022F000FC017090C80F88E090E09383828388246B
:10230000839499249A9495828482AA24AA94B12CC5
:10231000B782A68211861086108E83E8682E618EA1
:1023200099E5C92E97E0D92ED38EC28E2AE6E22EE9
:1023300022E0F22EF182E08201E110E111A300A37C
:1023400072A2F0935106E093500683E290E00E945F
:10235000B2ADFC0189E090E0938382839582848210
:10236000B782A68211861086108E618ED38EC28EA1
:10237000F182E08211A300A372A210C180E290E07A
:102380000E94B2ADFC0188E090E0938382838824B0
:10239000839499249A9495828482AA24AA94B12C35
:1023A000B782A68211861086108EAAE0DA2ED18E10
:1023B000B9E5EB2EB7E0FB2EF38EE28E02E512E0DC
:1023C000D2C089E190E00E94B2ADFC0188E090E0CB
:1023D00093838283CC24C394DD24DA94D582C4828F
:1023E000EE24EA94F12CF782E68211861086108E94
:1023F00006E412E011830083F0935106E093500647
:1024000089E190E00E94B2ADFC0189E090E0938305
:102410008283D582C482F782E68211861086108E6E
:1024200011830083F0935306E093520610920B0E33
:1024300010920E0EB7C0923049F481E08093BC0F29
:1024400061E070E085E591E00E94387989E190E0F3
:102450000E94B2AD8C0186E8882E85E0982ED801C6
:1024600011969C928E9287E090E013969C938E93A7
:102470001297AA24A394BB24BA941596BC92AE9248
:102480001497CC24CA94D12C1796DC92CE9216972E
:1024900019961C921E92189758961C92C8010E9479
:1024A000FE8136EEE32E33E0F32EF801F182E08276
:1024B000109351060093500689E190E00E94B2AD5E
:1024C0008C01DC0111969C928E9286E090E013962E
:1024D0009C938E9312971596BC92AE921497179672
:1024E000DC92CE92169719961C921E9218975896C7
:1024F0001C92C8010E94FE81F801F182E0821093D3
:102500005306009352061092F60D1092F90D4AC030
:1025100089E08093800F69E070E089E191E00E949A
:10252000387980E290E00E94B2ADFC0188E090E052
:10253000938382838824839499249A9495828482B5
:10254000AA24AA94B12CB782A68211861086108E76
:10255000A0E8DA2ED18EB9E5EB2EB7E0FB2EF38E94
:10256000E28E0EE512E011830083F0935106E093B2
:10257000500680E290E00E94B2ADFC0189E090E05C
:102580009383828395828482B782A6821186108685
:10259000108ED18EF38EE28E11830083F09353065A
:1025A000E09352068091520690915306DC01ED9122
:1025B000FC910280F381E02D199580915006909155
:1025C0005106DC01ED91FC910280F381E02D19951B
:1025D0008091BC0F8250823050F589E190E00E94DA
:1025E000B2AD8C0186E895E0F8019183808386E0A6
:1025F00090E09383828381E09FEF958384838FEFC4
:1026000090E09783868311861086108EC8010E9401
:10261000FE8186EE93E0D8018D939C9310934A0639
:1026200000934906C8010E94615C1092F90DE09187
:10263000810F8E2FEE0F990BAA0BBB0BFC01389765
:10264000E830F10508F0B9C08827EE58FF4F8F4FEA
:102650000C9498AC83E290E00E94B2ADFC0188E05B
:1026600090E09383828381E09FEF958384838FEF53
:1026700090E09783868311861086108E84E8818F80
:1026800089E597E0938F828F8AE692E09183808339
:1026900081E190E191A380A312A21EC080E290E0AC
:1026A0000E94B2ADFC0188E090E09383828381E0D8
:1026B0009FEF958384838FEF90E0978386831186C5
:1026C0001086108E87E8818F89E597E0938F828F3F
:1026D0008EE592E091838083F0935806E09357064D
:1026E0009CC080E290E00E94B2ADFC0188E090E0E6
:1026F0009383828381E09FEF958384838FEF90E0C3
:102700009783868311861086108E8DE0818F89E5F0
:1027100097E0938F828F82E592E0DCCF89E190E0B1
:102720000E94B2ADFC0188E090E09383828381E057
:102730009FEF958384838FEF90E097838683118644
:102740001086108E86E492E091838083F093580681
:10275000E093570610920B0E60C08CE190E00E944F
:10276000B2AD8C0186E895E0F8019183808385E025
:1027700090E09383828381E09FEF958384838FEF42
:1027800090E09783868311861086108EC8010E9480
:10279000FE818AE795E038C089E190E00E94B2AD01
:1027A000FC0113821282158214821782168211860E
:1027B0001086108E82E292E08DCF8CE08093810FA4
:1027C0006CE070E08AE191E00E94387989E190E064
:1027D0000E94B2AD8C0186E895E0F8019183808378
:1027E00085E090E09383828381E09FEF95838483EB
:1027F0008FEF90E09783868311861086108EC80134
:102800000E94FE8186EE93E0D8018D939C931093F5
:102810005806009357061092FC0D80915706909130
:102820005806DC01ED91FC910280F381E02D1995B1
:102830008091890F843658F4853608F084E664E682
:10284000681B80915706909158060E94534A8091C8
:10285000810F8C508230A8F460918A0F70918B0F99
:1028600085E00E94843B60918C0F70918D0F85E014
:102870000E94693B80918E0FE0915706F0915806B7
:10288000808FE091820F8E2FEE0F990BAA0BBB0B5E
:10289000FC013897E830F10508F0E5C08827E658D4
:1028A000FF4F8F4F0C9498AC83E290E00E94B2AD42
:1028B000FC0189E090E09383828381E09FEF958320
:1028C00084838FEF90E09783868311861086108E25
:1028D00084E8818F89E597E0938F828F8AE692E082
:1028E0009183808381E190E191A380A312A21EC015
:1028F00080E290E00E94B2ADFC0189E090E0938319
:10290000828381E09FEF958384838FEF90E09783AC
:10291000868311861086108E87E8818F89E597E07F
:10292000938F828F8EE592E091838083F0935C0693
:10293000E0935B06C8C080E290E00E94B2ADFC016B
:1029400089E090E09383828381E09FEF9583848385
:102950008FEF90E09783868311861086108E8DE02E
:10296000818F89E597E0938F828F82E592E0DCCFBB
:1029700089E190E00E94B2ADFC0189E090E0938390
:10298000828381E09FEF958384838FEF90E097832C
:10299000868311861086108E86E492E09183808370
:1029A000F0935C06E0935B0610920E0E8CC08CE1F7
:1029B00090E00E94B2AD8C0196E8692E95E0792EE8
:1029C000F8017182608224E0822E912C93828282AF
:1029D000AA24A394BB24BA94B582A482CC24CA941A
:1029E000D12CD782C68211861086108EC8010E9413
:1029F000FE815AE7E52E55E0F52ED801ED92FC92C6
:102A000010935C0600935B068CE190E00E94B2ADEF
:102A10008C01FC017182608293828282B582A482E1
:102A2000D782C68211861086108E0E94FE81D80140
:102A3000ED92FC9210937D0D00937C0DC8010E94D5
:102A4000235D3FC089E190E00E94B2ADFC0113829A
:102A50001282158214821782168211861086108EB9
:102A600082E292E061CF8CE08093820F6CE070E0B4
:102A70008BE191E00E94387989E190E00E94B2AD4B
:102A80008C0186E895E0F8019183808384E090E0F2
:102A90009383828381E09FEF958384838FEF90E01F
:102AA0009783868311861086108EC8010E94FE814E
:102AB00086EE93E0D8018D939C9310935C0600936F
:102AC0005B061092FF0D80915B0690915C06DC0125
:102AD000ED91FC910280F381E02D19958091880F92
:102AE000843658F4853608F084E664E6681B8091E5
:102AF0005B0690915C060E94534A8091820F8C5035
:102B0000823000F56091830F7091840F84E00E9401
:102B1000843B6091850F7091860F84E00E94693B31
:102B20008091870FE0915B06F0915C06808F809129
:102B3000820F8D3039F48091870FE0917C0DF091F8
:102B40007D0D808F8EE190E00E94B2AD8C01D0901F
:102B5000930FA090970FB090980F8090950F909042
:102B6000960F86E895E0F8019183808383E090E0FA
:102B70009383828381E09FEF95838483EE24EA949C
:102B8000F12CF782E68211861086108EC8010E9411
:102B9000FE818AE392E0D80111969C938E935A9617
:102BA0009C928E9259975C96BC92AE925B975D9682
:102BB000DC9210933C0E00933B0E6091990F709144
:102BC0009A0F83E00E94843B60919B0F70919C0F51
:102BD00083E00E94693B8091930FE0913B0EF0915E
:102BE0003C0E808F8091930F0E94037980913B0E61
:102BF00090913C0EDC01ED91FC910280F381E02D7F
:102C0000199580919D0F882339F185E290E00E940B
:102C1000B2ADFC018091A20F9091A30F2091A00F63
:102C20003091A10F40919E0F50919F0F68E070E08E
:102C30007383628315821482F782E682118610867E
:102C4000108E6EE272E071836083528F418F348FF9
:102C5000238F968F858F22C085E290E00E94B2ADCF
:102C6000FC018091A00F9091A10F20919E0F3091B7
:102C70009F0F48E050E05383428315821482F7820D
:102C8000E68211861086108E4EE252E05183408318
:102C9000328F218F948F838FF68EE58EF093E70528
:102CA000E093E6058091E6059091E7050E94A75D17
:102CB00080910B0E8823F9F089E190E00E94B2AD7B
:102CC000FC0188E090E093838283158214828FEF69
:102CD00093E0978386838FEF91E091878087108EB2
:102CE00086E492E091838083F0930A0EE093090ECC
:102CF000CF010E94C95D80910E0E8823F9F089E111
:102D000090E00E94B2ADFC0189E090E09383828361
:102D1000158214828FEF93E0978386838FEF91E083
:102D200091878087108E86E492E091838083F09370
:102D30000D0EE0930C0ECF010E94C95D87EB9AE067
:102D400090932612809325121091CB0F2091CA0FD9
:102D50008091B90F9091BB0F3091BC0F3093B805A3
:102D60009093BB058093BC0530E0AFEFB0E00E94CC
:102D700049B224E630E040E050E00E94FBB12093ED
:102D8000B412612F70E080E090E00E94B6B023ECB6
:102D900034E64AEA5AE30E9417B12AE939E949E5DB
:102DA0005FE30E94ADAC6093AE127093AF1280935C
:102DB000B0129093B112109295001092940010925C
:102DC00090008CE08093910084EF90E090939900C4
:102DD0008093980011E018BB82E08093710080918D
:102DE00000020E94AD7E80915D0690915E0620916A
:102DF00060064091B50F5091B60F50937F124093EB
:102E00007E12209315129093141280931312109235
:102E1000BD05109380128091D20F853040F0109242
:102E2000D20F60E070E08BE691E00E94387910915B
:102E3000D20F123009F441C0F0F4112309F463C039
:102E4000113009F058C08BE090E00E94B2AD2EE244
:102E500033E0FC013183208329E537E03287218785
:102E600090935A06809359061093020E1093050E04
:102E70001093080E67C0133009F45EC01430D9F502
:102E800085E090E00E94B2AD8C012AE833E0FC01BD
:102E900021933193CF0141E067EB7AE00E946938DA
:102EA00086E792E0D8018D939C9310935A06009385
:102EB000590681E08093020E41C086E090E00E94B6
:102EC000B2AD22ED32E0DC012D933C9390935A0693
:102ED000809359068FB7F8942CED35E03093531159
:102EE00020935211109258118FBF81E08093020EEF
:102EF0008093050E25C01092D20F60E070E08BE643
:102F000091E00E94387985E090E00E94B2AD8C019A
:102F10002AE833E0FC0121933193CF0140E067EBD5
:102F20007AE00E94693886E792E0D8018D939C93FD
:102F300010935A06009359061092020E1092050E35
:102F40001092080E8091590690915A06DC01ED917D
:102F5000FC910190F081E02D19958091F60D811181
:102F60001FC08091F90D81111BC08091FC0D811152
:102F700017C08091FF0D811113C08091020E811145
:102F80000FC08091050E81110BC08091080E811138
:102F900007C081E00E940D7F882309F43DC335C33B
:102FA000A12CB12C812C712C312C412C912C512C29
:102FB000612C06E815E0EE24EA94A3E0FA2ECC2476
:102FC000CA94DD24D394C5018959914FFC01ED5574
:102FD000FF4FE081EE2309F40FC3DC01AF55BF4F73
:102FE0008D919C91892B09F407C38E2F90E0FC01F1
:102FF000F797EB32F10508F0FFC28827EE57FF4F35
:103000008F4F0C9498AC8091F60D882309F4F4C28C
:103010006110F2C289E190E00E94B2AD9C01FC0116
:103020001183008387E090E093838283158214826A
:10303000F782E682D186C086108EC90128A739A7FB
:103040000E94FE8128A539A5E6EEF3E0D901ED93B3
:10305000FC933093E70D2093E60DC9010E94615C5B
:103060007AC18091F90D882309F4C6C25110C4C2F7
:1030700089E190E00E94B2AD9C01DC0111961C93A5
:103080000E93E6E0F0E01396FC93EE9312971596FC
:103090001C921E9214971796FC92EE921697199610
:1030A000DC92CE92189758961C9228A739A70E94B6
:1030B000FE8128A539A5E6EEF3E0D901ED93FC9356
:1030C0003093E90D2093E80DC9010E94615C7CC139
:1030D0008091FC0D882309F48FC291108DC289E183
:1030E00090E00E94B2AD9C01DC0111961C930E93FE
:1030F000E5E0F0E01396FC93EE93129715961C9280
:103100001E9214971796FC92EE9216971996DC92DF
:10311000CE92189758961C9228A739A70E94FE8134
:1031200028A539A5E6EEF3E0D901ED93FC933093A1
:10313000EB0D2093EA0DC9010E94615C7EC1809174
:10314000FF0D882309F458C2411056C289E190E06E
:103150000E94B2AD9C01DC0111961C930E93E4E039
:10316000F0E01396FC93EE93129715961C921E9224
:1031700014971796FC92EE9216971996DC92CE92BF
:10318000189758961C9228A739A70E94FE8128A557
:1031900039A5E6EEF3E0D901ED93FC933093ED0D04
:1031A0002093EC0DC9010E94615C80C18091020EE8
:1031B000882309F421C231101FC289E190E00E94E6
:1031C000B2AD1C01DC0111961C930E93E2E0F0E01D
:1031D0001396FC93EE93129715961C921E921497D9
:1031E0001796FC92EE9216971996DC92CE9218974B
:1031F00058961C920E94FE81E6EEF3E0D101ED9319
:10320000FC933092EF0D2092EE0DC1010E94615CA3
:1032100082C18091050E882309F4EEC17110ECC1C2
:1032200089E190E00E94B2AD9C01DC0111961C93F3
:103230000E93E1E0F0E01396FC93EE93129715964F
:103240001C921E9214971796FC92EE92169719965E
:10325000DC92CE92189758961C9228A739A70E9404
:10326000FE8128A539A5E6EEF3E0D901ED93FC93A4
:103270003093F10D2093F00DC9010E94615C84C16F
:103280008091080E882309F4B7C18110B5C189E186
:1032900090E00E94B2AD9C01DC0111961C930E934C
:1032A00013961C921E92129715961C921E921497BA
:1032B0001796FC92EE9216971996DC92CE9218977A
:1032C00058961C9228A739A70E94FE8128A539A5E7
:1032D00086EE93E0F901918380833093F30D209380
:1032E000F20DC9010E94615C85C18091F60D8823B1
:1032F00009F482C1611080C18CE190E00E94B2ADFE
:103300009C01DC0111961C930E93E7E0F0E013960C
:10331000FC93EE93129715961C921E921497179693
:10332000FC92EE9216971996DC92CE9218975896C8
:103330001C9228A739A70E94FE8128A539A5EAE793
:10334000F5E0D901ED93FC933093F50D2093F40D46
:10335000C9010E94235D662463944EC18091F90DDA
:10336000882309F449C1511047C18CE190E00E94C3
:10337000B2AD9C01DC0111961C930E93E6E0F0E0E7
:103380001396FC93EE93129715961C921E92149727
:103390001796FC92EE9216971996DC92CE92189799
:1033A00058961C9228A739A70E94FE8128A539A506
:1033B000EAE7F5E0D901ED93FC933093F80D209303
:1033C000F70DC9010E94235D5524539415C18091C6
:1033D000FC0D882309F410C191100EC18CE190E01E
:1033E0000E94B2AD9C01DC0111961C930E93E5E0A6
:1033F000F0E01396FC93EE93129715961C921E9292
:1034000014971796FC92EE9216971996DC92CE922C
:10341000189758961C9228A739A70E94FE8128A5C4
:1034200039A5EAE7F5E0D901ED93FC933093FB0D64
:103430002093FA0DC9010E94235D99249394DCC066
:103440008091FF0D882309F4D7C04110D5C08CE1CD
:1034500090E00E94B2AD9C01DC0111961C930E938A
:10346000E4E0F0E01396FC93EE93129715961C920D
:103470001E9214971796FC92EE9216971996DC926C
:10348000CE92189758961C9228A739A70E94FE81C1
:1034900028A539A5EAE7F5E0D901ED93FC9330932F
:1034A000FE0D2093FD0DC9010E94235D4424439429
:1034B000A3C08091020E882309F49EC031109CC0E5
:1034C0008CE190E00E94B2AD1C01DC0111961C93CE
:1034D0000E93E2E0F0E01396FC93EE9312971596AC
:1034E0001C921E9214971796FC92EE9216971996BC
:1034F000DC92CE92189758961C920E94FE81EAE7C1
:10350000F5E0D101ED93FC933092010E2092000E74
:10351000C1010E94235D332433946EC08091050E57
:10352000882309F469C0711067C08CE190E00E94A3
:10353000B2AD9C01DC0111961C930E93E1E0F0E02A
:103540001396FC93EE93129715961C921E92149765
:103550001796FC92EE9216971996DC92CE921897D7
:1035600058961C9228A739A70E94FE8128A539A544
:10357000EAE7F5E0D901ED93FC933093040E209334
:10358000030EC9010E94235D7724739435C0809196
:10359000080E882389F181102FC08CE190E00E94F1
:1035A000B2AD9C01DC0111961C930E9313961C92F4
:1035B0001E92129715961C921E9214971796FC92C3
:1035C000EE9216971996DC92CE92189758961C9206
:1035D00028A739A70E94FE8128A539A58AE795E08A
:1035E000F901918380833093070E2093060EC90161
:1035F0000E94235D8824839493E0A90EB11CA8E760
:10360000AA16B10409F0DFCCC4CC82E00E940D7F81
:10361000882311F01DA216C081E00E940D7F88232F
:1036200029F082E00E94F17E811194C68CE30E9411
:103630001742892B09F07FC68CE30E941742892B21
:1036400009F07FC686E0EFEFFFE0DE0154960190BF
:103650000D928A95E1F79090F80FA0900810B09025
:10366000F90F7091FA0F6091FB0F5091FC0F409190
:10367000FD0F3091FE0F2091051080910610909162
:103680000710A0915906B0915A06BFA3AEA30091AE
:103690003B0E10913C0E50902610E0901F10F090C1
:1036A00020107090291060902810C090910FD09039
:1036B000920F4090940F30908F0F2090900FBDA1EB
:1036C000BB8B9A8EAB8EBC8E7D8F6E8F5F8F48A327
:1036D00039A32AA39CA38BA3F2E18F2EFE0173963C
:1036E000DE01119601900D928A94E1F7E7EBFAE082
:1036F000F093C605E093C505EDA1E9839886A986F8
:10370000BA867B876C875D874E873F87288B9A8B2D
:10371000898B82E1FE013196A2EDB5E001900D9218
:103720008A95E1F720924C0E30924D0E40924B0E4E
:10373000D092340EC092330E50923D0E6092380EED
:103740007092370EF092360EE092350E10934A0EBC
:103750000093490E8EA19FA19093C8058093C70541
:1037600087E08093B4091092B50961E00E946E422F
:103770000E94A7791092B6091092B7098091DD05D1
:10378000811102C01092DE059091D905911105C0FA
:10379000811103C010928D0AA3C081E080938D0A2D
:1037A0000091880A1091890A8091180A60E00E94AD
:1037B0006E42D801ED91FC910190F081E02DC8019D
:1037C00019958091D205882359F1813071F08330A9
:1037D000C1F488E293E29093D4058093D30589E005
:1037E0008093D70580E197E217C088EB9BE0909328
:1037F000D4058093D30583E08093D70588E99AE3C5
:103800000BC088E893E19093D4058093D30586E0BC
:103810008093D70580EE9EE29093D6058093D505E0
:103820008091D9058823E9F18091DD056091D70564
:1038300070E08823C9F08091DF058823A9F080E03B
:1038400090E00E94B6B09B01AC0160E070E088ECB3
:1038500092E40E9411AD6093C9057093CA058093EC
:10386000CB059093CC0525C080E090E00E94B6B0D7
:103870009B01AC0160E070E088EC92E40E9411AD25
:103880006093C9057093CA058093CB059093CC05CE
:103890001092C0051092C1051092C2051092C30586
:1038A0001FC01092C9051092CA051092CB05109244
:1038B000CC056091D80570E080E090E00E94B6B041
:1038C0009B01AC0160E070E088EC92E40E9411ADD5
:1038D0006093C0057093C1058093C2059093C305A2
:1038E0001092E5051092D1051092C4051092CD05F5
:1038F0001092CE051092CF051092D0050E944D7106
:103900006E98769AEE9880916A008F7C80936A0018
:1039100080914D0E882321F080916A00806203C05F
:1039200080916A00806380936A00EE980E94ED7334
:1039300080E090E040E09C012959314FF901ED55BC
:10394000FF4F5081552331F0329720813181232B55
:1039500009F04F5F03968837910569F74093EA05B0
:10396000A9EFB5E020E030E080ED282E85E6382E86
:1039700095E5492E94E6592E4BE7642E44E6742EC5
:103980005BE3852E54E6952E68E4A62E64E6B62EFB
:1039900041EF55E608ED15E672E1E72E7EE6F72EDB
:1039A000E4E2CE2EE6E6DE2EC9018959914FFC01F4
:1039B000ED55FF4F6081662309F4C6C28F559F4FB6
:1039C000FC0180819181892B09F4BEC270E0FB016A
:1039D0003197E637F10508F0B7C28827E355FF4F66
:1039E0008F4F0C9498AC82E89BE611969C938E9333
:1039F000ABC280E89BE611969C938E93A5C28EE79E
:103A00009BE611969C938E939FC287E79BE6119647
:103A10009C938E9399C285E79BE611969C938E9317
:103A200093C283E09BE611969C938E938DC285E0B2
:103A30009BE611969C938E9387C286EE9AE611962A
:103A40009C938E9381C282ED9AE611969C938E93FD
:103A50007BC283EC9AE611969C938E9375C287E69F
:103A60009AE611969C938E936FC28EE19AE6119618
:103A70009C938E9369C281E19AE611969C938E93F2
:103A800063C284E09AE611969C938E935DC282E0B5
:103A90009AE611969C938E9357C28EE191E7119608
:103AA0009C938E9351C287E191E711969C938E93DC
:103AB0004BC287E091E711969C938E9345C285E0B7
:103AC00091E711969C938E933FC283E091E7119604
:103AD0009C938E9339C283EF90E711969C938E93BB
:103AE00033C281EF90E711969C938E932DC28FEE97
:103AF00090E711969C938E9327C28FED90E71196D5
:103B00009C938E9321C28DED90E711969C938E939A
:103B10001BC28BED90E711969C938E9315C282E0A9
:103B20009EE611969C938E930FC280E09EE61196BE
:103B30009C938E9309C28EEF9DE611969C938E9373
:103B400003C280E794E411969C938E93FDC188ECA8
:103B500090E711969C938E93F7C18EE390E71196B0
:103B60009C938E93F1C18FE190E711969C938E9375
:103B7000EBC186EC90E711969C938E93E5C187E9A3
:103B800090E711969C938E93DFC180E990E71196A0
:103B90009C938E93D9C18FE590E711969C938E9359
:103BA000D3C18BE89BE611969C938E93CDC18EE595
:103BB00090E711969C938E93C7C18DE590E711967F
:103BC0009C938E93C1C185E090E711969C938E9350
:103BD000BBC18BEE9FE611969C938E93B5C181ED90
:103BE0009FE611969C938E93AFC187EB9FE611964B
:103BF0009C938E93A9C18DE99FE611969C938E9319
:103C0000A3C183E89FE611969C938E939DC189E69C
:103C10009FE611969C938E9397C18FE49FE6119631
:103C20009C938E9391C185E39FE611969C938E930E
:103C30008BC18BE19FE611969C938E9385C181E0A9
:103C40009FE611969C938E937FC187EE9EE6119618
:103C50009C938E9379C18DEC9EE611969C938E93E6
:103C600073C183EB9EE611969C938E936DC189E997
:103C70009EE611969C938E9367C18FE79EE6119600
:103C80009C938E9361C185E69EE611969C938E93DC
:103C90005BC18BE49EE611969C938E9355C18EEE8C
:103CA0009DE611969C938E934FC18CEE9DE61196E6
:103CB0009C938E9349C18AEE9DE611969C938E93B8
:103CC00043C186E39EE611969C938E933DC18AED97
:103CD0009DE611969C938E9337C188ED9DE61196D3
:103CE0009C938E9331C186ED9DE611969C938E93A5
:103CF0002BC181E29EE611969C938E9325C189E3A8
:103D000095E611969C938E931FC18EEE94E61196C4
:103D10009C938E9319C185EE9CE711969C938E938C
:103D200013C181ED9CE711969C938E930DC18DEB91
:103D30009CE711969C938E9307C18AED99E61196A4
:103D40009C938E9301C188E194E611969C938E9387
:103D5000FBC086E094E611969C938E93F5C08FE4A9
:103D600093E611969C938E93EFC08DE393E61196A4
:103D70009C938E93E9C083EE94E611969C938E9368
:103D8000E3C088ED94E611969C938E93DDC08DEC94
:103D900094E611969C938E93D7C082EC94E611968C
:103DA0009C938E93D1C087EB94E611969C938E934F
:103DB000CBC08CEA94E611969C938E93C5C081EAA1
:103DC00094E611969C938E93BFC08DEC93E611966A
:103DD0009C938E93B9C08BEB93E611969C938E9334
:103DE000B3C089EA93E611969C938E93ADC087E9A0
:103DF00093E611969C938E93A7C085E893E611965F
:103E00009C938E93A1C083E793E611969C938E9327
:103E10009BC081E693E611969C938E9395C08EE1AC
:103E20009EE611969C938E938FC08BE19EE6119631
:103E30009C938E9389C085E19EE611969C938E9308
:103E400083C01196DC92CE927FC01196FC92EE92C6
:103E50007BC011961C930E9377C082ED95E6119668
:103E60009C938E9371C011965C934E936DC0119686
:103E7000BC92AE9269C011969C928E9265C01196CA
:103E80007C926E9261C011965C924E925DC01196CA
:103E90003C922E9259C0E5EAFCE71196FC93EE9312
:103EA00053C082E99CE711969C938E934DC0E8EA3B
:103EB000F5E41196FC93EE9347C08DEC95E61196D0
:103EC0009C938E9341C0EAECF5E61196FC93EE9339
:103ED0003BC081EC95E611969C938E9335C0EAEB3E
:103EE000F5E61196FC93EE932FC080EC95E61196C3
:103EF0009C938E9329C0EBEBF5E61196FC93EE9321
:103F000023C089EF93E611969C938E931DC0ECEE2F
:103F1000F3E61196FC93EE9317C08FED93E611969E
:103F20009C938E9311C0E8EAF5E61196FC93EE930C
:103F30000BC086E995E611969C938E9305C0E4E844
:103F4000F5E61196FC93EE932D5F3F4F12962837BE
:103F5000310509F029CD1092EB058091F005811112
:103F600014C080E090E0FC01E85FF04F20813181D7
:103F7000245631092436310528F0039688379105F7
:103F800091F703C081E08093EB051092F2058091D8
:103F9000F705811114C080E090E0FC01E85FF04F6C
:103FA00020813181285C31092436310528F00396BF
:103FB0008837910591F703C081E08093F2058091E5
:103FC000590690915A06DC01ED91FC91EC5BFF4F94
:103FD0002091D50F3091D60F4091D30F5091D40F2F
:103FE0000190F081E02D61E0199580915906909142
:103FF0005A06DC01ED91FC91EC5BFF4F2091D90F4B
:104000003091DA0F4091D70F5091D80F0190F08185
:10401000E02D62E019958091590690915A06DC01D5
:10402000ED91FC91EC5BFF4F2091DD0F3091DE0FA5
:104030004091DB0F5091DC0F0190F081E02D63E0A7
:1040400019958091590690915A06DC01ED91FC91E9
:10405000EC5BFF4F2091E80F3091E90F4091E60FA4
:104060005091E70F0190F081E02D64E01995809167
:10407000590690915A06DC01ED91FC91EC5BFF4FE3
:104080002091EC0F3091ED0F4091EA0F5091EB0F22
:104090000190F081E02D65E019958091590690918D
:1040A0005A06DC01ED91FC91EC5BFF4F2091F00F83
:1040B0003091F10F4091EE0F5091EF0F0190F08190
:1040C000E02D66E019958091590690915A06DC0121
:1040D000ED91FC91EA5BFF4F0190F081E02D409162
:1040E000DF0F61E019958091590690915A06DC0125
:1040F000ED91FC91EA5BFF4F0190F081E02D409142
:10410000E00F62E019958091590690915A06DC0102
:10411000ED91FC91EA5BFF4F0190F081E02D409121
:10412000E10F63E019958091590690915A06DC01E0
:10413000ED91FC91EA5BFF4F0190F081E02D409101
:10414000F20F64E019958091590690915A06DC01AE
:10415000ED91FC91EA5BFF4F0190F081E02D4091E1
:10416000F30F65E019958091590690915A06DC018C
:10417000ED91FC91EA5BFF4F0190F081E02D4091C1
:10418000F40F66E019958091590690915A06DC016A
:10419000ED91FC9106A8F7A9E02D6091E30F199528
:1041A0008091590690915A06DC01ED91FC9104A48E
:1041B000F5A5E02D6091E40F199580915906909135
:1041C0005A06DC01ED91FC9102A8F3A9E02D609163
:1041D000E50F199580E090E09C012959314FF901D4
:1041E000ED55FF4F4081423731F4329720813181C4
:1041F000232B09F0B5C003968837910569F70E9413
:10420000166C8091590690915A06DC01ED91FC9153
:10421000EA5AFF4F0190F081E02D40E06091F50FE8
:1042200019958091590690915A06DC01ED91FC9107
:10423000EA5AFF4F0190F081E02D41E06091F70FC5
:1042400019958091590690915A06DC01ED91FC91E7
:10425000EA5AFF4F0190F081E02D42E06091F60FA5
:1042600019958091CC0F882331F08091820F8D3089
:1042700011F01092CC0F1092BB0610921C0D809181
:10428000CD0F8093BA058091CF0F8093B90520910F
:104290001D1030E0AFEFB0E00E9449B224E630E0FC
:1042A00040E050E00E94FBB120931D0D80911C1056
:1042B00081110E9477460E949B5A0E94ED436B0138
:1042C0007C0110E011110FC080916006882359F025
:1042D0002AE234E640ED57E060E070E087EB9AE0D8
:1042E0000E946C3A11E00E944060882351F00E94C5
:1042F000B4450E948B480E9436460E94CD5F0E94C2
:10430000D1450E943F84029711F00E94294F0E94DC
:10431000E56C0E943F840297A9F60E94ED43DC0100
:10432000CB018C199D09AE09BF098C3B9240A105B8
:10433000B10540F218C082E00E940D7F81110DC0CE
:104340007BC982E00E94F17E882309F47BC9F3E0F7
:10435000FDA378C9B1E0BDA375C9E2E0EDA372C9C0
:104360000E940A6C4ECF0E94485A0E9436468091A5
:10437000A10A811102C00E94E07A0E94148486E39F
:104380000E947143BC01990F880B990B611571054F
:104390008105910511F00E943DB028E333E648EE17
:1043A00053E060E070E087EB9AE0A9960FB6F894CE
:1043B000DEBF0FBECDBFDF91CF911F910F91FF9058
:1043C000EF90DF90CF90BF90AF909F908F907F90B5
:1043D0006F905F904F903F902F900C946C3A2F927B
:1043E0003F924F925F926F927F928F929F92AF9285
:1043F000BF92CF92DF92EF92FF920F931F93CF93D2
:10440000DF93CDB7DEB7E7970FB6F894DEBF0FBEE8
:10441000CDBF80915D0690915E060E9425400E946E
:10442000906669EE74E080915D0690915E060E9450
:10443000C73E6EE875E0CE0101960E94883E00916D
:104440005D0610915E06D801ED91FC914D815E8173
:1044500069817A810280F381E02DC8011995C80134
:104460000E942540CE0101960E94583E0E94E56CB4
:1044700080915D0690915E06DC01ED91FC910284D5
:10448000F385E02D199580915D0690915E060E945E
:1044900025400E9490666EE775E080915D069091E0
:1044A0005E060E94C73EE091A20AE4300CF0E0E014
:1044B0008AE095E09A83898386E095E09C838B83EC
:1044C00081E095E09E838D838CEF94E098878F83C5
:1044D000EE0FFF0B81E090E08C0F9D1FE80FF91F9E
:1044E0006081718180915D0690915E060E943840E6
:1044F0000E94906668E475E080915D0690915E068A
:104500000E9438400E9490666CE375E080915D06E1
:1045100090915E060E94C73EE0913111F0913211F8
:1045200081819281883E934014F40E948066E091DC
:104530003111F09132116181728180915D0690910B
:104540005E060E945B7A84E00E94728AE0913111DB
:10455000F09132116581768180915D0690915E06C1
:104560000E945B7A85E00E94728AE0913111F0919D
:1045700032116381748180915D0690915E060E9484
:104580005B7A84E00E94728AE0913111F0913211DD
:10459000678180915D0690915E060E94417A88E075
:1045A0000E94728AE0913111F091321180850E944F
:1045B0006C6660E375E080915D0690915E060E94F6
:1045C000C73EE0913B11F0913C1181819281883E80
:1045D000934014F40E948066E0913B11F0913C11ED
:1045E0006181728180915D0690915E060E945B7A86
:1045F00084E00E94728AE0913B11F0913C11658148
:10460000768180915D0690915E060E945B7A85E0DE
:104610000E94728AE0913B11F0913C116381748198
:1046200080915D0690915E060E945B7A84E00E9414
:10463000728AE0913B11F0913C11678180915D0697
:1046400090915E060E94417A88E00E94728AE09111
:104650003B11F0913C1180850E946C6664E275E02C
:1046600080915D0690915E060E94C73EE0914511E3
:10467000F091461181819281883E934014F40E940A
:104680008066E0914511F0914611618172818091BF
:104690005D0690915E060E945B7A84E00E94728AB9
:1046A000E0914511F09146116581768180915D061A
:1046B00090915E060E945B7A85E00E94728AE0918A
:1046C0004511F09146116381748180915D0690914E
:1046D0005E060E945B7A84E00E94728AE091451136
:1046E000F0914611678180915D0690915E060E946F
:1046F000417A88E00E94728AE0914511F09146115A
:1047000080850E946C6668E175E080915D069091FD
:104710005E060E94C73EE0914F11F09150118181D9
:104720009281883E934014F40E948066E0914F117C
:10473000F09150116181728180915D0690915E06C9
:104740000E945B7A84E00E94728AE0914F11F0919E
:1047500050116581768180915D0690915E060E9480
:104760005B7A85E00E94728AE0914F11F0915011BE
:104770006381748180915D0690915E060E945B7AF0
:1047800084E00E94728AE0914F11F091501167818C
:1047900080915D0690915E060E94417A88E00E94B9
:1047A000728AE0914F11F091501180850E946C66E1
:1047B00080915D0690915E060E9425400E941484BF
:1047C000C82E60EB75E080915D0690915E060E94B8
:1047D00038400E94906600ED10E1E12CF12CD12CC4
:1047E00057012FEFA21AB20AB50180915D06909190
:1047F0005E060E945B7A49E0E416F10410F48BE057
:1048000001C08AE00E94728AD8012C9180915D06D5
:1048100090915E062223C9F11596ED91FC911697B1
:10482000618172810E945B7AD8011596ED91FC91AD
:10483000169781819281883E934014F40E9480668D
:1048400084E00E94728AD8011596ED91FC9116972A
:104850006381748180915D0690915E060E945B7A0F
:1048600084E00E94728AD8011596ED91FC9116970A
:10487000278180915D0690915E06222319F068EAF7
:1048800075E00BC061EA75E008C0EC14FD041CF48F
:1048900069E975E002C06CE875E00E943840095F84
:1048A0001F4F7501BCE0AB16B10409F099CF0E940F
:1048B000906665EE75E080915D0690915E060E94BF
:1048C000C73E0E941484682F80915D0690915E0619
:1048D0000E94EC7861ED75E080915D0690915E0636
:1048E0000E94C73E60919F0A7091A00A80915D0668
:1048F00090915E060E94917A0E94E56C80915D061F
:1049000090915E06DC01ED91FC910284F385E02D2F
:10491000199580915D0690915E060E9425400E9447
:1049200090666CE976E080915D0690915E060E944B
:1049300038400E94906668E876E080915D0690912C
:104940005E060E94C73E8091800F0E947F4ABC0194
:1049500080915D0690915E060E94384064E776E0A3
:1049600080915D0690915E060E94C73E8091810F06
:104970000E947F4ABC0180915D0690915E060E9474
:10498000C73E2091810F80915D0690915E062B308D
:104990003CF4293054F4283069F463E676E007C02B
:1049A0002B3041F46FE676E002C069E676E00E94C3
:1049B000384002C00E9425406FE476E080915D0699
:1049C00090915E060E94C73E8091820F0E947F4AAE
:1049D000BC0180915D0690915E060E94C73E2091C9
:1049E000820F80915D0690915E062B303CF4293059
:1049F00054F4283069F46EE376E007C02B3041F4BC
:104A00006AE476E002C064E476E00E94384002C0C6
:104A10000E9425406AE276E080915D0690915E06F4
:104A20000E94C73E20918F0F80915D0690915E0697
:104A3000222319F062E276E002C060E176E00E9493
:104A4000C73E20914C0E80915D0690915E06222318
:104A500019F065E076E002C069EF75E00E94C73E9C
:104A600080915D0690915E060E9425400E94E56C53
:104A700080915D0690915E06DC01ED91FC910284CF
:104A8000F385E02D199580910002823011F40C9489
:104A9000F62DF090A60F0091A90F11E080915D0610
:104AA00090915E060E9425400E94906665E679E03E
:104AB00080915D0690915E060E9438400E9490664B
:104AC0006CE479E080915D0690915E060E94C73E9D
:104AD000E091BC0FE6300CF0E0E081EE96E09A83C6
:104AE00089838CED96E09C838B8382ED96E09E8398
:104AF0008D838EEC96E098878F838AEB96E09A8779
:104B0000898788EA96E09C878B87EE0FFF0B81E010
:104B100090E08C0F9D1FE80FF91F608171818091DB
:104B20005D0690915E060E94384063E379E08091D3
:104B30005D0690915E060E94C73E609100028091E2
:104B40005D0690915E060E94EC786AE179E08091C2
:104B50005D0690915E060E94C73E8F2D0E945766AB
:104B6000FF2009F44BC060E179E080915D069091EF
:104B70005E060E94C73E80915D0690915E061123FD
:104B800039F06091A70F0E94417A9091A70F06C05B
:104B90006091AD0F0E94417A9091AD0F8091AB1260
:104BA00098130C94FD2D64EF78E080915D06909150
:104BB0005E060E94C73E80915D0690915E061123BD
:104BC00039F06091A80F61110CC06FEE78E006C05B
:104BD0006091AE0F611105C06AEE78E00E94C73E99
:104BE00005C0062E000C770B0E945B7A68EE78E019
:104BF00080915D0690915E060E94C73E80915D06A1
:104C000090915E060E9425406FEC78E080915D06F1
:104C100090915E060E94C73E802F0E945766002337
:104C200009F44AC065EC78E080915D0690915E06DB
:104C30000E94C73E80915D0690915E06112339F077
:104C40006091AA0F0E94417A9091AA0F06C06091CC
:104C5000B00F0E94417A9091B00F8091AD129813DD
:104C6000E6C769EA78E080915D0690915E060E9451
:104C7000C73E80915D0690915E06112339F06091E8
:104C8000AB0F61110CC064EA78E006C06091B10F0F
:104C9000611105C06FE978E00E94C73E05C0062E8D
:104CA000000C770B0E945B7A6DE978E080915D06DD
:104CB00090915E060E94C73E80915D0690915E06CF
:104CC0000E94254064E878E080915D0690915E0640
:104CD0000E94C73E8091C50F811103C00E94656686
:104CE00035C069EE76E080915D0690915E060E9487
:104CF000C73E61E878E080915D0690915E060E9473
:104D0000C73E6091C50F80915D0690915E060E943E
:104D1000417A61E778E080915D0690915E060E949D
:104D2000C73E4091C60F5091C70F60E070E02AE087
:104D300080915D0690915E060E94003F6CE678E0EF
:104D400080915D0690915E060E94384063E578E0B0
:104D500080915D0690915E060E94C73E8091BD0FD6
:104D60008436C8F46CE478E080915D0690915E062C
:104D70000E94C73E6091BD0F80915D0690915E06D6
:104D80000E94417A6AE478E080915D0690915E0627
:104D90000E94384003C080E00E94656661E378E0CD
:104DA00080915D0690915E060E94C73E8091BE0F85
:104DB0008436C8F46AE278E080915D0690915E06E0
:104DC0000E94C73E6091BE0F80915D0690915E0685
:104DD0000E94417A68E278E080915D0690915E06DB
:104DE0000E94384003C080E00E9465666FE078E072
:104DF00080915D0690915E060E94C73E2091560606
:104E000080915D0690915E06222319F068E078E0BB
:104E100002C06EEF77E00E94384065EE77E0809147
:104E20005D0690915E060E94C73E6091B30F70913F
:104E3000B40F072E000C880B990B0E94B8B020E02D
:104E400030E04AE754E40E9411ADAB01BC0121E01F
:104E500080915D0690915E060E94483F60EE77E08B
:104E600080915D0690915E060E94384067EC77E085
:104E700080915D0690915E060E94C73E6091B50FDD
:104E80007091B60F072E000C880B990B0E94B8B0DA
:104E900020E030E04AE754E40E9411ADAB01BC01D0
:104EA00021E080915D0690915E060E94483F62EC91
:104EB00077E080915D0690915E060E94384069EA35
:104EC00077E080915D0690915E060E94C73E6091FA
:104ED000B70F7091B80F072E000C880B990B0E942A
:104EE000B8B020E030E04AE754E40E9411ADAB01D5
:104EF000BC0121E080915D0690915E060E94483FD2
:104F000064EA77E080915D0690915E060E943840E9
:104F10006BE877E080915D0690915E060E94C73E47
:104F20009091BC0F913011F09430F9F48091B90F49
:104F30000E9457668091B90F882329F167E877E0CE
:104F400080915D0690915E060E94C73E6091BA0F07
:104F500080915D0690915E060E94417A65E877E057
:104F600080915D0690915E060CC020915D063091A7
:104F70005E06953019F468E777E002C063E677E0F3
:104F8000C9010E94C73E80915D0690915E060E9415
:104F900025406AE477E080915D0690915E060E946C
:104FA000C73E9091BC0F2FEF290F80915D06909125
:104FB0005E06223028F46091BB050E94EC7804C0A4
:104FC00065E377E00E9438406CE177E080915D0610
:104FD00090915E060E94C73E8091C90F0E9457665D
:104FE0008091C90F882341F16AE077E080915D06E6
:104FF00090915E060E94C73E6091CA0F80915D0647
:1050000090915E060E94417A62EF76E080915D06A3
:1050100090915E060E94C73E6091CB0F80915D0625
:1050200090915E060E94417A60EF76E080915D0685
:1050300090915E060E94C73E80915D0690915E064B
:105040000E9425400E94E56C80915D0690915E066D
:10505000DC01ED91FC910284F385E02D199580919E
:105060005D0690915E060E9425400E9490666EEE5D
:1050700079E080915D0690915E060E9438400E9422
:1050800090666DEC79E080915D0690915E060E94DD
:10509000C73E8091890F8436C8F466EC79E0809130
:1050A0005D0690915E060E94C73E6091890F8091D7
:1050B0005D0690915E060E94417A64EC79E08091F1
:1050C0005D0690915E060E94384003C080E00E9419
:1050D000656663EA79E080915D0690915E060E94C4
:1050E000C73E8091880F8436C8F46CE979E08091DE
:1050F0005D0690915E060E94C73E6091880F809188
:105100005D0690915E060E94417A6AE979E080919D
:105110005D0690915E060E94384003C080E00E94C8
:10512000656669E779E080915D0690915E060E9470
:10513000C73E6091910F7091920F1616170614F5E5
:1051400000915D0610915E06072E000C880B990BEE
:105150000E94B8B020E030E04AE754E40E9411AD6C
:10516000AB01BC0122E0C8010E94483FC8010E9477
:10517000254064E779E080915D0690915E060E948B
:10518000384003C080E00E9465660E94E56C809113
:105190005D0690915E06DC01ED91FC910284F38541
:1051A000E02D199580915D0690915E060E94254044
:1051B0000E9490666EE57BE080915D0690915E06B0
:1051C0000E9438400E9490662091D90580915D062A
:1051D00090915E06222309F4BFC16FE27BE00E943A
:1051E000C73E0E9421670E9465660E942167209148
:1051F0005D0630915E06882389F06CE17BE0C90191
:105200000E94C73E8091DC050E947E85BC01809192
:105210005D0690915E060E9438404FC069E07BE0D9
:10522000C9010E94C73E8091D9050E947E85BC01BC
:1052300080915D0690915E060E94C73E8091DA05DE
:105240008823A9F161E07BE080915D0690915E0684
:105250000E94C73EE091DA05E4300CF0E0E08BEF0D
:1052600092E09A83898389EF92E09C838B8387EF16
:1052700092E09E838D8385EF92E098878F83EE0F77
:10528000FF0B81E090E08C0F9D1FE80FF91F6081FC
:10529000718180915D0690915E060E94C73E6FEF1E
:1052A0007AE080915D0690915E060E94C73E8091F3
:1052B0005D0690915E060E9425406CEE7AE080913A
:1052C0005D0690915E060E94C73E8091DB050091CD
:1052D0005D0610915E06882321F00E947E85BC0148
:1052E00002C068EE7AE0C8010E94384065ED7AE0BD
:1052F00080915D0690915E060E94C73E8091DC051C
:1053000000915D0610915E06882321F00E947E8543
:10531000BC0102C061ED7AE0C8010E9438406EEB2A
:105320007AE080915D0690915E060E94C73E809172
:10533000DE058823E1F068EB7AE080915D069091CC
:105340005E060E94C73E8091DD050E947E85BC01FD
:1053500080915D0690915E060E94C73E66E975E009
:1053600080915D0690915E060E94284003C080E017
:105370000E94656665EA7AE080915D0690915E061E
:105380000E94C73E8091DF058823E1F06FE97AE053
:1053900080915D0690915E060E94C73E8091DD057A
:1053A0000E947E85BC0180915D0690915E060E9400
:1053B000C73E66E975E080915D0690915E060E94A9
:1053C000284003C080E00E9465666CE87AE0809126
:1053D0005D0690915E060E94C73EE091E005E230D6
:1053E0000CF0E2E084E39AE09A83898388E29AE011
:1053F0009C838B8380E29AE09E838D83EE0FFF0B6C
:10540000A1E0B0E0AC0FBD1FEA0FFB1F608171810E
:1054100080915D0690915E060E94384069E77AE0CF
:1054200080915D0690915E060E94C73EE091D20594
:10543000E4300CF0E4E089E19AE09A83898383E127
:105440009AE09C838B838CE09AE09E838D8386E038
:105450009AE098878F838EEF99E09A878987EE0F7D
:10546000FF0B81E090E08C0F9D1FE80FF91F60811A
:10547000718180915D0690915E060E94384067E7D9
:105480007AE080915D0690915E060E94C73E609131
:10549000D70580915D0690915E060E94417A68E68C
:1054A0007AE080915D0690915E060E94C73E8091F1
:1054B000D205811110C06091D80580915D06909150
:1054C0005E060E94417A6DE57AE080915D069091DA
:1054D0005E060E94C73E6091D3057091D405072EE9
:1054E000000C880B990B0E94B8B020E030E04AE72E
:1054F00054E40E9411ADAB01BC0121E080915D0636
:1055000090915E060E94483F6FE47AE080915D06CC
:1055100090915E060E94C73E6091D5057091D605B8
:10552000072E000C880B990B0E94B8B020E030E0E9
:105530004AE754E40E9411ADAB01BC0121E0809127
:105540005D0690915E060E94483F60E47AE080919B
:105550005D0690915E0602C062E47BE00E943840E6
:105560000E94E56C80915D0690915E06DC01ED91F4
:10557000FC910284F385E02D199580915D06909150
:105580005E060E9425400E9490666CED7BE0809153
:105590005D0690915E060E9438400E9490666FEC16
:1055A0007BE080915D0690915E060E94C73EE0918F
:1055B000D20FE5300CF0E5E08DEB9BE09A83898318
:1055C00086EA9BE09C838B8384E99BE09E838D83AA
:1055D00085E89BE098878F8382E79BE09A8789879D
:1055E0008AE69BE09C878B87EE0FFF0B81E090E0C3
:1055F0008C0F9D1FE80FF91F6081718180915D06FE
:1056000090915E060E9438400E94E56C80915D0694
:1056100090915E06DC01ED91FC910284F385E02D12
:10562000199580915D0690915E060E9425400E942A
:1056300090666CE57CE080915D0690915E060E942C
:1056400038400E9490662091BB0680915D06909143
:105650005E062223C9F165E27CE00E94C73E80918C
:105660005D0690915E060E94254066E07CE0809198
:105670005D0690915E060E94C73E8091CC0F0E940D
:1056800057668091CC0F81110E94F68A80915D0649
:1056900090915E060E94254067EE7BE080915D065A
:1056A00090915E060E94C73E8091CE0F0E94576681
:1056B0008091CE0F81110E94C88A80915D069091E1
:1056C0005E060E94254004C067E47CE00E943840EA
:1056D0000E94E56C80915D0690915E06DC01ED9183
:1056E000FC910284F385E02D199587E295E6A1E00F
:1056F000BB278BAB9CABADABBEAB80915D069091F5
:105700005E060E9425400E94906662EE7DE08091D8
:105710005D0690915E060E9438400E94906669EC9A
:105720007DE080915D0690915E060E94C73E2091CB
:105730009D0A80915D0690915E06222319F065EC2A
:105740007DE002C060EC7DE00E94384080919D0ABF
:10575000882349F167EA7DE080915D0690915E06BD
:105760000E94C73E6091D00F7091D10F072E000CA0
:10577000880B990B0E94B8B020E030E04AE754E46F
:105780000E9411ADAB01BC0122E080915D069091B9
:105790005E060E94483F62EA7DE080915D0690913E
:1057A0005E060E9438409AE0E92E9FE0F92E28E13B
:1057B000422E2CEF522E3AE0A32EB12C44E6C42EFA
:1057C000D12C5EE0252ED7012C91222309F4CCC1E7
:1057D000F7013297008111810115110509F4C4C147
:1057E00080EB94E6A1E0BB27820F911DA11DB11DA6
:1057F000ABBFFC01879133243394811101C0312C5C
:1058000020915D0630915E06C8010197849790F55E
:1058100062E87DE0C9010E94C73E09500C3148F49E
:10582000E02FF0E0EE0FFF1FE251FC4F608171812D
:1058300002C066E77CE080915D0690915E060E9462
:10584000C73E0C3130F4E02FF0E0EA5DFB4F808181
:1058500001C080E090E08858924F092E000CAA0BFE
:10586000BB0BABBFFC018791B22DB81B8B2F09F08E
:105870001CC11DC1C801845691098438934008F0A9
:105880003FC068E67DE0C9010E94C73EC801B6017D
:105890000E9471AC6130710531F06230710559F4CC
:1058A00064E67DE002C066E67DE080915D06909151
:1058B0005E060E94C73E0E94886680905D069090BA
:1058C0005E063320B1F0C8010E94CD6B811107C084
:1058D00060E67DE0C4010E94C73E87E0E6C08130FB
:1058E00009F0E5C06DE57DE0C4010E94C73E88E097
:1058F000DCC064E57DE0C4010E94C73E82E0D5C003
:10590000C801885E93408035964408F069C0C8019C
:1059100068EE73E00E9471AC4B0167E47DE0C90161
:105920000E94C73E2AE08216910410F40E9480660D
:10593000B40180915D0690915E060E945B7A0E94A0
:10594000886660905D0670905E06332009F442C060
:10595000C8010E94CD6B282F62E47DE0C3012FAB0C
:105960000E94C73E849CC001859C900D949C900D24
:105970001124800F911FB5010E9485AC80915D06B6
:1059800090915E062FA9633059F06530C9F06230FE
:1059900009F08DC0243008F063C169E37DE062C185
:1059A000233018F467E27DE05DC1233019F46EE125
:1059B0007DE058C1243008F47AC065E17DE052C131
:1059C000622F0E94417A6DE07DE080915D069091AA
:1059D0005E0648C164E07DE0C3010E94C73E44C04A
:1059E000C80188539A44883E934008F509338AE4F5
:1059F000180779F00A339AE4190791F008331A442A
:105A000009F055C065EF7CE0C9010E94C73E8FE0F8
:105A10004CC06AEE7CE0C9010E94C73E83E145C0EC
:105A200068ED7CE0C9010E94C73E8CE03EC0C80121
:105A300080529E44883E934020F4005261EC7CE00A
:105A400009C0C80188509245883E934078F40850B8
:105A50006AEA7CE0C9010E94C73E0A3010F40E9445
:105A60008066802F0E94DB6584E01FC0013FF5E562
:105A70001F0739F469E97CE0C9010E94C73E8DE047
:105A800014C0023F45E5140739F46CE87CE0C90115
:105A90000E94C73E81E109C0033F154541F46EE70E
:105AA0007CE0C9010E94C73E80E10E94728A6DE9D4
:105AB0007DE080915D0690915E060E94C73E62E99E
:105AC0007DE080915D0690915E060E94C73ED70101
:105AD0006C9170E080915D0690915E060E945B7A09
:105AE000F70180818A3020F482E00E94728A04C02B
:105AF000843610F40E9480660E948866D7014C911B
:105B0000B9E2B49FA0011124052E000C660B770B9F
:105B10008BA99CA9ADA9BEA9480F591F6A1F7B1F5D
:105B2000DE0111968A019B010F5F1F4F2F4F3F4FE0
:105B30006BBFFA0187918D93B901A8018111F2CF52
:105B4000BE016F5F7F4F80915D0690915E060E945F
:105B5000284080915D0690915E06DC01ED91FC91FC
:105B60000284F385E02D1995B3E0EB0EF11CE2E819
:105B7000EE16EFE0FE0609F026CE0E94E56C80915D
:105B80005D0690915E06DC01ED91FC910284F38547
:105B9000E02D199580915D0690915E060E9425404A
:105BA0000E94906663E47EE080915D0690915E06BF
:105BB0000E9438400E94906660E37EE080915D061E
:105BC00090915E060E94C73E0E940C4720E030E0A4
:105BD00040E050E40E94B2B020915D0630915E0634
:105BE00087FF43C06DE27EE0C9015DC0F090AC0F5D
:105BF0000091AF0F10E00C944E2561E079E08091A8
:105C00005D0690915E060E94C73E6091AB12809146
:105C10005D0690915E060E94417A6FEF78E0809178
:105C20005D0690915E060E94C73E0C94D32566EBFC
:105C300078E080915D0690915E060E94C73E60917B
:105C4000AD1280915D0690915E060E94417A64EBF0
:105C500078E080915D0690915E060E94C73E01C883
:105C600060E37DE00E94C73E22CF69E27EE0C90189
:105C70000E94384066E17EE080915D0690915E066C
:105C80000E94C73E0E940C47AB01BC0122E08091FC
:105C90005D0690915E060E94483F64E17EE080913F
:105CA0005D0690915E060E94384061E07EE0809142
:105CB0005D0690915E060E94C73E809119100E9479
:105CC00057662091191080915D0690915E062223FF
:105CD00079F06EEF7DE00E94C73E0E94B18A64EFCA
:105CE0007DE080915D0690915E060E94384002C082
:105CF0000E9425400E94E56C80915D0690915E06B1
:105D0000DC01ED91FC910284F385E02D19958091E1
:105D10005D0690915E060E9425400E9490666BE9A8
:105D20007EE080915D0690915E060E9438400E9460
:105D3000906667E87EE080915D0690915E060E9425
:105D4000C73E4091091050910A1060910B1070915C
:105D50000C1080915D0690915E060E94487A63E780
:105D60007EE080915D0690915E060E94C73E409164
:105D700011105091121060911310709114108091B5
:105D80005D0690915E060E94487A6FE57EE0809104
:105D90005D0690915E060E94C73E40910D105091A5
:105DA0000E1060910F107091101080915D0690910F
:105DB0005E060E94487A6BE47EE080915D069091D9
:105DC0005E060E94C73E40911510509116106091DA
:105DD00017107091181080915D0690915E060E94D8
:105DE000487A0E94E56C80915D0690915E06DC0128
:105DF000ED91FC910284F385E02D199580915D066B
:105E000090915E060E9425400E949066E7960FB62C
:105E1000F894DEBF0FBECDBFDF91CF911F910F91E0
:105E2000FF90EF90DF90CF90BF90AF909F908F90BA
:105E30007F906F905F904F903F902F9008952F929A
:105E40003F924F925F926F927F928F929F92AF920A
:105E5000BF92CF92DF92EF92FF920F931F93CF9357
:105E6000DF93CDB7DEB7C65AD1090FB6F894DEBFBF
:105E70000FBECDBFCDB6DEB6CC55DF4F1882C45AAB
:105E8000D040CD55DF4F1882C35AD0408091FB0CD3
:105E90008A3709F447C0C0F4873709F4D9C238F407
:105EA0008F3109F435C5863709F4E2C1F7C5883763
:105EB00009F4DDC2893709F0F1C50E94FD830E9413
:105EC000ED432B013C0129C08E3709F42EC338F471
:105ED0008B3709F4CAC18C3709F4D8C2DFC58138C1
:105EE00009F407C5823809F4EDC4803809F0D6C535
:105EF00065C40E94ED43DC01CB0184199509A60914
:105F0000B70980329340A105B10508F00CC50E9485
:105F1000294F0E94FD830E944B550E943F840297A7
:105F200041F701C50E943F84029729F060E084E8B0
:105F30000E9457908BC18091A20A823031F0833049
:105F400039F482E08093320D03C081E080935712D0
:105F500081E08093050D8E010C551F4F2BE0AE01A3
:105F600044575F4F68E871E90E94D48F0E941484FF
:105F7000893058F0015011092BE0AE014F575F4FA7
:105F800068E872E981E00E94D48F1092040D7724B2
:105F900073940E942A84882309F43DC119822296B1
:105FA0001FAE22978091040D81110EC0BE0164576F
:105FB0007F4FCE018F5B9F4F0E94D0AFCC55DF4FFC
:105FC0000881C45AD0400FC07092040DBE016F57B3
:105FD0007F4FCE018F5B9F4F0E94D0AFCD55DF4FDB
:105FE0000881C35AD0401091040DADB6BEB6809161
:105FF0009E0AEDB7FEB722E0829FE019F109112455
:106000000FB6F894FEBF0FBEEDBF8DB79EB70196D9
:106010007C016EEA75E0CE0183569F4F0E94883E58
:106020008091A20A823089F0833061F1813009F0D9
:10603000A1C040919E0A50E0B7018091301290912A
:1060400031120E94F75110E039C020919E0A30E0D1
:106050005FB7F89440E0842F90E08217930774F4C0
:10606000880F991FF701E80FF91FDC01AA5CBD4EEC
:106070008D919C91918380834F5FEDCF5FBF109294
:1060800056121CC020919E0A30E05FB7F89440E0A1
:10609000842F90E08217930774F4880F991FF701FB
:1060A000E80FF91FDC01A85CB24F8D919C919183A0
:1060B00080834F5FEDCF5FBF10922D126DE270E0D5
:1060C000CE0183569F4F0E94B73D20919E0A2930F2
:1060D00048F0112321F0113021F418E004C028E029
:1060E00001C020E010E0121758F5F701E10FF11D93
:1060F000E10FF11D608171814AE0CE0189569F4F09
:10610000CB55DF4F2883C55AD0400E945D3EBE016B
:1061100069567F4FCE0183569F4F0E94DE3DCE01D0
:1061200089569F4F0E94583ECE0183569F4F0E9432
:106130002D8B1F5FCB55DF4F2881C55AD040D3CF61
:1061400040E450E0BE016F5F7F4FCE0183569F4F0A
:106150000E94248BCF55DF4F1881C15AD040CE0109
:1061600083569F4F0E94583E0FB6F894BEBE0FBE96
:10617000ADBE0BC0CE0183569F4F0E94583E0FB656
:10618000F894BEBE0FBEADBE10E0BE016F5F7F4F84
:10619000CE018F5B9F4F0E94D0AF010F10E0E1E472
:1061A000F0E0EC0FFD1FE00FF11F1082BE016F5BEE
:1061B0007F4F8091C8129091C9120E94EB3EB801A6
:1061C000CE018F5B9F4F0E946855BC018091C81221
:1061D0009091C9120E945B7A6AE08091C8129091F6
:1061E000C9120E94C03E8091C8129091C912DC0170
:1061F000ED91FC910284F385E02D19950E941484A1
:10620000893048F08091040D811103C07092040D13
:1062100002C01092040D0E94FD830E944B550E9403
:10622000CA5E81110CDE8091FA0C81110FC0809141
:10623000050D882359F080912D0D811107C08091A3
:10624000F80C9091F90C0A970CF4A3CE8091A20A55
:10625000823039F0833009F021C481E08093320D1F
:106260001DC481E08093571219C41092050D4DC3CF
:106270001091FE0C8FEF810F853028F060E089E8E7
:106280000E9457900BC4133079F018F41230F9F0D3
:1062900004C0143079F0153099F040E6442E49E0FE
:1062A000542E612C712C19C0412C3BE4532E612CCF
:1062B000712C13C0412C26E9522E612C712C0DC07B
:1062C000412C92EC592E66246394712C06C080E810
:1062D000482E85E2582E612C712C00E0E12EF12C25
:1062E0005701BFE8AB0EB11C1501E89427F8332421
:1062F000E6E9EE0EF11CE894E7F8FF24023091F095
:1063000018F4013051F004C0033089F00430A1F0DA
:1063100040E659E060E070E013C040E855E260E01C
:1063200070E00EC040E05BE460E070E009C040E077
:1063300056E960E070E004C040E052EC61E070E0DB
:1063400089E597E00E94356389E597E00E94DC3C8F
:106350000E94ED434B015C01F2E38F0E911CA11CE6
:10636000B11C0E940B550E94ED43681579058A0502
:106370009B05B8F360E870E089E597E00E94BF6094
:106380006FE070E089E597E00E94BF60612F89E5CA
:1063900097E00E94963CB10189E597E00E94BF60BA
:1063A0000E94ED434B015C012AE0820E911CA11C6E
:1063B000B11C0E940B550E94ED43681579058A05B2
:1063C0009B05B8F367E870E089E597E00E94BF603D
:1063D0006FE070E089E597E00E94BF60612F89E57A
:1063E00097E00E94963CB70189E597E00E94BF6064
:1063F00089E597E00E94DC3C0E94ED434B015C0183
:106400003EE5830E31E0931EA11CB11C0E940B558A
:106410000E94ED43681579058A059B05B8F30F5F67
:10642000053009F06BCFB301A20189E597E00E9426
:1064300035634092111050921210609213107092B6
:106440001410B301A2018AEA91E00E94608B5DC240
:1064500083E090E00E94B2AD2AE0DC012C9329E5B4
:1064600037E012963C932E9311976AE00CC083E0BC
:1064700090E00E94B2AD2DE0FC01208329E537E0D9
:10648000328321836DE00E9453513FC24091FE0C44
:106490005091FF0C0091000D1091010D6091FC0CCA
:1064A0007091FD0CCE010196CB55DF4F4883C55A44
:1064B000D040CA55DF4F5883C65AD0400E94288921
:1064C000CB55DF4F4881C55AD040CA55DF4F588160
:1064D000C65AD040892BE9F08D81873050F4853041
:1064E00080F48130B0F0642F8B819C810E94C67A49
:1064F0000DC0893070F4B8018B819C810E94608B43
:1065000005C0BA018B819C810E9438790E94D3908A
:1065100004C061E085E80E9457908091F70C8111DA
:10652000BDC281E08093F70CB9C2B090FC0CE09042
:10653000FD0CC956DF4F1882C759D0406EEA75E08E
:10654000CE018F579F4F0E94883E6B2D7E2DCE012E
:1065500084579F4F0E942889892B09F4C9C0C057CE
:10656000DF4FE881C059D0404E2F50E0FA013197FB
:10657000E830F10508F0BCC08827ED5DFE4F8F4F75
:106580000C9498ACC257DF4F88819981CE58D04087
:106590000E94DBB123961FAE1EAE239725961FAE39
:1065A0001EAE259727961FAE1EAE27974AE0BE0166
:1065B0006F5F7F4F90E03EC0C257DF4F8881998167
:1065C000CE58D0400E94DBB1682F880F770B4AE08D
:1065D0000AC0C257DF4F88819981CE58D0400E94AF
:1065E000E8B14AE0BC01CE0101960E945D3EBE01C9
:1065F0006F5F7F4FCE018F579F4F0E947E3DCE0130
:10660000019663C0C257DF4F88819981CE58D04030
:106610000E94E8B123961FAE1EAE239725961FAEAB
:106620001EAE259727961FAE1EAE27974AE0BE01E5
:106630006F5F7F4F0E9489B035C0C257DF4F88819E
:106640009981CE58D0400E94E3B123961FAE1EAE72
:10665000239725961FAE1EAE259727961FAE1EAE1A
:1066600027972AE0AE014F5F5F4F0E945AB01AC0D1
:10667000C257DF4F88819981CE58D0400E94E3B144
:1066800023961FAE1EAE239725961FAE1EAE2597EE
:1066900027961FAE1EAE27972AE0AE014F5F5F4FD1
:1066A0000E9468B0BE016F5F7F4FCE018F5B9F4F2E
:1066B0000E94383EBE016F5B7F4FCE018F579F4FC8
:1066C0000E947E3DCE018F5B9F4F0E94583E4BE063
:1066D00050E0BE016F5B7F4FCE018F579F4F0E94EE
:1066E000248BCB57DF4FF880C558D04011E002C053
:1066F000F12C10E0CE018F579F4F0E94583E11237E
:1067000009F4BCCD8E0109561F4F20E4AE014F5F46
:106710005F4F68E87B2D8E2D0E94D48FBE016F5B8A
:106720007F4FCE0101960E94D0AFC956DF4F8881BE
:10673000C759D040F80E81E08F0DC956DF4F8883CE
:10674000C759D040E1E0F0E0EC0FFD1FEF0DF11D67
:106750009CE79083E1E0F0E0EC0FFD1FE80FF11DF6
:106760001082BE016F5F7F4F8091C8129091C91255
:106770000E94EB3EC956DF4F6881C759D04070E098
:10678000CE0101960E946855BC018091C81290917B
:10679000C9120E945B7A6AE08091C8129091C91276
:1067A0000E94C03E8091C8129091C912DC01ED9107
:1067B000FC910284F385E02D199570C18091FC0C49
:1067C0009091FD0C8038910509F068C18E01045745
:1067D0001F4F20E4AE014F5F5F4F68E870E880E034
:1067E0000E94D48F6EE875E0CE018F579F4F0E94B4
:1067F000883ECE018F579F4F0E942D8BC457DF4F8D
:106800002881CC58D040CB57DF4F88819981C5581B
:10681000D040820F911DC457DF4F8883CC58D040A1
:1068200022961FAE22974BE050E0BE016F5B7F4F78
:10683000CE018F579F4F0E94647CBE016F5B7F4FDC
:10684000CE0101960E94D0AFC457DF4F8881CC584B
:10685000D040E1E0F0E0EC0FFD1FE80FF11D1082E9
:10686000BE016F5F7F4F8091C8129091C9120E9444
:10687000EB3EC457DF4F6881CC58D04070E0CE016A
:1068800001960E946855BC018091C8129091C9126E
:106890000E945B7A6AE08091C8129091C9120E94AE
:1068A000C03E8091C8129091C912DC01ED91FC911B
:1068B0000284F385E02D1995CE018F579F4F0E94DA
:1068C000583EECC08091FC0C9091FD0C82389105F3
:1068D00009F0E4C08E0104571F4F20E4AE014F5F62
:1068E0005F4F68E872E880E00E94D48F68E975E045
:1068F0007BCF8091FC0C9091FD0C8138910509F0C3
:10690000CDC08091050D8111C9C00E94D390C6C031
:106910008091FC0C9091FD0C4F9709F0BFC081E075
:106920008093FA0CBBC00E943F84029719F060E08C
:1069300084E8A6CC8091A10A811102C00E94E07A6D
:106940000E941484F82E6EEA75E0CE0184579F4FA2
:106950000E94883EC956DF4F1882C759D0408E0129
:1069600009561F4F20E4AE014F5F5F4F68E879E79B
:1069700080E00E94D48FCF57DF4F19821882C15810
:10698000D040CD57DF4F19821882C358D040CB5723
:10699000DF4F19821882C558D0406F2D70E080E01B
:1069A00090E02AE0AE014F5B5F4F0E945AB0BE01FB
:1069B0006F5B7F4FCE018F579F4F0E94383EBE01C5
:1069C0006F577F4FCE0184579F4F0E947E3DCE016F
:1069D0008F579F4F0E94583E4BE050E0BE016F5BC7
:1069E0007F4FCE0184579F4F0E94647CC057DF4F7A
:1069F0001881C059D040BE016F5B7F4FCE01019618
:106A00000E94D0AFC956DF4F8881C759D040810F4F
:106A100091E0980FC956DF4F9883C759D040E1E005
:106A2000F0E0EC0FFD1FE80FF11D8CE78083E1E043
:106A3000F0E0EC0FFD1FE90FF11D1082BE016F5F4A
:106A40007F4F8091C8129091C9120E94EB3EC956A7
:106A5000DF4F6881C759D04070E0CE0101960E9497
:106A60006855BC018091C8129091C9120E945B7A4E
:106A70006AE08091C8129091C9120E94C03E809134
:106A8000C8129091C912DC01ED91FC910284F3854A
:106A9000E02D1995CE0184579F4F11CF0FB6F89472
:106AA000DEBE0FBECDBECA55DF4F0FB6F894DEBFB7
:106AB0000FBECDBFDF91CF911F910F91FF90EF904F
:106AC000DF90CF90BF90AF909F908F907F906F900E
:106AD0005F904F903F902F9008958091100D90916E
:106AE000110D91609093110D8093100D0895809178
:106AF000100D9091110D80689093110D8093100DE1
:106B000008958091100D9091110D80619093110D59
:106B10008093100D0895FC018281882371F0838198
:106B2000882359F013828091100D9091110D24E06B
:106B300082279093110D8093100D0895FC0182819E
:106B4000882371F0838181110BC081E08383809160
:106B5000100D9091110D84609093110D8093100D84
:106B60000895FC018481882371F08581882359F080
:106B700015828091100D9091110D28E0822790933D
:106B8000110D8093100D0895FC018481882371F00C
:106B9000858181110BC081E085838091100D9091DA
:106BA000110D88609093110D8093100D08958091C0
:106BB000100D9091110D20E282279093110D80937A
:106BC000100D08958091100D9091110D8062909399
:106BD000110D8093100D0895DC01ED91FC9106805C
:106BE000F781E02D60E070E0199477FF03C07195A4
:106BF000619571096F3F710519F014F06FEF70E046
:106C00008091100D9091110D8C7B91709093110DCE
:106C10008093100D8091100D9091110D6F307105C2
:106C200014F480641FC06733710514F481641AC0C2
:106C30006F3571051CF48164906114C0673871056B
:106C40001CF4816490630EC06F3A71051CF481647A
:106C5000906408C0673D71051CF48164906502C0B2
:106C6000816490669093110D8093100D089580E0DB
:106C700094E09093110D8093100D08958091100D64
:106C80009091110D92609093110D8093100D809151
:106C9000100D9091110D80649093110D8093100D43
:106CA00008950895089508950895089508950895FC
:106CB00008950895089580E0089508950895089529
:106CC00008950895089508950895089508950895DC
:106CD00008950895089580E0089508950895FC01A9
:106CE00064830895FC0162830895FC011382148279
:106CF00015821682178210860895089508950895C2
:106D0000FC0183810895FC0164830895FC0167837D
:106D10000895FC0165830895FC0182810895FC01BA
:106D2000128213821482158261E086E10E946E4213
:106D300061E086E10E943F42E2E7F0E0808181600D
:106D400080831092110D1092100D0895FF920F93F1
:106D50001F93CF93DF938C01C62FF42ED22F6AEDB1
:106D600070E0DC0119968D919C911A970E94BF608A
:106D7000F80181859285DC01ED91FC910190F08113
:106D8000E02D6C2F1995F80181859285DC01ED913C
:106D9000FC910190F081E02D6F2D1995F80181850E
:106DA0009285DC01ED91FC910190F081E02D6D2F39
:106DB0001995EC2FF0E0BF0166527F4F6F0D711DEA
:106DC0006D0F711D6F777727F80181859285DF91AF
:106DD000CF911F910F91FF900C94BF6020E040E095
:106DE000B5CF65E4FBCF68E4F9CFCF93DF93FC0127
:106DF0002381222321F0EC0161E4F0DF1B82DF918B
:106E0000CF910895CF93DF93FC012381211105C019
:106E1000EC0160E4E3DF81E08B83DF91CF910895A3
:106E2000FC012481222311F06CE3D8CF0895FC01EA
:106E30002781222331F02085222319F010866BE36D
:106E4000CDCF0895FC012781222339F0208521111F
:106E500004C021E020876AE3C1CF0895FC012581A9
:106E6000222331F02681222319F0168269E3B6CF5E
:106E70000895FC012581222339F02681211104C0C7
:106E800021E0268368E3AACF089567E3A7CF6AE4E9
:106E9000A5CF69E4A3CF66E3A1CF65E39FCF6EE4FE
:106EA0009DCF64E39BCF63E399CF62E397CF61E328
:106EB00095CF60E393CF6FE291CF6DE28FCF6CE21D
:106EC0008DCF242F462F6CE441CF77FF03C07195FF
:106ED0006195710920E0462F6EE238CF462F20E001
:106EE00067E434CF462F20E066E430CF262F64E4F9
:106EF0002DCFCF92DF92FF920F931F93CF93DF930B
:106F00008C01F62E443F81E0580738F0413187E28A
:106F1000580728F040E157E202C044EF51E0243F17
:106F200081E0380738F0E9012131374228F0C0E12B
:106F3000D7E202C0C4EFD1E0CA01845F914022E3EE
:106F4000C22ED12CB6010E9471AC462F2F2D62E4C7
:106F5000C801FCDECE01845F9140B6010E9471AC95
:106F6000462F2F2D63E4C801DF91CF911F910F9120
:106F7000FF90DF90CF90EACE262F40E06FE3E6CE81
:106F8000262F40E06EE3E2CE262F40E06DE3DECE1A
:106F9000462F20E06DE4DACEFC016283611104C06B
:106FA00020E040E06BE4D2CE089577FF03C07195F6
:106FB0006195710920E0462F6BE4C8CE4F925F9235
:106FC0006F927F928F929F92AF92BF92CF92DF92F9
:106FD000EF92FF920F931F93CF93DF936C01A4EC7A
:106FE000CA1AADEFDA0AD601ED91FC917E970CF04A
:106FF0005DC0FC01E858FF4F812C912CA191B1910B
:10700000AB2B21F42115310549F450C0BFEF8B1A89
:107010009B0AAEE18A16910489F748C0EC0154013D
:10702000AA0CBB1CAA0CBB1CAC0EBD1EF501EC547B
:10703000FF4F40835183628373837401EE0CFF1C06
:10704000EC0EFD1EF701E858FF4F31832083EC540E
:10705000FF4F11830083BE01680D791DFB01EC55C4
:10706000FE4F81E080830E94ED43F50160837183D0
:1070700082839383C65CDD4F88819981F701E2505A
:10708000FE4F91838083D6012D913C9111972F5F04
:107090003F4F2D933C939C012F5F3F4F12161306D9
:1070A00014F021E030E03983288302C08FEF9FEF96
:1070B000DF91CF911F910F91FF90EF90DF90CF90D4
:1070C000BF90AF909F908F907F906F905F904F9008
:1070D00008950F931F93CF93DF93EC0170932C0EC1
:1070E00060932B0E4093320E81E090E00E94B2AD8F
:1070F0008C010E94FE811093130D0093120D91E0FC
:107100009093080D9093130E1092070D1092060D98
:107110001092160E1092150E1092170E1092140E59
:1071200024EF31E030931E0E20931D0E28EB3BE040
:107130003093200E20931F0E20E233E03093250E73
:107140002093240E2CEA3DE03093270E2093260E48
:1071500028E037E030932E0E20932D0E24E931E104
:107160003093300E20932F0E10921A0E1092190E9B
:107170001092180E1092210E1092280E1092310EBD
:1071800010921C0E10921B0E1092230E1092220EC3
:1071900010922A0E1092290E988399839A83DF9178
:1071A000CF911F910F9108951F920F920FB60F92DA
:1071B00011240BB60F922F933F934F935F936F93CE
:1071C0007F938F939F93AF93BF93EF93FF938091A0
:1071D0000F0D8F5F80930F0D90910E0D891708F49E
:1071E00001C110920F0D80910D0D90E08730910537
:1071F00008F0F8C0FC018827E55DFE4F8F4F0C9426
:1072000098AC60E086E10E943F4288E080930E0DDA
:1072100081E048C061E086E10E943F4281E08093C6
:107220000E0D36C060E086E10E943F4280910B0D5A
:1072300090910C0D97FF05C083E080930E0D84E0C4
:1072400031C081E080930E0D83E02CC061E086E1C7
:107250000E943F4283E080930E0D80910A0D8F5F64
:1072600080930A0D803150F010920A0D85E01AC00B
:1072700061E086E10E943F4281E0EDCF80910B0DFD
:1072800090910C0D880F991F90930C0D80930B0D0E
:1072900082E008C060E086E10E943F4281E0809386
:1072A0000E0D86E080930D0D9DC061E086E10E9489
:1072B0003F4288E180930E0D8091100D9091110D49
:1072C00090930C0D80930B0D8091100D9091110DEA
:1072D00091FF1DC08091090D8823B1F08091100DA0
:1072E0009091110D22E092279093110D8093100D33
:1072F0008091100D9091110D80649093110D8093E9
:10730000100D1092090D03C081E08093090D80914A
:10731000100D9091110D92FF0EC08091090D8823E0
:1073200039F01092110D1092100D1092090D03C03A
:1073300081E08093090D8091100D9091110D84FFD3
:1073400014C08091090D882369F08091100D9091EF
:10735000110D20E182279093110D8093100D109252
:10736000090D03C081E08093090D8091100D90916B
:10737000110D87FF13C08091090D882361F0809162
:10738000100D9091110D80589093110D8093100D58
:107390001092090D03C081E08093090D8091100DBA
:1073A0009091110D90FF14C08091090D882369F010
:1073B0008091100D9091110D21E092279093110D65
:1073C0008093100D1092090D03C081E08093090D88
:1073D0008091100D9091110D90930C0D80930B0DD9
:1073E00010920D0DFF91EF91BF91AF919F918F91F1
:1073F0007F916F915F914F913F912F910F900BBEB5
:107400000F900FBE0F901F901895DC01A250BE4F39
:1074100020E030E04D915D914617570739F4280F71
:10742000391FF901EC55FE4F808108952F5F3F4FC2
:107430002E31310579F780E00895CF93DF93EC0189
:10744000C45CDD4FA881B981109709F442C0FC01EA
:10745000E250FE4F20E030E041915191461757072E
:1074600099F5A901440F551F480F591FFA01E85813
:10747000FF4F60817181672B61F111821082FC01E5
:10748000E20FF31FEC55FE4F1082FA01EE53FE4F50
:1074900011821082235D3F4F220F331F220F331FB3
:1074A000FC01E20FF31F1082118212821382FA0193
:1074B000E859FE4F11821082EA56FF4F1182108266
:1074C0001197B983A88305C02F5F3F4F2E31310537
:1074D00019F6DF91CF9108950F931F9301E010E00B
:1074E0006DDD1F910F9108951092080D24ED3BE37F
:1074F00044EF51E060E070E080912B0E90912C0EF3
:10750000EBDF9093070D8093060D08950F931F9363
:1075100000E010E053DD1F910F9108952F923F92EC
:107520004F925F926F927F928F929F92AF92BF9293
:10753000CF92DF92EF92FF920F931F93CF93DF933F
:1075400000D000D0CDB7DEB78C010E94ED4398018A
:107550002E533E4F3C832B831E830D83D801AC55A5
:10756000BE4FBA83A9831801B2E02B1ABEEF3B0AC3
:10757000F901AA24A394B12C32E0832E912C11821C
:1075800010829F012A543140D9012D913C91232B27
:1075900009F44DC0AD81BE812D913D914D915C911D
:1075A00013977D01B4EBEB0EF11CD701CD90DD906C
:1075B000ED90FC902B013C01421A530A640A750AB3
:1075C0004C145D046E047F0490F1C20ED31EE41EC1
:1075D000F51EAD81BE81CD92DD92ED92FC921397A6
:1075E000A981BA812C91222311F19F0126593109D9
:1075F000D9012D913C912115310519F4B182A08258
:1076000016C07F01BAE5EB1AF108D7014D915C91E4
:107610001197421753075CF4B182A0824F5F5F4F0E
:107620004D935C934217530714F0918280823296F7
:107630002D813E812C5F3F4F3E832D83A981BA81EE
:107640001196BA83A983E215F30509F098CFEB816F
:10765000FC8181919191FC83EB838130910599F0BC
:107660000297C9F4EB81FC81EC54F1400190F08168
:10767000E02D1995AB81BC81DA966D917C91DB97F9
:10768000C801DBDE08C0EB81FC81EC54F1400190C5
:10769000F081E02D19952B813C8122153305B9F637
:1076A00026960FB6F894DEBF0FBECDBFDF91CF9107
:1076B0001F910F91FF90EF90DF90CF90BF90AF9010
:1076C0009F908F907F906F905F904F903F902F9002
:1076D00008956E3E22E0720738F06B3C98E079071F
:1076E00028F06AEC78E002C06EEE72E0660F771F59
:1076F0009FB7F89425E1829FF0011124EF5AFE4EC6
:10770000748363839FBF08956E3E22E0720738F052
:107710006B3C98E0790728F06AEC78E002C06EEEE6
:1077200072E0660F771F9FB7F89425E1829FF00102
:107730001124EF5AFE4E768365839FBF0895660F2E
:10774000771F282F30E095E1899FF0011124EF5A2F
:10775000FE4E858196816817790718F465817681D8
:1077600007C0838194818617970710F46381748121
:107770008FB7F89495E1929FF001939FF00D11243B
:10778000EF5AFE4E728361838FBF08958091320E4F
:10779000811109C08091080D882329F060ED77E000
:1077A00081E0CDDFA1CE089581E08093080D6CEDDE
:1077B00075E0C5CF6CED75E080E0C1CF0895CF9244
:1077C000DF92EF92FF920F931F93CF93DF936C01A1
:1077D0007A018B01C0E0D0E0CE15DF0589F0D80139
:1077E0006D918D01D601ED91FC910190F081E02D1C
:1077F000C6011995892B11F47E0102C02196ECCFA8
:10780000C701DF91CF911F910F91FF90EF90DF9013
:10781000CF900895FC01A089B1898C91A689B78980
:1078200082FD0FC09C91818D8F5F8F73228D821797
:1078300049F0218DDF01A20FB11D5D969C93818FD0
:1078400008958C910895FC01918D828D981761F0B7
:10785000828DDF01A80FB11D5D968C91928D9F5F87
:107860009F73928F90E008958FEF9FEF0895FC0132
:10787000918D828D981731F0828DE80FF11D858DE5
:1078800090E008958FEF9FEF0895FC01918D228D78
:10789000892F90E0805C9F4F821B91098F739927FD
:1078A00008958CEB96E0F1DF21E0892B09F420E0CC
:1078B000822F089589E597E0E8DF21E0892B09F41C
:1078C00020E0822F089586EF97E0DFDF21E0892B0B
:1078D00009F420E0822F089583E998E0D6DF21E0C3
:1078E000892B09F420E0822F0895FC01848DDF01AB
:1078F000A80FB11DA35ABF4F2C91848D90E0019623
:107900008F739927848FA689B7892C93A089B18911
:107910008C9180648C93938D848D981306C002881B
:10792000F389E02D80818F7D80830895EF92FF920F
:107930000F931F93CF93DF93EC0181E0888F9B8D92
:107940008C8D981305C0E889F989808185FD23C055
:10795000F62E0B8D10E00F5F1F4F0F731127E02ED7
:107960008C8DE8120BC00FB607FCFACFE889F989B5
:10797000808185FFF5CFCE01B8DFF2CF8B8DFE0180
:10798000E80FF11DE35AFF4FF0820B8FEA89FB8964
:107990008081806207C0EE89FF896083E889F98968
:1079A00080818064808381E090E0DF91CF911F919E
:1079B0000F91FF90EF900895CF93DF93EC01888DA6
:1079C0008823C1F0EA89FB89808185FD05C0A889EB
:1079D000B9898C9186FD0EC00FB607FCF5CF80816A
:1079E00085FFF2CFA889B9898C9185FFEDCFCE01B3
:1079F0007CDFE8CFDF91CF91089580E090E0892B84
:107A000019F06ADF811116C080E090E0892B19F02F
:107A10005ADF811112C080E090E0892B19F04ADF13
:107A200081110EC080E090E0892B79F03ADF81115E
:107A30000AC008950E940000E7CF0E940000EBCF2B
:107A40000E940000EFCF0C940000089590E0FC012C
:107A50003197E231F10508F04EC08827EE5CFE4F09
:107A60008F4F0C9498AC809180008F7703C08091E9
:107A700080008F7D80938000089580918000877FB3
:107A8000F9CF84B58F7702C084B58F7D84BD08950A
:107A90008091B0008F7703C08091B0008F7D80937C
:107AA000B0000895809190008F7707C0809190007A
:107AB0008F7D03C080919000877F80939000089510
:107AC0008091A0008F7707C08091A0008F7D03C0B8
:107AD0008091A000877F8093A0000895809120016D
:107AE0008F7707C0809120018F7D03C08091200196
:107AF000877F8093200108950E94C3AF0F931F9347
:107B0000CF93DF938C01EB01FC0180819181009781
:107B1000B1F0688179816115710579F042815381F5
:107B20002C813D814217530740F00E94DBAF8C81CE
:107B30009D81F8019583848313C00E9447AE88819C
:107B40009981F801918380838A819B8193838283C9
:107B50008C819D8195838483198218821B821A826D
:107B60001D821C82DF91CF911F910F9108950F9379
:107B70001F93CF93DF93EC0188819981009729F0BF
:107B80002A813B812617370788F48B016F5F7F4F6F
:107B90000E94DFAE009761F0998388831B830A837C
:107BA0002C813D81232B11F4FC01108281E001C066
:107BB00080E0DF91CF911F910F910895EF92FF9296
:107BC0000F931F93CF93DF93FB0124813581E080D6
:107BD000F180FC0104811581E114F10411F480E0CD
:107BE00016C02115310591F0EC01020F131FB801E9
:107BF000BEDF8823A1F3288139818C819D81B70163
:107C0000820F931F0E94DBAF1D830C8381E0DF9105
:107C1000CF911F910F91FF90EF900895EF92FF92F7
:107C20000F931F93CF93DF93EC017B018A01BA017D
:107C30009EDF2881398181110DC02115310519F090
:107C4000C9010E9447AE198218821D821C821B82C4
:107C50001A8206C01D830C83B701C9010E94DBAFE5
:107C6000CE01DF91CF911F910F91FF90EF9008957A
:107C7000CF93DF93EC016115710551F0FB01019089
:107C80000020E9F73197AF01461B570BC7DF0CC047
:107C900088819981009711F00E9447AE198218825D
:107CA0001D821C821B821A82CE01DF91CF91089522
:107CB000FC01808191810C9447AE0F931F93CF9369
:107CC000DF93CDB7DEB762970FB6F894DEBF0FBE75
:107CD000CDBF8C01CB01F801118210821382128278
:107CE0001582148250E0BE016F5F7F4F0E9446B044
:107CF000BE016F5F7F4FC801BBDF62960FB6F8947D
:107D0000DEBF0FBECDBFDF91CF911F910F910895C0
:107D1000FC01118210821382128215821482611575
:107D2000710549F0FB0101900020E9F73197AF019F
:107D3000461B570B73CF0895CF93DF9300D01F924C
:107D4000CDB7DEB7611571058105910579F09B010D
:107D5000AC0169833A834B835C830E943AB02981EA
:107D60003A814B815C810E94FBB103C060E070E00E
:107D7000CB010F900F900F900F90DF91CF9108954E
:107D8000DC01ED91FC910190F081E02D1994EF92CE
:107D9000FF920F931F93CF93DF938C017B01C0E081
:107DA000D0E0F701EC0FFD1F6491662361F0D8016C
:107DB000ED91FC910190F081E02DC8011995892B7E
:107DC00011F02196EECFCE01DF91CF911F910F914F
:107DD000FF90EF9008956115710579F0FB01019016
:107DE0000020E9F73197AF01461B570BDC01ED91FD
:107DF000FC910280F381E02D199480E090E00895D9
:107E00004F925F926F927F92EF92FF920F931F9328
:107E1000CF93DF93CDB7DEB7A1970FB6F894DEBF4F
:107E20000FBECDBF7C01FA01CB0119A2223008F4AC
:107E30002AE08E010F5D1F4F422E512C612C712CB8
:107E4000BF01A30192010E9427B2F901CA010150AA
:107E500011096A3014F4605D01C0695CD8016C934B
:107E6000232B242B252B61F7B801C701B4DFA19682
:107E70000FB6F894DEBF0FBECDBFDF91CF911F913B
:107E80000F91FF90EF907F906F905F904F900895CB
:107E90004F925F926F927F928F929F92AF92BF921A
:107EA000CF92DF92EF92FF92CF93DF93EC016A01C2
:107EB0007B01B22E9A01AB01C701B6010E94AEADA3
:107EC000882319F060EA75E027C026013701E8949D
:107ED00077F82FEF3FEF4FE75FE7C301B2010E9452
:107EE000AEAD81110DC02FEF3FEF4FE75FE7C3014C
:107EF000B2010E94B2B018161CF464EA75E00CC01E
:107F00002FEF3FEF4FE75FE4C701B6010E94AAAD34
:107F1000181694F468EA75E0CE01DF91CF91FF90D6
:107F2000EF90DF90CF90BF90AF909F908F907F9019
:107F30006F905F904F904FCF2FEF3FEF4FE75FEC89
:107F4000C701B6010E94B2B087FDE4CF20E030E067
:107F5000A901C701B6010E94B2B087FF09C06DE256
:107F6000CE010EDF4C01F7FAF094F7F8F09402C05E
:107F7000812C912CA12C60E070E080E09FE3AB1499
:107F800041F020E030E040E251E40E9411ADA394C2
:107F9000F6CF9B01AC01C701B6010E94ADAC2B012D
:107FA0003C010E947EAD6B017C010E94B6B09B013A
:107FB000AC01C301B2010E94ACAC2B013C012AE030
:107FC000B701A601CE011CDF7C01E80CF91CBB2027
:107FD00029F06EE2CE01D4DEE80EF91EDB2CDD20A6
:107FE00021F120E030E040E251E4C301B2010E94FF
:107FF00017B12B013C010E947EAD4B01A12CB12C8D
:108000002AE0B501A401CE01FBDEE80EF91EC50190
:10801000B4010E94B6B09B01AC01C301B2010E9441
:10802000ACAC2B013C01DA94DACFC701DF91CF91E0
:10803000FF90EF90DF90CF90BF90AF909F908F9088
:108040007F906F905F904F9008956CEA75E0C3CE7B
:108050000F931F93CF93DF93EC01BDDE8C01CE0114
:10806000F4DF800F911FDF91CF911F910F91089541
:108070000F931F93CF93DF93EC0189DE8C01CE0128
:10808000E4DF800F911FDF91CF911F910F91089531
:108090001F920F920FB60F9211240BB60F922F93CF
:1080A0003F934F935F936F937F938F939F93AF9380
:1080B000BF93EF93FF938CEB96E017DCFF91EF916A
:1080C000BF91AF919F918F917F916F915F914F91F0
:1080D0003F912F910F900BBE0F900FBE0F901F90EE
:1080E00018951F920F920FB60F9211240BB60F9294
:1080F0002F933F934F935F936F937F938F939F93B0
:10810000AF93BF93EF93FF938CEB96E083DBFF91EC
:10811000EF91BF91AF919F918F917F916F915F91FF
:108120004F913F912F910F900BBE0F900FBE0F906C
:108130001F9018951F920F920FB60F9211240BB635
:108140000F922F933F934F935F936F937F938F93F0
:108150009F93AF93BF93EF93FF9389E597E0C5DBC0
:10816000FF91EF91BF91AF919F918F917F916F910F
:108170005F914F913F912F910F900BBE0F900FBECB
:108180000F901F9018951F920F920FB60F92112407
:108190000BB60F922F933F934F935F936F937F9301
:1081A0008F939F93AF93BF93EF93FF9389E597E0EE
:1081B00031DBFF91EF91BF91AF919F918F917F91B3
:1081C0006F915F914F913F912F910F900BBE0F9048
:1081D0000FBE0F901F9018951F920F920FB60F921F
:1081E00011240BB60F922F933F934F935F936F938E
:1081F0007F938F939F93AF93BF93EF93FF9386EFFC
:1082000097E073DBFF91EF91BF91AF919F918F91B9
:108210007F916F915F914F913F912F910F900BBE86
:108220000F900FBE0F901F9018951F920F920FB6D0
:108230000F9211240BB60F922F933F934F935F939E
:108240006F937F938F939F93AF93BF93EF93FF931E
:1082500086EF97E0DFDAFF91EF91BF91AF919F91A9
:108260008F917F916F915F914F913F912F910F90DF
:108270000BBE0F900FBE0F901F9018951F920F927C
:108280000FB60F9211240BB60F922F933F934F937B
:108290005F936F937F938F939F93AF93BF93EF936E
:1082A000FF9383E998E021DBFF91EF91BF91AF91BC
:1082B0009F918F917F916F915F914F913F912F91FE
:1082C0000F900BBE0F900FBE0F901F9018951F922E
:1082D0000F920FB60F9211240BB60F922F933F936C
:1082E0004F935F936F937F938F939F93AF93BF93BE
:1082F000EF93FF9383E998E08DDAFF91EF91BF91BF
:10830000AF919F918F917F916F915F914F913F912D
:108310002F910F900BBE0F900FBE0F901F901895CE
:10832000CF93DF93EC01E881F9810284F385E02D9E
:108330001995EA89FB8980818F7E8083EA89FB8990
:108340008081877F8083EA89FB8980818F77808322
:10835000EA89FB8980818F7D80838A8D898FDF9177
:10836000CF910895CF92DF92EF92FF921F93CF9318
:10837000DF93EC016A017B01122FE889F98982E021
:1083800080834115514E61057105B1F060E079E0DF
:108390008DE390E0A70196010E9427B2DA01C9019E
:1083A0000197A109B109B695A79597958795AC0155
:1083B000411580E15807A8F0E889F989108260E842
:1083C00074E88EE190E0A70196010E9427B2BA01FD
:1083D000A901415051096109710976956795579531
:1083E0004795EC85FD855083EE85FF854083188E8B
:1083F000EC89FD891083EA89FB8980818061808313
:10840000EA89FB89808188608083EA89FB89808191
:1084100080688083EA89FB8980818F7D8083DF91FA
:10842000CF911F91FF90EF90DF90CF900895CF9361
:10843000DF93282F30E0F901E058F04F8491F901E3
:10844000E65CF04FD491F901EC50F14FC491CC238C
:1084500089F08111FBDAEC2FF0E0EE0FFF1FE652FE
:10846000F14FA591B491EC91ED2381E090E021F4DE
:1084700080E002C080E090E0DF91CF9108951F93EB
:10848000CF93DF93282F30E0F901E058F04F84912B
:10849000F901E65CF04FD491F901EC50F14FC49131
:1084A000CC23C1F0162F8111D1DAEC2FF0E0EE0FC2
:1084B000FF1FE054F14FA591B4918FB7F8941111BB
:1084C00005C09C91ED2FE095E92302C0EC91ED2BC6
:1084D000EC938FBFDF91CF911F910895CF93DF93DE
:1084E00090E0FC01E65CF04F2491FC01EC50F14F70
:1084F0008491882361F190E0880F991FFC01EA556F
:10850000F14FC591D491FC01E054F14FA591B49184
:10851000611109C09FB7F8948881209582238883D0
:10852000EC912E230BC0623061F49FB7F894388130
:10853000822F809583238883EC912E2B2C939FBFD1
:1085400006C08FB7F894E8812E2B28838FBFDF9168
:10855000CF9108951F93CF93DF93182FEB0161E024
:10856000BDDF209711F460E004C0CF3FD10531F4A6
:1085700061E0812FDF91CF911F9181CFE12FF0E05A
:10858000E058F04FE4914E2F50E0FA013197E2317C
:10859000F10508F09DC08827EC5BFE4F8F4F0C94CF
:1085A00098AC84B5806884BDC7BD97C084B580622F
:1085B00084BDC8BD92C08091800080688093800097
:1085C000D0938900C093880088C080918000806229
:1085D00080938000D0938B00C0938A007EC08091EE
:1085E0008000886080938000D0938D00C0938C00C1
:1085F00074C08091B00080688093B000C093B300D5
:108600006CC08091B00080628093B000C093B400D1
:1086100064C080919000806880939000D09399000E
:10862000C09398005AC0809190008062809390001F
:10863000D0939B00C0939A0050C0809190008860B6
:1086400080939000D0939D00C0939C0046C0809181
:10865000A00080688093A0008091A0008F7B809311
:10866000A000D093A900C093A80037C08091A000BB
:1086700080628093A000D093AB00C093AA002DC06D
:108680008091A00088608093A000D093AD00C0933B
:10869000AC0023C080912001806880932001D0939A
:1086A0002901C093280119C0809120018062809324
:1086B0002001D0932B01C0932A010FC0809120018B
:1086C000886080932001D0932D01C0932C0105C0B8
:1086D000C038D1050CF04CCF46CFDF91CF911F9120
:1086E0000895863308F0865390917B00282F2870D8
:1086F000977F922B90937B008770806480937C009F
:1087000080917A00806480937A0080917A0086FD5F
:10871000FCCF809178002091790090E0922B089511
:108720003FB7F8948091180D9091190DA0911A0DF2
:10873000B0911B0D26B5A89B05C02F3F19F00196DF
:10874000A11DB11D3FBFBA2FA92F982F8827820FD7
:10875000911DA11DB11DBC01CD0142E0660F771F27
:10876000881F991F4A95D1F708958F929F92AF92D3
:10877000BF92CF92DF92EF92FF926B017C01D0DF2C
:108780004B015C01C114D104E104F104E9F0C8DF3C
:10879000DC01CB0188199909AA09BB09883E9340DD
:1087A000A105B10578F321E0C21AD108E108F1086A
:1087B00088EE880E83E0981EA11CB11CC114D10460
:1087C000E104F10421F7DECFFF90EF90DF90CF902E
:1087D000BF90AF909F908F9008952FB7F8946091BD
:1087E000140D7091150D8091160D9091170D2FBFDE
:1087F0000895CF93C0910E026C2F89E340DE81E093
:10880000C8276C2F8AE33BDEC0930E02CF910895F8
:10881000CF93DF93C0910D026C2F89E330DED1E05E
:10882000DC276D2F8AE32BDE6C2F85E328DE6D2F8E
:1088300085E025DE6D2F84E022DE6C2F87E01FDED1
:10884000CC2311F0729801C0729A90910D0281E0D0
:10885000892780930D02DF91CF910895CF93C09126
:10886000290D6C2F70E088E075DE89E18093280D7A
:1088700090910C02992311F0CD5F01C0C350C093B9
:10888000290D8091290D873970F0992321F08FEF00
:108890008093290D08C08D3D30F086E98093290D25
:1088A00088E78093280D8091290D8F3F19F410924D
:1088B0000C0205C08A3118F481E080930C024091CB
:1088C000280D50E060E070E02EE234E487EB9AE09F
:1088D0000E946C3A90937C1280937B12CF91089502
:1088E000CF92DF92EF92FF92CF93DF93EC019C0146
:1088F000AFEFB0E00E9449B2CC24CA9423E0D22E5C
:10890000E12CF12CA70196010E94FBB1B90188E08E
:1089100021DE9E01A4E6B0E00E9449B2A7019601C3
:108920000E94FBB180912510821320932510DF91C6
:10893000CF91FF90EF90DF90CF900895CF93DF938A
:10894000C0917B12D0917C12BE0187EB9AE00E940D
:10895000053A882329F0BE0187EB9AE00E941D3A70
:1089600060E088E08CDD80915F068823C9F080910B
:108970007D12882319F06CE671E10DC080917A12A6
:10898000882319F063E571E106C080917B0D8111A8
:1089900007C064E471E180915D0690915E0668DB3A
:1089A00010927D1210927A12DF91CF91089561E0BA
:1089B00088E065DD80915F06882359F080917D1203
:1089C000811107C066E371E180915D0690915E06BA
:1089D0004FCB089580917D1281110FC0AFDF81E0F0
:1089E00080937D1280915F06882339F065E871E1FC
:1089F00080915D0690915E063BDB8091270D882378
:108A000021F060E088E03BDD01C0D1DF9091270DCF
:108A100081E089278093270D882329F04091211038
:108A20005091221004C0409123105091241060E016
:108A300070E02AEE34E487EB9AE00E946C3A90935F
:108A40007C1280937B120895CF938091250D811124
:108A50000EC081E08093250D80915F06882339F058
:108A600064E071E180915D0690915E0601DBC0914A
:108A7000240D6C2F85E003DD40912A1050E060E06A
:108A800070E024E235E487EB9AE00E946C3A909320
:108A9000230D8093220D81E06C2F68276093240DB5
:108AA000CF9108958091070180FF10C060E08EE3B0
:108AB000E6DC1092F60580915F06882339F06BE7BB
:108AC00070E180915D0690915E06D2CA0895809112
:108AD000070180FF11C061E08EE3D1DC81E080936B
:108AE000F60580915F06882339F065E670E1809194
:108AF0005D0690915E06BCCA08958091070181FFD2
:108B000010C060E08FE3BBDC1092EF0580915F0640
:108B1000882339F06EE470E180915D0690915E06E5
:108B2000A7CA08958091070181FF11C061E08FE31A
:108B3000A6DC81E08093EF0580915F06882339F001
:108B400068E370E180915D0690915E0691CA089598
:108B50008091BC05882321F080E090E00C94927C09
:108B600080E090E00C94A57CCF93DF93C0912A0D18
:108B7000D0912B0DBE0187EB9AE00E94053A882325
:108B800069F0BE0187EB9AE00E941D3A10922B0D0E
:108B900010922A0DDF91CF910C94B35ADF91CF91AF
:108BA000089560912A0D70912B0D87EB9AE00E9439
:108BB000053A811128C060E089E361DC60E08AE366
:108BC0005EDC60E085E35BDC60E085E058DC60E073
:108BD00084E055DC60E087E052DC729880912710D9
:108BE000882319F028E034E402C029EF33E442E39B
:108BF00050E060E070E087EB9AE00E94863A909344
:108C00002B0D80932A0D089560E08AE338CC61E053
:108C10008AE335CC0F931F93CF93DF938C01C1E090
:108C2000D0E00C171D078CF0F2DF64E670E080E006
:108C300090E09BDDE9DFC017D1072CF46AE570E016
:108C400080E090E092DD2196ECCFDF91CF911F91F3
:108C50000F91089583E090E0DDCF82E090E0DACFDD
:108C600081E090E0D7CF60E089E309CC61E089E35F
:108C700006CC0F931F93CF93DF938C01C1E0D0E01C
:108C80000C171D078CF0F2DF64E670E080E090E0E6
:108C90006CDDE9DFC017D1072CF46AE570E080E0F5
:108CA00090E063DD2196ECCFDF91CF911F910F9182
:108CB000089583E090E0DDCF82E090E0DACF81E0BC
:108CC00090E0D7CF1092260D80914B06811103C002
:108CD00060E084E0D4DB80915F06882339F063E2B2
:108CE00071E180915D0690915E06C2C9089581E0B0
:108CF0008093260D80914B06811105C060911D0D5A
:108D000070E084E027DC80915F06882339F061E120
:108D100071E180915D0690915E06AAC90895109256
:108D20004B068091260D811103C060E084E0A7CB43
:108D300060911D0D70E084E00DCCCF93DF9360E077
:108D400085E09DDBC091220DD091230DBE0187EB04
:108D50009AE00E94053A882329F0BE0187EB9AE049
:108D60000E941D3A80915F06882371F02091250DA5
:108D700080915D0690915E06222319F068EF70E104
:108D800002C06CEE70E174D91092250DDF91CF9185
:108D9000089561E085E073DB80915F06882339F0F8
:108DA00061EE70E180915D0690915E0661C9089563
:108DB00060E085E364DB8091590690915A06DC01FE
:108DC000ED91FC9104A8F5A9E02D199580915F061D
:108DD000882339F065ED70E180915D0690915E0623
:108DE00047C9089561E085E34ADB80915906909177
:108DF0005A06DC01ED91FC9104A8F5A9E02D199526
:108E000080915F06882339F06AEC70E180915D06FD
:108E100090915E062DC908958F929F92AF92BF9256
:108E2000CF92DF92EF92FF9285E45BDCBC01990F59
:108E3000880B990B0E94B8B020E030E040E85AE37C
:108E40000E9417B120E030E040EA50E40E9417B1E0
:108E50006B017C0180910B02882351F0C0921E0DA2
:108E6000D0921F0DE092200DF092210D10920B0276
:108E700026E636E646E65FE360911E0D70911F0D13
:108E80008091200D9091210D0E9417B14B015C0142
:108E900020ED3CEC4CEC5DE3C701B6010E9417B13C
:108EA0009B01AC01C501B4010E94ADAC60931E0DE5
:108EB00070931F0D8093200D9093210D2DE33CE2C4
:108EC00048E450E40E9417B12AE939E949E95EE330
:108ED0000E94ADACFF90EF90DF90CF90BF90AF902D
:108EE0009F908F900895CF93DF938091070180FD2D
:108EF00028C0C091F305D091F4058091F80588232E
:108F000069F08EE3EEDB813092402CF01092F40594
:108F10001092F30509C081E090E002C08EE3E1DB2E
:108F20009093F4058093F3058091F3059091F405F7
:108F30008C179D0719F41092F50503C081E080930A
:108F4000F505DF91CF910895CF93DF9380910701CD
:108F500081FD28C0C091EC05D091ED058091F1050F
:108F6000882369F08FE3BDDB813092402CF01092B2
:108F7000ED051092EC0509C081E090E002C08FE39E
:108F8000B0DB9093ED058093EC058091EC0590911A
:108F9000ED058C179D0719F41092EE0503C081E0D2
:108FA0008093EE05DF91CF91089590915F0688231D
:108FB000D1F08091BB068823B1F081E08093CE0F81
:108FC00080931C0D992301F167E070E180915D06AB
:108FD00090915E060E94C73E0E94C88A80915D06FD
:108FE00090915E0632C81092CE0F992339F06FE14E
:108FF00070E180915D0690915E063AD88091CC0F29
:10900000811102C010921C0D089590915F06882373
:10901000F9F08091BB068823D9F08091820F8D30C2
:10902000B9F481E08093CC0F80931C0D992309F152
:1090300066EC7FE080915D0690915E060E94C73EDF
:109040000E94F68A80915D0690915E060C94254000
:109050001092CC0F992339F066EE7FE080915D0687
:1090600090915E0605D88091CE0F811102C01092BA
:109070001C0D08958091BC0F833041F12CF4813098
:10908000A9F0823099F02DC086305CF580914E06B3
:1090900090914F06DC01ED91FC910480F581E02D6B
:1090A000199580914C0690914D0614C080915206FE
:1090B00090915306DC01ED91FC910480F581E02D47
:1090C0001995809150069091510604C080914E06EA
:1090D00090914F06DC01ED91FC910480F581E02D2B
:1090E00019958091590690915A06DC01ED91FC91F9
:1090F000E05CFF4F0190F081E02D199580915906B9
:1091000090915A06DC01ED91FC910284F385E02DEB
:1091100060E070E01994AEDF8091590690915A0694
:10912000DC01ED91FC910084F185E02D1995809191
:10913000590690915A06DC01ED91FC910480F5816D
:10914000E02D19950E94D3750E94D8898091BD05A4
:1091500081110E94037E80915B0690915C06DC0188
:10916000ED91FC910480F581E02D199580915706D1
:1091700090915806DC01ED91FC910480F581E02D81
:10918000199580919D0F882359F08091E605909163
:10919000E705DC01ED91FC910480F581E02D199447
:1091A000089580910A02882351F036DE20E030E0F5
:1091B00040E050E40E94B2B087FF39C008952CDE31
:1091C00020E030E04AE754E40E9417B10E947EADEF
:1091D00020911A1030911B1040916206621773079C
:1091E00010F4442351F1442309F445C015DE20E076
:1091F00030E04AE754E40E9417B10E947EAD20910E
:109200001A1030911B1062177307A8F110926206B2
:1092100081E08093610680915F06882361F162E9B5
:1092200070E180915D0690915E060C94384010923A
:109230000A0281E080936106089581E080936206CE
:109240001092610680915F06882391F061EB70E1D6
:1092500080915D0690915E060E94C73E0E94B18A91
:109260006EEA70E180915D0690915E060E94384042
:1092700052DF0C94465B089508950895089508956B
:109280001092860A08950F931F93CF93DF93EC01FA
:109290001F8A1E8A8C01075E1F4F40E060E0C801F4
:1092A0000E94B98240E064E0C8010E94B98295DA68
:1092B0006C8F7D8F8E8F9F8FDF91CF911F910F913C
:1092C00008950F931F93CF93DF93EC0180912C0DA2
:1092D000811112C00A8D1B8D6AEA70E0C8010E94DC
:1092E000BF60D801ED91FC910284F385E02DC801A7
:1092F000199581E080932C0D4AE06EE0CE014996ED
:109300000E94B98221E83FEF3B872A878FE790E0F0
:109310009D878C871F861E86398B288B9B8B8A8B1B
:109320001D8A1C8ADF91CF911F910F9108950F9391
:109330001F93CF93DF93EC011F8A1E8A8C01075E77
:109340001F4F40E060E0C8010E947C8240E064E082
:10935000C8010E947C8241DA6C8F7D8F8E8F9F8F37
:10936000DF91CF911F910F9108950F931F93CF938A
:10937000DF93EC01E8A1F9A180819181A281B38101
:109380008E01075E1F4F81159649A105B10509F4AD
:1093900050C040E056E960E070E089E597E00E9447
:1093A000356364E170E080E090E0DFD9E8A1F9A1E5
:1093B00080819181A281B38181152BE49207A1055F
:1093C000B105E9F068F4803629E09207A105B105FE
:1093D000A1F080389542A105B105C1F442E012C068
:1093E000811521EE9207A105B10559F08115924C26
:1093F000A140B10559F445E005C041E003C043E098
:1094000001C046E06FE0C8010E947C8289E597E0D8
:109410000E94DC3CE8A1F9A1408151816281738105
:1094200089E597E00E94356364E170E080E090E0B8
:109430009CD94AE06EE0C8010E947C8241E067E16D
:10944000C8010E947C824AA168E1C8010E947C8216
:1094500021E83FEF3B872A878FE790E09D878C8745
:109460001F861E86398B288B9B8B8A8B1D8A1C8AB4
:10947000DF91CF911F910F9108950C94C660CF9307
:10948000DF93C8E1DAE081E090E09A83898310926B
:10949000860A46D96C837D838E839F83E49AEC9AF7
:1094A000DF91CF910895EF92FF920F931F93CF9387
:1094B000DF93EC016623E1F0262F653608F024E601
:1094C0000A891B89E888F988D801AE19BF0930E0FC
:1094D0000E94A6AC28EC30E040E050E00E9427B2A9
:1094E000E20EF31EFB86EA86021B130B1D870C8718
:1094F000DF91CF911F910F91FF90EF900895CF933F
:10950000DF93CDB7DEB7A2970FB6F894DEBF0FBEDC
:10951000CDBF80310CF080E12EE532E13A83298322
:1095200026E532E13C832B832EE432E13E832D831A
:1095300026E432E138872F832EE332E13A87298708
:1095400026E332E13C872B872EE232E13E872D87EE
:1095500026E232E1388B2F8728E132E13A8B298BE2
:1095600026E032E13C8B2B8B29EE31E13E8B2D8BBB
:1095700024ED31E1388F2F8B2AEC31E13A8F298F9E
:1095800020EC31E13C8F2B8F23EB31E13E8F2D8F8F
:1095900027EA31E138A32F8F2FE931E13AA329A33C
:1095A000E82FEE0FFF0BEC0FFD1F81819281A29639
:1095B0000FB6F894DEBF0FBECDBFDF91CF910895F7
:1095C0008F929F92AF92BF92CF92DF92EF92FF92D3
:1095D0000F931F93DC0118968D919C9119971E96FD
:1095E000CD90DC901F976817790709F456C05896FC
:1095F000FC9058974C01092E000CAA08BB088B015F
:10960000072E000C220B330B861797073CF4169697
:10961000ED91FC911797FF2039F015C01496ED914C
:10962000FC911597FF2079F00D2C000CEE08FF0837
:10963000A9019801281939094A095B091C966D91FD
:109640007C911D970EC00D2C000CEE08FF08A9019F
:109650009801281939094A095B091A966D917C917C
:109660001B97CB01770FAA0BBB0BBC01CD016C196B
:109670007D098E099F090E9462AC8F01FF0F220BAA
:10968000330BA9019801281939094A095B090E947D
:10969000FBB1C20ED31EE41EF51EC6011F910F9131
:1096A000FF90EF90DF90CF90BF90AF909F908F9002
:1096B0000895CF93DF93EC017F8B6E8B81DF9C014C
:1096C0008A819B8188309105C1F437FF06C061E033
:1096D00021388FEF38074CF001C060E0A901203835
:1096E00031052CF04FE750E002C041E85FEF57FF33
:1096F0001FC05195419551091BC00997E9F4922F5C
:10970000832F2038310514F09FE780E0492F582F30
:1097100041388FEF580714F441E85FEF57FF03C05B
:10972000519541955109632F661F6627661F6C5F2F
:10973000CE0149960E94B98250D86C8F7D8F8E8F52
:109740009F8FDF91CF910895CF93DF93EC017F8BB3
:109750006E8B36DF9C018A819B8188309105C1F434
:1097600037FF06C061E021388FEF38074CF001C0A9
:1097700060E0A901203831052CF04FE750E002C02D
:1097800041E85FEF57FF1FC05195419551091BC03C
:109790000997E9F4922F832F2038310514F09FE7C1
:1097A00080E0492F582F41388FEF580714F441E8D3
:1097B0005FEF57FF03C0519541955109632F661F15
:1097C0006627661F6C5FCE0149960E947C8205D891
:1097D0006C8F7D8F8E8F9F8FDF91CF9108950F9328
:1097E0001F93CF93DF93EC010E94ED430C8D1D8DF1
:1097F0002E8D3F8DDC01CB01801B910BA20BB30B97
:10980000853F9140A105B10540F06E897F89CE0169
:10981000DF91CF911F910F9197CFDF91CF911F9142
:109820000F910895CF93DF93EC0161E089E00E94EE
:109830006E4260E089E00E943F4210929D0988EFED
:1098400094E099838883DF91CF910895CF92DF923E
:10985000EF92FF9280919E09833009F061C0809160
:109860009F098130D1F488EE93E0A0E0B0E08093CE
:10987000300990933109A0933209B093330980E7FE
:1098800097E1A0E0B0E08093340990933509A0936C
:109890003609B093370932E001C030E0E0919F090A
:1098A000F0E0E056F64F2081A0E1A30F48EE53E030
:1098B00060E070E088EBC82E8BE0D82EE12CF12C14
:1098C000832F90E0FC01EE0FFF1FEE0FFF1FE05D06
:1098D000F64F27FF10C0C082D182E282F382880F48
:1098E000991F880F991FFC01EC5CF64F4083518350
:1098F000628373830FC04083518362837383880FB5
:10990000991F880F991FFC01EC5CF64FC082D18231
:10991000E282F3823E5F220F3A13D2CF309399094D
:10992000FF90EF90DF90CF900895CF93DF938091D9
:109930009D09811153C010929B0910929809C1E0B2
:10994000C0939D09D0919C0961E089E00E946E421C
:1099500060E089E00E943F422D2F30E040E050E07F
:1099600060E47FE180E090E00E94FBB1C093B00032
:1099700089E08093B1002093B3008BEA289F212DCA
:10998000112426952093B40080916F008B7F8093E3
:109990006F008091B00080628093B00020918400BD
:1099A00030918500E091980981E08E0F80939809AD
:1099B00084E0E89FF0011124E05DF64F8081918101
:1099C000A281B381820F931F90938B0080938A00B2
:1099D000B29A80916F00846080936F00DF91CF9185
:1099E00008954F925F926F927F928F929F92AF9263
:1099F000BF92CF92DF92EF92FF928AE18093990912
:109A000020939A0988E280939C0981E080939F09C2
:109A10008093A0098EE080939E0980EC92E1A0E003
:109A2000B0E08093300990933109A0933209B0934C
:109A3000330980EB94E0A0E0B0E080933409909388
:109A40003509A0933609B0933709A4E1440F551F97
:109A5000661F771FAA95D1F722E030E0B0EBCB2E3E
:109A6000B4E0DB2EE12CF12C80E6482E89E0582E64
:109A7000612C712C90E4892E9CE9992EA12CB12C9B
:109A8000C901880F991F880F991FFC01E05DF64FEF
:109A900077FF05C0408251826282738204C0C08217
:109AA000D182E282F382C9010196880F991F880F43
:109AB000991FFC01E05DF64F283129F0C082D18268
:109AC000E282F38204C080829182A282B382440F38
:109AD000551F661F771F2E5F3F4F2A31310581F6D4
:109AE000FF90EF90DF90CF90BF90AF909F908F90BE
:109AF0007F906F905F904F9018CF8F929F92AF9210
:109B0000BF92CF92DF92EF92FF9282E18093990908
:109B100086E080939A0996E290939C0991E0909355
:109B20009F099093A00980939E0988ED90E4A0E09E
:109B3000B0E08093300990933109A0933209B0933B
:109B400033098CE19CE0A0E0B0E08093340990936D
:109B50003509A0933609B0933709742F6627552726
:109B6000442722E030E0ACE1CA2EACE0DA2EE12C52
:109B7000F12CB8E38B2EB8E19B2EA12CB12CC9019E
:109B8000880F991F880F991FFC01E05DF64F77FF42
:109B900005C080829182A282B38204C0C082D18239
:109BA000E282F382F901EE0FFF1FEE0FFF1FEC5C64
:109BB000F64FC082D182E282F382440F551F661FA6
:109BC000771F2E5F3F4F22313105C9F68CE199E8AE
:109BD000A0E0B0E08093740990937509A093760992
:109BE000B0937709FF90EF90DF90CF90BF90AF9048
:109BF0009F908F909ACE1F920F920FB60F921124C2
:109C00000BB60F922F933F934F935F936F937F9376
:109C10008F939F93AF93BF93EF93FF939091980986
:109C200080919909981316C01092980980919F0904
:109C30008F5F80939F0990919F098091A009891758
:109C400040F481E080939F0980919B098F5F80930E
:109C50009B09FCDD90919B0980919A0998130DC096
:109C60008091B0008F7D8093B00080916F008B7FDA
:109C700080936F0010929D0927C08091B00085FFEE
:109C800004C08091B0008F7D03C08091B0008062DD
:109C90008093B0002091840030918500E091980974
:109CA00081E08E0F8093980984E0E89FF0011124F1
:109CB000E05DF64F80819181A281B381820F931F75
:109CC00090938B0080938A00FF91EF91BF91AF91A9
:109CD0009F918F917F916F915F914F913F912F91C4
:109CE0000F900BBE0F900FBE0F901F9018951F92F4
:109CF0000F920FB60F9211240BB60F921F932F9352
:109D00003F934F935F936F937F938F939F93AF9303
:109D1000BF93EF93FF93CF93DF9300D01F92CDB704
:109D2000DEB78091180A0E94174211E0892B09F0D2
:109D300010E00E94904369837A838B839C8389819E
:109D40009A81AB81BC8140911C0A50911D0A60919F
:109D50001E0A70911F0A841B950BA60BB70B20914E
:109D6000190A30911A0A2430310509F44CC0253003
:109D7000310521F021303105E9F414C020911B0A8E
:109D8000222339F02091860A20FF02C0289A01C0C0
:109D90002898112379F0813E2EE29207A105B105A2
:109DA00048F02BC0112379F125E030E030931A0AF6
:109DB0002093190A2091190A30911A0A2530310589
:109DC00011F5E091860AF0E0EE0FFF1FE05EF54F1F
:109DD0009183808389819A81AB81BC8180931C0AA5
:109DE00090931D0AA0931E0AB0931F0A8091860AC1
:109DF0008F5F8093860A833330F084E090E0909305
:109E00001A0A8093190A0F900F900F900F90DF910C
:109E1000CF91FF91EF91BF91AF919F918F917F91E2
:109E20006F915F914F913F912F911F910F900BBEBA
:109E30000F900FBE0F901F90189581E08093990AA4
:109E4000089581E080939A0A089581E080939B0AA7
:109E50000895CF938091760DC0910F02811101C1B9
:109E6000C23009F450C0C33009F49DC0C13009F0BC
:109E700028C180919B0A811124C181E090E00E9459
:109E8000B2AD909331128093301262E083E00E9471
:109E90006E421092750D10922A1210922912109291
:109EA0002E1280E090E0FC01EE0FFF1FED59F24F03
:109EB00011821082019688309105A9F71092740DD5
:109EC0001092730D80916A008C6080936A00ED9A05
:109ED0008FB7F89420918400309185003093620D03
:109EE0002093610D8FBF25E23FE44AEF50E060E030
:109EF00070E080912512909126120E946C3A81E0C8
:109F00008093760DDEC080919A0A8111DAC081E0DB
:109F100090E00E94B2AD9093331280933212809100
:109F200004018E7F809304018091050181608093FC
:109F300005018CEB96E090935D1280935C122EE20B
:109F400040EA56E861E070E00E94B241809165000D
:109F50008B7F809365001092350189E080933401F6
:109F60008EE2809332018CEF8093300180E9809300
:109F7000310110925B1210925A12109259121092E3
:109F8000581210925612E6E3F2E18CED95E08193BF
:109F9000919322E1E635F207D1F7C1E0C093571261
:109FA00021E23FE451C08091990A81118AC081E089
:109FB00090E00E94B2AD909335128093341280915C
:109FC00004018E7F8093040180910501816080935C
:109FD00005018CEB96E09093370D8093360D26E0CB
:109FE00040E052EC61E070E00E94B2418091650077
:109FF0008B7F809365001092350180E1809334015E
:10A0000086E0809332018EEF8093300180E9809367
:10A01000310110922C1210922B121092350D1092C9
:10A02000340D10922D12E8E3FDE08CED95E0819364
:10A0300091932DE0E435F207D1F71092330DC1E092
:10A04000C093320D2DE13FE44AEF50E060E070E054
:10A0500080912512909126120E946C3AC093760D41
:10A0600030C0C23069F0C330D1F0C13051F58091B9
:10A070009B0A811126C08091291290912A121DC03D
:10A0800080919A0A81111DC08091321290913312F1
:10A090000E94F68280915A1290915B120EC08091BC
:10A0A000990A81110EC080913412909135120E944C
:10A0B000D78580912B1290912C12029711F4C093A6
:10A0C000A20A80910F028230A1F1833009F454C0BA
:10A0D000813009F074C080919B0A882309F46FC015
:10A0E000ED98E59A1092750D10922F1210922A1287
:10A0F0001092291210922E1280E090E0FC01EE0FD7
:10A10000FF1FED59F24F11821082019688309105A0
:10A11000A9F71092740D1092730D809130129091E6
:10A1200031120E9447AE1092760D10929A0A82E088
:10A1300044C080919A0A882309F441C080915C123E
:10A1400090915D120E949041809131018F778093B0
:10A150003101809131018F7E809331011092300165
:10A1600080913212909133120E9447AE1092760D78
:10A170001092990A83E021C08091990A8823F9F00E
:10A180008091360D9091370D0E9490418091310160
:10A190008F7780933101809131018F7E80933101DF
:10A1A0001092300180913412909135120E9447AE86
:10A1B0001092760D10929B0A81E080930F0280919D
:10A1C000251290912612CF910C948E3AAF92BF92A5
:10A1D000CF92DF92EF92FF920F931F93CF93DF9373
:10A1E0007C016B015A01D0E0C0E08D2F90E0F701B7
:10A1F000A181B2818A159B05D0F4F601E80FF91F01
:10A20000608106E318E721E03327C6270C0F111DF4
:10A21000211D311D2BBFF801C791ED91FC911197C4
:10A220000190F081E02DCD011995DF5FDECFED913A
:10A23000FC9111970190F081E02D6C2FCD01DF9101
:10A24000CF911F910F91FF90EF90DF90CF90BF9033
:10A25000AF901994CF93DF9300D01F921F92CDB788
:10A26000DEB7FE01319625E0DF011D922A95E9F760
:10A2700024E8298325E52C832AE22D836A834B83F6
:10A2800045E050E0BF01A2DF65E070E080E090E0D3
:10A290000E94B54380E00F900F900F900F900F90A9
:10A2A000DF91CF910895EF92FF921F93CF93DF93A9
:10A2B0001F92CDB7DEB77C01162FFC016181728140
:10A2C0000E94767965E070E080E090E00E94B543FE
:10A2D00042E462E4C701BEDF412F60E0C701BADF9C
:10A2E000811163C040E061E0C701B4DF81115DC04E
:10A2F00040E062E0C701AEDF811157C046E062E096
:10A30000C701A8DF811151C040E063E0C701A2DFAF
:10A3100081114BC040E064E0C7019CDF11E0811176
:10A3200010E040E065E0C70195DF811101C01F5FCB
:10A3300040E066E0C7018EDF811101C01F5F40E091
:10A3400067E0C70187DF811101C01F5F40E068E05F
:10A35000C70180DF811101C01F5F40E069E0C701D4
:10A3600079DF811101C01F5F44E06AE0C70172DF3D
:10A37000811101C01F5F44E06AE0C7016BDF8111FA
:10A3800001C01F5F62E370E080E090E00E94B5438F
:10A3900082E8898341E050E0BE016F5F7F4FC701D3
:10A3A00015DF81E0183011F0111180E00F90DF917E
:10A3B000CF911F91FF90EF900895CF93DF9300D03E
:10A3C0001F92CDB7DEB72AEA2983FC0120812A83B8
:10A3D0006B834C8344E050E0BE016F5F7F4FF6DE3D
:10A3E0000F900F900F900F90DF91CF9108953FB78E
:10A3F000F89420E0822F90E0841795079CF4FC01EC
:10A40000EE0FFF1FEB59F24FA081B181880F991F0A
:10A41000FB01E80FF91FCD01969587959183808305
:10A420002F5FE8CF3FBF10922E120895AF92BF92D8
:10A43000CF92DF92EF92FF920F931F93CF93DF9310
:10A44000CDB7DEB7EDB6FEB60E94F3830E94E98376
:10A450000E943F84029709F0BCC10E942A8488238D
:10A4600009F4B1C1A0902712B0902812C090251213
:10A47000D0902612B501C6010E94053A8823F1F05A
:10A48000F601E250FE4F00E010E0819191918A15B3
:10A490009B0571F40E94ED43000F111F000F111F67
:10A4A000F601E00FF11F608371838283938308C0FC
:10A4B0000F5F1F4F0E31110541F702C00E94138537
:10A4C00010929C0ACDB6DEB640919F0A5091A00A28
:10A4D000CA01880F991F2DB73EB7281B390B0FB63D
:10A4E000F8943EBF0FBE2DBF0DB71EB70F5F1F4FB5
:10A4F0008091A20A823061F0833021F1813009F02D
:10A5000070C0B801809130129091311270DF33C069
:10A510003FB7F89420E0822F90E08417950774F4F9
:10A52000880F991FF801E80FF91FDC01AA5CBD4EE6
:10A530008D919C91918380832F5FEDCF3FBF1092CF
:10A54000561219C03FB7F89420E0822F90E084178C
:10A55000950774F4880F991FF801E80FF91FDC01C3
:10A56000A85CB24F8D919C91918380832F5FEDCF3A
:10A570003FBF10922D1220E06AE071E0822F90E040
:10A5800040919F0A5091A00A8417950754F5689F3F
:10A59000F001699FF00D1124E05DFF4EA085B185AB
:10A5A0008C918823E1F0A081B1813C91C801830F97
:10A5B000911D830F911DDC0112978D919C91A281B9
:10A5C000B3814D915C9111970480F581E02D48177E
:10A5D000590711F4108203C070838D939C932F5FF1
:10A5E000CDCF0FB6F894DEBE0FBECDBE80912A113E
:10A5F000882321F089E291E10E945B8480913411EB
:10A60000882321F083E391E10E945B8480913E11D5
:10A61000882321F08DE391E10E945B8480914811B1
:10A62000882321F087E491E10E945B8480919D0A58
:10A63000882309F465C080913E11811105C0809185
:10A640004811882309F450C0809141119091421122
:10A65000E0914511F0914611238134812817390783
:10A6600024F48085811109C00EC0218132818217B6
:10A67000930734F48085811106C088E090E005C01E
:10A6800080E190E002C080E290E020914B11309197
:10A690004C11E0914F11F0915011438154814217B8
:10A6A000530724F42085222349F00AC041815281B6
:10A6B000241735073CF42085222311F0816003C064
:10A6C000846001C0826020912411309125112817E7
:10A6D000390719F41092261107C090932511809321
:10A6E000241181E0809326118091241190912511ED
:10A6F000429709F472C081E080934A11809340111F
:10A70000E0EDF0E181EDC82E80E1D82E24ED30E1BE
:10A7100041E08081882309F44AC065817681DB01AC
:10A7200017968C91882309F442C0D6018C91882316
:10A73000F1F18281938140838A33B7E09B0794F4DF
:10A740008C0101541640093F110570F007531F4F4B
:10A75000093C110558F08F579440893F910540F00E
:10A7600081E007C085E005C084E003C083E001C04C
:10A7700082E0DB0119969C91992379F0813041F0B8
:10A78000823041F0843041F0853039F481E005C0F9
:10A7900085E003C084E001C082E0D9019C91D6012C
:10A7A000981302C01C9203C04C93D9018C93379626
:10A7B000B7E0CB0ED11C295F3F4F51E1E432F507E2
:10A7C00009F0A7CF04C00E94FF830E94138581E097
:10A7D00066C00E94FF8380E062C0C0902711D090C5
:10A7E00028111C141D040CF055C080913F110091DC
:10A7F0002512109126126091790D70917A0D88239F
:10A80000B1F081E080934011C8010E94053A8111A6
:10A8100015C0A601DD0C660B770B25E830E8C801F2
:10A820000E946C3A90937A0D8093790D07C0C8010D
:10A830000E94053A811102C0109240118091491185
:10A8400000912512109126126091770D7091780D6C
:10A850008823D1F081E080934A11C8010E94053A13
:10A8600081114ECF4091271150912811052E000CD7
:10A87000660B770B22E830E8C8010E946C3A90938F
:10A88000780D8093770D3CCFC8010E94053A811165
:10A8900037CF02C01092401110924A1131CF0FB63B
:10A8A000F894FEBE0FBEEDBEDF91CF911F910F91C8
:10A8B000FF90EF90DF90CF90BF90AF9008951F92E0
:10A8C0000F920FB60F9211240BB60F922F933F9356
:10A8D0004F938F939F93EF93FF9380918400909178
:10A8E00085002091610D3091620D821B930B2091A8
:10A8F0008400309185003093620D2093610D803784
:10A9000027E1920770F19093640D8093630D80911D
:10A91000291290912A12029751F49091750D80910D
:10A920002F1298133CC081E080932E123EC080917C
:10A93000291290912A12892B49F481E090E090939A
:10A940002A12809329121092600D2FC08091291233
:10A9500090912A12019761F58091750D8430D8F598
:10A9600027C02091750D283008F047C09C012C5D50
:10A970003540293B3B4068F4E091750DEF5FE09373
:10A98000750DF0E0EE0FFF1FED59F24F91838083BC
:10A9900034C08091291290912A12029771F583E0B8
:10A9A00090E090932A12809329121092750D25C081
:10A9B0008091291290912A120397B9F79091750D01
:10A9C00080912F129813F1CF80912F12843068F369
:10A9D00082E090E0E6CF8091600D8F5F8093600D04
:10A9E000863018F382E090E090932A128093291227
:10A9F0008091750D80932F12D8CFFF91EF919F9189
:10AA00008F914F913F912F910F900BBE0F900FBEE2
:10AA10000F901F9018950F931F938091580D8111DF
:10AA20000DC00E94ED436093540D7093550D8093BB
:10AA3000560D9093570D81E08093580D0E94ED4381
:10AA40000091540D1091550D2091560D3091570DD8
:10AA5000DC01CB01801B910BA20BB30B893E934011
:10AA6000A105B105A8F08AE30E941742892B11F0D5
:10AA700060E001C061E08AE30E943F420E94ED4332
:10AA80006093540D7093550D8093560D9093570D10
:10AA90001F910F9108950F931F930E94ED43009112
:10AAA0002E0D10912F0D2091300D3091310DDC01C4
:10AAB000CB01801B910BA20BB30B85339142A105F7
:10AAC000B10518F081E080932D0D1F910F91A3CF58
:10AAD000FC0180E090E06150710977FD18C0219180
:10AAE000022E000C330B322F22278227932728E0D7
:10AAF000AC01440F551F97FF06C0CA0131E28327FE
:10AB000030E1932701C0CA01215091F7E4CF0895A5
:10AB10002F923F924F925F926F927F928F929F926D
:10AB2000AF92BF92CF92DF92EF92FF920F931F935B
:10AB3000CF93DF9300D0CDB7DEB75C010E948B4886
:10AB40000E9404460E94364680915D0690915E0602
:10AB50000E9425400E94906624E0A216B10409F4E8
:10AB600048C085E0A816B10409F479C0A3E0AA168C
:10AB7000B10409F0B1C08CE190E00E94B2AD9B83BA
:10AB80008A8386E895E0EA81FB8191838083B382A2
:10AB9000A28281E09FEF958384838FEF90E097837B
:10ABA000868311861086108ECF010E94FE818AE76F
:10ABB00095E0AA81BB818D939C93E0913B0EF0912F
:10ABC0003C0ED08C00919511109196111695079519
:10ABD000E0909311F0909411F694E79468E673E195
:10ABE00080915D0690915E060E9438402224239455
:10ABF00090C08CE190E00E94B2AD9B838A8386E88E
:10AC000095E0EA81FB8191838083B382A28281E017
:10AC10009FEF958384838FEF90E0978386831186DF
:10AC20001086108ECF010E94FE818AE795E0AA81EE
:10AC3000BB818D939C93E0915B06F0915C06D08C78
:10AC40000091AA111091AB1116950795E090A811EB
:10AC5000F090A911F694E7946BE973E135C08CE1AB
:10AC600090E00E94B2AD9B838A8386E895E0EA81FA
:10AC7000FB8191838083B382A28281E09FEF9583E1
:10AC800084838FEF90E09783868311861086108EE1
:10AC9000CF010E94FE818AE795E0AA81BB818D9356
:10ACA0009C93E0915706F0915806D08C0091BF110B
:10ACB0001091C01116950795E090BD11F090BE114E
:10ACC000F694E7946BE773E180915D0690915E06E0
:10ACD0000E943840212C1DC06FE473E180915D0615
:10ACE00090915E060F900F900F90DF91CF911F9182
:10ACF0000F91FF90EF90DF90CF90BF90AF909F901B
:10AD00008F907F906F905F904F903F902F900C941A
:10AD100038400E94906662E473E180915D069091F4
:10AD20005E060E94384066E373E180915D06909173
:10AD30005E060E94C73EB80180915D0690915E0656
:10AD40000E94917A6AE273E180915D0690915E06BD
:10AD50000E94C73EB70180915D0690915E060E94F9
:10AD6000917A6EE173E180915D0690915E060E949A
:10AD7000C73E8D2D0E946C6680915D0690915E06A7
:10AD80000E942540AA81BB81ED91FC911197028020
:10AD9000F381E02DCD011995CA2C8A2D0E941A81CC
:10ADA0008D3D9540A8F464E378E08A2D0E941081DF
:10ADB000EA81FB81F78AE68AB70182810E942A81B3
:10ADC0006CED75E08A2D0E941581DD20C1F01AC05E
:10ADD00064E873E08A2D0E941581AA81BB81579691
:10ADE0001C930E935697B80112968C910E942A815B
:10ADF0006CED75E08A2D0E941081DD2019F09924F8
:10AE0000939401C0912C33243394812C21E0298325
:10AE10000DDB80913E11882359F1AA81BB81ED9110
:10AE2000FC91119760914311709144110190F08150
:10AE3000E02DCD0119958C2D0E941A818D3DB5E034
:10AE40009B075CF48438E3E09E0784F08C018D3D21
:10AE5000954074F00CED15E00BC07C0185339840F3
:10AE60003CF064E3E62E68E0F62E02C004E813E04E
:10AE7000298121111FC0809134118823C9F1E091EB
:10AE80003B11F0913C118581968140913711509191
:10AE900038119C0121533109421753074CF1C196D7
:10AEA000841795072CF10E94ED43641575058605FE
:10AEB0009705F0F0809134118823C1F0409137114B
:10AEC00050913811E0913B11F0913C1185819681B0
:10AED0009C01285C3109421753072CF088539F4F7F
:10AEE000841795071CF481E0982605C021E029838A
:10AEF000882009F47CC0992009F445C0DD20F9F0D0
:10AF000064E873E08C2D0E941581222009F458C05A
:10AF10006091970F7091980F41E08C2D0E94CF8027
:10AF20000E94E56CAA81BB8112968C910E941A81C5
:10AF300008171907ACF38C2D0E94A18041C064E36F
:10AF400078E08C2D0E9410812220B1F06091970F43
:10AF50007091980F40E08C2D0E94CF800E94E56C8C
:10AF6000AA81BB8112968C910E941A818E159F0531
:10AF7000ACF38C2D0E94A180EA81FB81F78AE68ADE
:10AF8000B701828110C0DD20B1F064E378E08C2D40
:10AF90000E941081AA81BB815796FC92EE9256972F
:10AFA000B70112968C910E942A816CED75E08C2D70
:10AFB0000E94158112C064E873E08C2D0E941581F7
:10AFC000EA81FB81178B068BB80182810E942A815E
:10AFD0006CED75E08C2D0E9410810E94ED432B01D9
:10AFE0003C01F8EC4F0E511C611C711C198233207E
:10AFF000D9F180912A118823A9F140912D11509106
:10B000002E11E0913111F0913211858196819C01D0
:10B01000285C3109421753072CF088539F4F84173F
:10B02000950704F581E0D82680915D0690915E0633
:10B03000DD2039F06FE073E10E94384082E090E05B
:10B0400006C06DEF72E10E94384081E090E00E94FE
:10B050000A460E94ED43AA81BB815896DC9288245F
:10B06000839403C0812C1EC0812C80912A118823D7
:10B0700009F409C2E0913111F09132118581968174
:10B0800040912D1150912E119C01215331094217ED
:10B0900053070CF4F8C1C1963324339484179507F1
:10B0A0000CF4F1C10E94FD830E94D27987EB9AE0F3
:10B0B0000E948E3A8091A60A882309F4A9CE809135
:10B0C000A80A882309F4A4CE0E94D2790E94ED8BAD
:10B0D0008823D1F3B4E0AB16B10459F0E5E0AE1625
:10B0E000B10409F465C0F3E0AF16B10409F059C129
:10B0F000CBC01093840F0093830FF092860FE092E1
:10B10000850FD092870FB8018CE191E00E943879C9
:10B11000B7018EE191E00E9438796D2D80E291E0D7
:10B120000E94C67AB80184E00E94843BB70184E0A3
:10B130000E94693BE0915B06F0915C06D08E8091A5
:10B14000820F8D3029F4E0917C0DF0917D0DD08E31
:10B150006CED75E084E00E942A8166E970E080E091
:10B1600090E00E94B5438091820F8D30E1F484E03D
:10B170000E941A81A0915B06B0915C06ED91FC9152
:10B1800011970190F081E02D8D3D95401CF06FEFFF
:10B190007FEF02C061E070E0CD01199580915B0600
:10B1A00090915C065BC080915B0690915C0664C0E8
:10B1B00010938B0F00938A0FF0928D0FE0928C0FFB
:10B1C000D0928E0FB80183E291E00E943879B701E6
:10B1D00085E291E00E9438796D2D87E291E00E942E
:10B1E000C67AB80185E00E94843BB70185E00E94E1
:10B1F000693BE0915706F0915806D08E6CED75E0F2
:10B2000085E00E942A8166E970E080E090E00E947B
:10B21000B5438091810F8D3059F585E00E941A81E8
:10B22000A0915706B09158068D3D95404CF0ED9198
:10B23000FC9111970190F081E02D6FEF7FEF08C036
:10B24000ED91FC9111970190F081E02D61E070E0AB
:10B25000CD0119958091570690915806DC01ED912A
:10B26000FC910190F081E02D60E070E0199599C0AB
:10B270008091570690915806DC01ED91FC91048075
:10B28000F581E02D19958DC010939A0F0093990FB9
:10B29000F0929C0FE0929B0FD092930FB80182E343
:10B2A00091E00E943879B70184E391E00E943879F7
:10B2B0006D2D8CE291E00E94C67AB80183E00E9475
:10B2C000843BB70183E00E94693B8091930FE0913A
:10B2D0003B0EF0913C0E808F8091930F0E9403797A
:10B2E00083E00E941A812091930F222369F1B9E033
:10B2F000BC1538F02091951130919611369527950F
:10B3000002C02EEE32E08217930709F44AC0609122
:10B31000970F7091980F41E083E00E94CF800E94C8
:10B32000E56CEA81FB8182810E941A810817190766
:10B33000B4F383E00E94A180AA81BB8157961C933D
:10B340000E935697B80129C029E02C1508F49DC02A
:10B350002091931130919411369527958217930778
:10B3600001F16091970F7091980F40E083E00E9487
:10B37000CF800E94E56CEA81FB8182810E941A8164
:10B380008E159F05B4F383E00E94A180AA81BB8142
:10B390005796FC92EE925697B70112968C910E94A6
:10B3A0002A8180915D0690915E060E9425400E9450
:10B3B0009066B4E0AB16B10459F0E5E0AE16B10406
:10B3C00051F0F3E0AF16B10471F463EB72E105C024
:10B3D00063EE72E102C06AEC72E180915D069091C9
:10B3E0005E060E9438400E94906668EA72E1809191
:10B3F0005D0690915E060E9438406CE972E1809192
:10B400005D0690915E060E94C73EB80180915D0680
:10B4100090915E060E94917A60E972E180915D06EA
:10B4200090915E060E94C73EB70180915D069091A3
:10B430005E060E94917A64E872E180915D069091C7
:10B440005E060E94C73E8D2D0E946C6680915D064F
:10B4500090915E060E9425400F900F900F90DF9113
:10B46000CF911F910F91FF90EF90DF90CF90BF9001
:10B47000AF909F908F907F906F905F904F903F9094
:10B480002F900C943346312C0DCE2AEC38E066CF49
:10B49000CF93DF93CDB7DEB728970FB6F894DEBF12
:10B4A0000FBECDBF80917B0D8823E1F110927B0D03
:10B4B0000E94B44581E08093030280916006882356
:10B4C00089F165E772E180915D0690915E060E94C8
:10B4D000C73EE091A20AE4300CF0E0E08AE095E09B
:10B4E0009A83898386E095E09C838B8381E095E055
:10B4F0009E838D838CEF94E098878F83EE0FFF0BF4
:10B50000EC0FFD1F6181728180915D0690915E0656
:10B5100028960FB6F894DEBF0FBECDBFDF91CF9156
:10B520000C94384028960FB6F894DEBF0FBECDBFFE
:10B53000DF91CF91089580917B0D811113C00E94FE
:10B540008B4881E080937B0D0E94D14580915F06FE
:10B55000882341F066E672E180915D0690915E0677
:10B560000C943840089560E089E30E943F4260E017
:10B570008AE30E943F4260E085E30E943F4260E030
:10B5800085E00E943F4260E084E00E943F4260E02C
:10B5900087E00E943F4272980895CF93DF93809195
:10B5A000840D81110DC01092830D1092820D81E0E7
:10B5B00090E09093810D8093800D8093840D36C030
:10B5C0008091820D9091830D863191057CF18F38A9
:10B5D000910534F48091800D9091810D019609C000
:10B5E0008D3521E0920754F48091800D9091810D6A
:10B5F00002969093810D8093800D18C0863222E0D0
:10B60000920734F48091800D9091810D0496F1CFD2
:10B61000883E93403CF48091800D9091810D8A5B2F
:10B620009F4FE7CF1092810D1092800D0E94084429
:10B63000C091820DD091830DC93E83E0D80754F0AC
:10B640001092840D90DF26E43BE548EE53E060E085
:10B6500070E007C02DEC3AE5AE010D2E000C660B34
:10B66000770B87EB9AE00E946C3A90937F0D809362
:10B670007E0D8091800D9091810D8C0F9D1F909378
:10B68000830D8093820DDF91CF910895CF93DF9347
:10B6900080916206882319F0DF91CF917ECFC0910F
:10B6A0007E0DD0917F0DBE0187EB9AE00E94053A96
:10B6B000882329F0BE0187EB9AE00E941D3ADF91B2
:10B6C000CF9151CF08950895FC01828193818830F4
:10B6D000910529F410922B0110922A0108950997DF
:10B6E00021F410922901109228010895FC01178A73
:10B6F000168A6CED75E082810C942A81CF93DF93DA
:10B70000EC011F8A1E8A8A810E94A1808B8D88236A
:10B7100031F08A810E941A819A8F898F1B8EDF9166
:10B72000CF910895DF92EF92FF920F931F93CF93E3
:10B73000DF93EC018A81893010F40E948880DD8CCF
:10B740006B8D7C8D098D1A8DEA80FB8089E08E15CA
:10B7500008F466C00F30110538F001369DE6190770
:10B7600028F000E61DE602C00FE010E06F30710522
:10B7700038F061368DE6780728F060E67DE602C095
:10B780006FE070E080E090E00E94B6B020E030E032
:10B790004AE754E40E9411AD20E030E04CE852E466
:10B7A0000E9417B19B01AC0160E070E08AEF94E465
:10B7B0000E9411AD0E9479ADFF2425E12E9DF0017C
:10B7C0002F9DF00D1124EF5AFE4EDD2071F02381E4
:10B7D0003481AB0177FF04C044275527461B570B24
:10B7E00088279927841B950B0AC025813681AB01D8
:10B7F00077FF04C044275527461B570BCA014FB794
:10B80000F89455E15E9DF0015F9DF00D1124EF5A13
:10B81000FE4E108B0787328B218B948B838B4FBF0F
:10B820009D8D6B8D7C8D8A819923F9F08A3058F437
:10B8300095E1899FF0011124EF5AFE4E0581168192
:10B840001695079502C00EEE12E041E00E94CF80EF
:10B8500061E070E080E090E00E94B5438A810E9440
:10B860001A8108171907A0F31EC08A3058F495E111
:10B87000899FF0011124EF5AFE4E03811481169521
:10B88000079502C00AEC18E040E00E94CF8061E01A
:10B8900070E080E090E00E94B5438A810E941A81A6
:10B8A00080179107A0F38A810E94A180B8018A8144
:10B8B000DF91CF911F910F91FF90EF90DF900C944B
:10B8C0002A81CF93DF93EC018A81893010F40E94A2
:10B8D000888048EE53E05B874A8720ED37E03D875C
:10B8E0002C878CED95E09F878E87598B488B3B8BFF
:10B8F0002A8B9D8B8C8BDF91CF910895CF93DF9313
:10B90000EC017F8B6E8B888599856817790769F4C0
:10B910008A810E94A1808B8D882329F18A810E94CF
:10B920001A819A8F898F1B8E1EC0CE010E94E04A19
:10B93000EA81EA30B0F49C01C39714F022E330E0CE
:10B940002E3C8FEF380714F42EEC3FEF8FB7F894AE
:10B9500095E1E99FF0011124EF5AFE4E31872087CF
:10B960008FBF81E08B8FDF91CF910895CF93DF93CD
:10B97000EC018BA19CA1892B11F01CA21BA29B01A5
:10B9800077FF03C0319521953109B901CE010E949D
:10B99000E04A90932D0180932C019F8B8E8B0E9407
:10B9A000ED436F8F78A389A39AA3DF91CF91089578
:10B9B0000F931F93CF93DF938C01FC01778B668BE2
:10B9C0000E94E04AEC01F801828193818830910560
:10B9D000D1F4D7FF06C060E08AE00E943F4261E0F8
:10B9E00005C061E08AE00E943F4260E086E00E947C
:10B9F0003F42D7FF03C0D195C195D109D0932B0108
:10BA0000C0932A011BC00997C9F4D7FF06C060E0A4
:10BA10008DE00E943F4261E005C061E08DE00E9440
:10BA20003F4260E08BE00E943F42D7FF03C0D195C8
:10BA3000C195D109D0932901C0932801DF91CF91FD
:10BA40001F910F910895CF93DF93EC018A81893084
:10BA500010F40E9488802EEC3FEF3B872A8782E318
:10BA600090E09D878C871F861E86398B288B9B8B49
:10BA70008A8B1D8A1C8A6EEE72E08A810E94158173
:10BA80006AEC78E08A810E9410818CED95E09A8FB3
:10BA9000898F1B8EDF91CF910895CF93DF93EC01B7
:10BAA0008BA19CA1892B11F01CA21BA2CE01CFD58A
:10BAB00010922D0110922C011F8A1E8A0E94ED43C4
:10BAC0006F8F78A389A39AA3DF91CF9108950F93E5
:10BAD0001F93CF93DF93FC0123A134A1232B91F17A
:10BAE000EC010E94ED430F8D18A129A13AA1DC01C0
:10BAF000CB01801B910BA20BB30B4097A105B105A5
:10BB000008F18BA19CA10197E9F46E897F896150AE
:10BB100071097F8B6E8BCE01161617062CF0DF9104
:10BB2000CF911F910F91B9CF0E94E04A90932D01C0
:10BB300080932C019F8B8E8B0E94ED436F8F78A397
:10BB400089A39AA3DF91CF911F910F910895CF936D
:10BB5000DF93EC018D8D9E8D1B861A869D878C87C9
:10BB60001F861E86198A188A9B8B8A8B1D8A1C8ABF
:10BB700061E08CE20E946E428A819B81089721F4E9
:10BB800010922D0110922C011CA21BA2DF91CF91CB
:10BB90000895CF93DF93EC0121E03FEF3B872A87A5
:10BBA0008FEF90E09D878C871F861E86398B288BB0
:10BBB0009B8B8A8B1D8A1C8A61E08AE00E946E4200
:10BBC00061E086E00E946E4261E08DE20E946E427A
:10BBD00061E08DE00E946E4261E08BE00E946E4267
:10BBE00061E08EE20E946E428A819B8188309105DD
:10BBF00029F410922B0110922A0106C0099721F412
:10BC00001092290110922801DF91CF9108950F938E
:10BC10001F93CF93DF93EC011F8A1E8A8C01075E6E
:10BC20001F4F40E068E0C8010E94DD5140E06CE039
:10BC3000C8010E94DD510E94ED436C8F7D8F8E8F75
:10BC40009F8FDF91CF911F910F910895CF93DF9335
:10BC5000EC017F8B6E8B0E94E04AAC018A819B8154
:10BC60008830910541F4CE01499657FF02C06AE041
:10BC700009C068E00DC00997D1F4CE01499657FF7D
:10BC800006C06EE042382FEF520744F001C06CE06E
:10BC90004F3751052CF04EE750E002C042E85FEF0D
:10BCA00057FF03C05195419551090E94DD510E94F3
:10BCB000ED436C8F7D8F8E8F9F8FDF91CF91089595
:10BCC0000F931F93CF93DF93EC010E94ED430C8DF4
:10BCD0001D8D2E8D3F8DDC01CB01801B910BA20BA6
:10BCE000B30B853F9140A105B10540F06E897F8976
:10BCF000CE01DF91CF911F910F91A8CFDF91CF910E
:10BD00001F910F910895CF93DF93EC018091860DE1
:10BD1000811109C06A8D7B8DCE0149960E9476798A
:10BD200081E08093860D21E83FEF3B872A878FE7EC
:10BD300090E09D878C871F861E86398B288B9B8B76
:10BD40008A8B1D8A1C8ADF91CF9108950F931F93D0
:10BD5000CF93DF93EC010E94ED430C8D1D8D2E8D52
:10BD60003F8DDC01CB01801B910BA20BB30B853FF8
:10BD70009140A105B10548F06E897F89CE01DF9120
:10BD8000CF911F910F910C94594BDF91CF911F913F
:10BD90000F9108956F927F928F929F92AF92BF9270
:10BDA000CF92DF92EF92FF920F931F93CF93DF9387
:10BDB0008091C8129091C912DC01ED91FC91048030
:10BDC000F581E02D1995B12C181619060CF0D5C087
:10BDD000AA24A3948091C8129091C912DC01ED911C
:10BDE000FC910480F581E02D1995892B09F4C5C0DB
:10BDF000C091E00D81E08C0F8093E00D8091C8121E
:10BE00009091C912DC01ED91FC910680F781E02D43
:10BE10001995EC2FF0E0E056F24F80838A30D1F68E
:10BE2000E090E00DF12C1092030D1092020D109293
:10BE3000FE0C1092FF0C1092000D1092010D10924A
:10BE4000FD0C1092FC0C1092FB0C80EAC82E8DE0C9
:10BE5000D82E00E010E0D0E0C0E00E151F050CF079
:10BE60006FC0F60191916F019D3009F466C09C3757
:10BE7000A1F19A3009F055C0CC2359F16C2E712CE8
:10BE8000C30101970E94A28B7093030D6093020D72
:10BE90000E94ED4360932E0D70932F0D8093300D13
:10BEA0009093310D8091850D882309F462C08090B4
:10BEB000020D9090030DB8016619770980EA9DE0A4
:10BEC0000E9468558816990609F453C010929F0D78
:10BED00052C010929F0DD0E030C08C2F90E0FC013A
:10BEE000E854FD4E1082D13099F068F0D230B1F4B0
:10BEF0000E94A28B6093FE0C7093FF0C8093000D48
:10BF00009093010D0BC00E94A28B6093FB0C06C0A6
:10BF10000E94A28B7093FD0C6093FC0CDF5FC0E06D
:10BF20000CC00F3311053CF4EC2FF0E0E854FD4E4B
:10BF30009083CF5F02C010929F0D0F5F1F4F8DCF78
:10BF400080919F0D81110EC08091F80C9091F90C99
:10BF500001969093F90C8093F80C60E087E80E94BA
:10BF6000579002C0BB24B3941092A00D1092E00D24
:10BF700031CFA0929F0DD1E0E0CF8B2DDF91CF91FB
:10BF80001F910F91FF90EF90DF90CF90BF90AF90F7
:10BF90009F908F907F906F900895CF931092FA0C9E
:10BFA0001092F70C1092F90C1092F80C61E089E3F2
:10BFB0000E943F420E940B558091C8129091C91275
:10BFC000DC01ED91FC910480F581E02D1995892B20
:10BFD00061F08091C8129091C912DC01ED91FC9141
:10BFE0000680F781E02D1995E7CF0E94D3908091CC
:10BFF000C8129091C912DC01ED91FC910284F38585
:10C00000E02D199510922D0D0E94ED4360932E0D99
:10C0100070932F0D8093300D9093310DC1E0BADEF7
:10C0200081110E941F2F0E944B550E94FD83809119
:10C03000F80C9091F90C0A9724F480912D0D882327
:10C0400031F060E08AE80E945790C093FA0C80912A
:10C05000FA0C882321F38091F70C882341F049ECF6
:10C0600051E060E070E087E69EE00E94CBB160E0C6
:10C0700089E30E943F4260E08AE3CF910C943F4203
:10C08000EF92FF920F931F93CF93DF9300D000D0D6
:10C09000CDB7DEB76FEA75E0CE0101960E94883E0B
:10C0A0000D811E81F02EEE24E3948091C8129091B0
:10C0B000C912DC01ED91FC910480F581E02D199508
:10C0C000892B21F18091C8129091C912DC01ED9168
:10C0D000FC910680F781E02D19958F3439F4E092B8
:10C0E0009E0D8093930DE092920DDFCF90919E0D67
:10C0F0009923D9F2E091920D91E09E0F9093920DC9
:10C10000F0E0ED56F24F80839F1578F28091920D0A
:10C110008F1510F4F12C21C04BE050E067E87DE072
:10C12000CE0101960E94647CA3E9BDE0EFEAF5E050
:10C13000FF24F3941127CF018F5A95408017910760
:10C1400034F49D9181919817B1F3F12CF4CF1092B2
:10C15000930D10929E0D1092920DCE0101960E94A9
:10C16000583E8F2D26960FB6F894DEBF0FBECDBF7A
:10C17000DF91CF911F910F91FF90EF900895DC0117
:10C18000ED91FC910190F081E02D1994CF93DF9314
:10C19000EC017F8B6E8B0E94E04ABC018A81DF91AB
:10C1A000CF910C942A8108950895089508950895D3
:10C1B000623039F0633041F0613041F440931A0E3F
:10C1C00008954093190E08954093180E0895623013
:10C1D00069F06330A1F06130D1F450931E0E4093AA
:10C1E0001D0E3093200E20931F0E08955093250EA0
:10C1F0004093240E3093270E2093260E08955093DB
:10C200002E0E40932D0E3093300E20932F0E089556
:10C2100008952091320E211102C0FC01628308951D
:10C220002091320E211102C0FC01648308952091F7
:10C23000320E211102C0FC0163830895089580919C
:10C24000320E811102C00C94D43B0895089580E011
:10C250000895089508950895089508950895809182
:10C26000320E811103C08FE090E0E8C608958091FE
:10C27000320E811120C0633091F028F4613049F012
:10C28000623051F00895653081F060F0663081F0E1
:10C29000089589E090E00EC08AE090E00BC08BE04A
:10C2A00090E008C08CE090E005C08DE090E002C016
:10C2B0008EE090E0C3C608952091320E211107C090
:10C2C000FC018481882319F082E090E0B7C60895CC
:10C2D0002091320E211107C0FC018381882319F0BF
:10C2E00081E090E0ABC608958091320E811103C0C9
:10C2F0008BE090E0A3C608958091320E811104C0B6
:10C3000060E080E190E0D8C608958091320E8111FE
:10C3100004C060E08FE090E0CFC608958091320EB7
:10C32000811126C06330A1F028F4613049F06230F9
:10C3300059F008956530A1F078F06630A9F00895BD
:10C3400060E089E090E013C060E08AE090E00FC018
:10C3500060E08BE090E00BC060E08CE090E007C014
:10C3600060E08DE090E003C060E08EE090E0A4C665
:10C3700008958091320E811126C06330A1F028F417
:10C38000613049F0623059F008956530A1F078F0DD
:10C390006630A9F0089561E089E090E013C061E0A3
:10C3A0008AE090E00FC061E08BE090E00BC061E0BC
:10C3B0008CE090E007C061E08DE090E003C061E0B8
:10C3C0008EE090E079C608952091320E211108C0C8
:10C3D000FC018281882321F061E088E090E06CC656
:10C3E00008952091320E211108C0FC018481882318
:10C3F00021F061E082E090E05FC608952091320E66
:10C40000211108C0FC018381882321F061E081E0D3
:10C4100090E052C608958091320E811104C061E00F
:10C4200086E090E049C608958091320E811104C0E3
:10C4300060E08BE090E040C608958091320E81115B
:10C4400004C061E087E090E037C608958091320E25
:10C45000811104C061E085E090E02EC608958091CE
:10C46000320E81112EC060911B0E70911C0E8091B6
:10C470002B0E90912C0E0E941D3A1092210E80914D
:10C48000320E81110CC06091220E7091230E8091AA
:10C490002B0E90912C0E0E941D3A1092280E809126
:10C4A000320E81110CC06091290E70912A0E80917C
:10C4B0002B0E90912C0E0E941D3A1092310E10926C
:10C4C000E50D08958091320E811117C08091E50D20
:10C4D000811113C029EA39E648EB5BE060E070E0C7
:10C4E00080912B0E90912C0E0E946C3A90931C0E12
:10C4F00080931B0E81E08093E50D08958091320EAC
:10C50000882329F06CED75E081E00C949F3B84E07A
:10C5100090E094C58091320E882329F068EE73E094
:10C5200081E00C949F3B60E084E090E0C5C5809181
:10C53000320E81111BC08091080D8823B9F068EE7E
:10C5400073E081E00E949F3B1092080D24ED3BE3D5
:10C5500048E95AE360E070E080912B0E90912C0E38
:10C560000E946C3A9093070D8093060D08956CED30
:10C5700075E080E00C949F3B24EF31E0DB010E94EA
:10C58000A6AC2FEF30E040E050E00E94FBB1CA01C2
:10C59000B90164527A4F8F4F9F4F80E00C949F3BBC
:10C5A0008091320E882339F060ED77E081E00E94BF
:10C5B0009F3B0C94743A61E083E090E07DC520914C
:10C5C000320E211103C002960C94C63B08952091AF
:10C5D000320E222389F06FE676E080E00E949F3BD6
:10C5E0002AED3BE342E350E060E070E080912B0EE7
:10C5F00090912C0E0C946C3A02960C94C63B80E001
:10C600000E94888081E00E9488808091320E811192
:10C6100003C082E00E9488806CED75E080E00E949B
:10C620009F3B6CED75E081E00E949F3B8091320E54
:10C6300081110CC086E399E7A1E0BB27ABBFFC01E9
:10C640006791769182E00E949F3BE4C30895FC01CC
:10C650008089918993878287828993899587848746
:10C660008489958997878687089526E00C94B2413E
:10C670008091600680935F06089520910E0E22231C
:10C6800069F0A0910C0EB0910D0EED91FC911197F7
:10C690000190F081E02DBC01CD0119940895209105
:10C6A0000B0E222369F0A091090EB0910A0EED91B4
:10C6B000FC9111970190F081E02DBC01CD011994FE
:10C6C00008952091080E222369F0A091060EB091E2
:10C6D000070EED91FC9111970190F081E02DBC01C6
:10C6E000CD01199408952091050E222369F0A0919F
:10C6F000030EB091040EED91FC9111970190F08121
:10C70000E02DBC01CD01199408952091020E222341
:10C7100069F0A091000EB091010EED91FC9111977E
:10C720000190F081E02DBC01CD0119940895209174
:10C73000FF0D222369F0A091FD0DB091FE0DED914A
:10C74000FC9111970190F081E02DBC01CD0119946D
:10C7500008952091FC0D222369F0A091FA0DB0916B
:10C76000FB0DED91FC9111970190F081E02DBC0142
:10C77000CD01199408952091F90D222369F0A0911B
:10C78000F70DB091F80DED91FC9111970190F081AA
:10C79000E02DBC01CD01199408952091F60D2223BE
:10C7A00069F0A091F40DB091F50DED91FC91119708
:10C7B0000190F081E02DBC01CD0119940895809184
:10C7C000590690915A06DC01ED91FC91EC5AFF4F0D
:10C7D0000190F081E02D19948091590690915A06AC
:10C7E000DC01ED91FC91EE5AFF4F0190F081E02DBC
:10C7F00019948091590690915A06DC01ED91FC91B3
:10C80000E05BFF4F0190F081E02D199480919D0F26
:10C8100081110DC08091E6059091E705DC01ED9155
:10C82000FC910190F081E02D60E070E01994089592
:10C8300080919D0F81110DC08091E6059091E705D3
:10C84000DC01ED91FC910190F081E02D6FEF70E043
:10C850001994089580916006882361F00E943F84B6
:10C86000029741F06AEA74E180915D0690915E065C
:10C870000C943840089580915F06882341F06CEC59
:10C8800073E180915D0690915E060C9438400895A6
:10C8900080915F06882341F06CEB73E180915D0627
:10C8A00090915E060C9438400895CF93DF932091C9
:10C8B000110E3091120E28173907D1F09093120EF5
:10C8C0008093110E20915F06222391F0EC016BE71B
:10C8D00074E180915D0690915E060E94C73EBE01A4
:10C8E00080915D0690915E06DF91CF910C947976F0
:10C8F000DF91CF910895CF93DF9320910F0E309168
:10C90000100E28173907D1F09093100E80930F0E58
:10C9100020915F06222391F0EC0161E674E18091A1
:10C920005D0690915E060E94C73EBE0180915D0645
:10C9300090915E06DF91CF910C947976DF91CF9143
:10C9400008952091080E222331F0BC018091F20D50
:10C950009091F30D1BCC08952091050E222331F008
:10C96000BC018091F00D9091F10D10CC08952091B3
:10C97000020E222331F0BC018091EE0D9091EF0D5B
:10C9800005CC08952091FF0D222331F0BC01809148
:10C99000EC0D9091ED0DFACB08952091FC0D222322
:10C9A00031F0BC018091EA0D9091EB0DEFCB089531
:10C9B0002091F90D222331F0BC018091E80D909176
:10C9C000E90DE4CB08952091F60D222331F0BC014E
:10C9D0008091E60D9091E70DD9CB0895CF92DF922B
:10C9E000EF92FF9220910002213019F42091A90FBB
:10C9F00004C02230C9F52091AF0F2223A9F19C0178
:10CA0000211584E0380710F02FEF33E0ADE0B0E0FF
:10CA10000E9449B22FEF33E040E050E00E94FBB1AA
:10CA200069017A018FEFC81AD80AE80AF80A8091DA
:10CA3000AD128C15C9F0C092AD1280915F068823AB
:10CA400099F06AE174E180915D0690915E060E9422
:10CA5000C73E6C2D80915D0690915E06FF90EF9031
:10CA6000DF90CF900C94EC78FF90EF90DF90CF9018
:10CA70000895CF92DF92EF92FF9220910002213031
:10CA800019F42091A60F04C02230C9F52091AC0FF3
:10CA90002223A9F19C01211584E0380710F02FEF23
:10CAA00033E0ADE0B0E00E9449B22FEF33E040E068
:10CAB00050E00E94FBB169017A018FEFC81AD80AD1
:10CAC000E80AF80A8091AB128C15C9F0C092AB123B
:10CAD00080915F06882399F063E074E180915D06A0
:10CAE00090915E060E94C73E6C2D80915D069091EC
:10CAF0005E06FF90EF90DF90CF900C94EC78FF9063
:10CB0000EF90DF90CF90089581E0809356060E94C9
:10CB1000607D80915F06882341F069EE73E180912A
:10CB20005D0690915E060C943840089583E08093F2
:10CB300056060E94F97C80915F06882341F066EFDB
:10CB400073E180915D0690915E060C9438400895E3
:10CB500082E0809356060E94F97C80915F068823CC
:10CB600041F06CED73E180915D0690915E060C944E
:10CB7000384008950BC7809101028111EBC606C7AA
:10CB8000E9C680910002813011F482E001C081E0A9
:10CB90000C94AD7E82E00C94AD7E81E00C94AD7E71
:10CBA0000C94EF219091CE0F81E089270C94D5470A
:10CBB00080E00C94D547682F80915D0690915E06C9
:10CBC0000E94417A68EA74E180915D0690915E0668
:10CBD0000C94C73EF0DF80915D0690915E060C9448
:10CBE0002540CF92DF92EF92FF929C01A3E6B0E046
:10CBF0000E9449B22FEF33E040E050E00E94FBB1C9
:10CC000069017A018FEFC81AD80AE80AF80A8091F8
:10CC1000B9058C15A1F0C092B90580915F068823F3
:10CC200071F06AE474E180915D0690915E060E9465
:10CC3000C73E8C2DFF90EF90DF90CF90CBCFFF9031
:10CC4000EF90DF90CF900895CF92DF92EF92FF9216
:10CC50009C01A3E6B0E00E9449B22FEF33E040E030
:10CC600050E00E94FBB169017A018FEFC81AD80A1F
:10CC7000E80AF80A8091BA058C15A1F0C092BA05AD
:10CC800080915F06882371F061E374E180915D0615
:10CC900090915E060E94C73E8C2DFF90EF90DF9032
:10CCA000CF9098CFFF90EF90DF90CF900895209194
:10CCB0005D0630915E06882319F069EE76E002C0C9
:10CCC0006DEE76E0C9010C94C73EF1DF80915D0600
:10CCD00090915E060C94254020915D0630915E0691
:10CCE000882319F06DE974E102C062EA74E1C901B8
:10CCF0000E94C73E80915D0690915E060C9425408F
:10CD00006BE974E180915D0690915E060C94C73EDC
:10CD100067E974E180915D0690915E060C94C73ED0
:10CD2000CF93CDE265E974E180915D0690915E0656
:10CD30000E94C73EC150B1F780915D0690915E069A
:10CD40000E94254080915D0690915E06DC01ED9188
:10CD5000FC910284F385E02DCF911994FF920F93FB
:10CD60001F93CF93DF93CDB7DEB765970FB6F894D7
:10CD7000DEBF0FBECDBFFF24F394F0928E0A0E9457
:10CD8000BD790AEA19E0F801118A8CE890E09A83EB
:10CD9000898324E630E03C832B8328E730E03E8320
:10CDA0002D8324EF31E038872F831D8A25E1FE0192
:10CDB0003196ACEBB9E001900D922A95E1F7F801BC
:10CDC000908B878784E086870E94B2790E94ED432A
:10CDD000F8016083718382839383F48665960FB62E
:10CDE000F894DEBF0FBECDBFDF91CF911F910F91A1
:10CDF000FF90089510928E0A4091D3055091D4056A
:10CE000060E070E02EEA36E68091C5059091C60597
:10CE10000C946C3A8091320E811112C086E399E72E
:10CE2000A1E0BB27ABBFFC016791769182E00E9435
:10CE30009F3B81E08093130E1092170E1092140EF8
:10CE4000089581E20E94174221E0892B09F420E035
:10CE5000822F08958091D905882309F447C081E085
:10CE600080938A0AEEDF882329F08091DC058823ED
:10CE7000D9F106C08091DA05811105C08091D905EC
:10CE80000E948F7631C09091D905963069F5823035
:10CE900081F08330D1F0813039F5E091F809F091DB
:10CEA000F90972978081918145E550E060E070E07A
:10CEB00017C0E091F809F091F9097297808191818A
:10CEC0004AE550E060E070E00BC0E091F809F091B5
:10CED000F9097297808191814FE550E060E070E040
:10CEE0008850964F0E947D4D0C944D71089580910D
:10CEF0004D0E882319F081E08093870A8091C70541
:10CF00009091C805DC01ED91FC910688F789E02D30
:10CF100019958091380E81110E94F9758091370E14
:10CF2000882391F061E088E00E943F424091350EF5
:10CF30005091360E60E070E025EE33E78091C50534
:10CF40009091C6050E946C3A80914D0E882321F085
:10CF500080914C0E811101C07DDF80914C0E8823A1
:10CF600079F080914D0E882359F080914B0E8823E3
:10CF700039F0E091490EF0914A0E82810E94AF8013
:10CF800039CF80918C0A811158C05BDF8823F1F082
:10CF900081E080938C0A8091C7059091C805DC01DF
:10CFA000ED91FC910288F389E02D19950E94087299
:10CFB0002CE232E748E95AE360E070E08091C50571
:10CFC0009091C6050E946C3A15DF0AC080914C0E04
:10CFD000882339F180914D0E882319F00E946376E1
:10CFE00039CF0E944D7680914B0E882339F0E09125
:10CFF000490EF0914A0E82810E94AF804091330E1B
:10D000005091340E14161506BCF4052E000C660B58
:10D01000770B27E737E68091C5059091C6050C94FC
:10D020006C3A80914B0E882339F0E091490EF091D3
:10D030004A0E82810E94AF805ACF08950F931F93AA
:10D040002091320E211135C046E359E761E0772780
:10D050009C01220F331F820F931F092E000CAA0B75
:10D06000BB0B0296A11DB11D840F951FA61FB71FF4
:10D07000ABBFFC01879106E319E721E0332740911C
:10D08000170E93E0499FA0011124052E000C660B9A
:10D09000770B4E5F5F4F6F4F7F4F040F151F261F9B
:10D0A000371F2BBFF8010791801718F01F910F91C0
:10D0B000B1CE1F910F9108958F929F92AF92BF9220
:10D0C000CF92DF92EF92FF920F931F93CF93DF9354
:10D0D000EC01A62E8091320E81116BC046E359E718
:10D0E00061E077276E01CC0CDD1CCC0EDD1E0D2C13
:10D0F000000CEE08FF08D701C6010296A11DB11D64
:10D10000480F591F6A1F7B1F6BBFFA01879146E3C7
:10D1100059E761E07727B090170E93E0B99E800140
:10D120001124012E000C220B330B0E5F1F4F2F4FCB
:10D130003F4F400F511F621F731F6BBFFA01479192
:10D14000481708F036C08090150E9090160E00918A
:10D150002B0E10912C0EB401C8010E94053A8823B1
:10D1600021F0B401C8010E941D3A86E399E7A1E0CD
:10D17000BB278C0D9D1DAE1DBF1DABBFFC01679174
:10D18000769182E00E949F3BB092140EC093170EDE
:10D19000AA2079F01092130E2AE037E642E350E01D
:10D1A00060E070E0C8010E946C3A9093160E809384
:10D1B000150EDF91CF911F910F91FF90EF90DF90AF
:10D1C000CF90BF90AF909F908F900895CF92DF92B5
:10D1D000EF92FF928091320E811134C08091310E16
:10D1E000882381F161E08EE090E066DF60912F0E90
:10D1F0007091300ECB01A0E0B0E0C0902D0ED09029
:10D200002E0EE12CF12CC816D906EA06FB0664F4B2
:10D21000BC01CD016C197D098E099F090E949C3EBD
:10D22000C60ED71EE81EF91E26EE38E6B701A60187
:10D2300080912B0E90912C0E0E946C3A90932A0EA6
:10D240008093290EFF90EF90DF90CF900895CF92BA
:10D25000DF92EF92FF928091320E811134C0809163
:10D26000280E882381F161E08DE090E025DF609158
:10D27000260E7091270ECB01A0E0B0E0C090240EE6
:10D28000D090250EE12CF12CC816D906EA06FB0633
:10D2900064F4BC01CD016C197D098E099F090E94BF
:10D2A0009C3EC60ED71EE81EF91E27E239E6B701DE
:10D2B000A60180912B0E90912C0E0E946C3A9093B7
:10D2C000230E8093220EFF90EF90DF90CF90089571
:10D2D000CF92DF92EF92FF928091320E811134C093
:10D2E0008091210E882381F161E08CE090E0E4DE02
:10D2F00060911F0E7091200ECB01A0E0B0E0C090B5
:10D300001D0ED0901E0EE12CF12CC816D906EA068F
:10D31000FB0664F4BC01CD016C197D098E099F09DF
:10D320000E949C3EC60ED71EE81EF91E28E639E66E
:10D33000B701A60180912B0E90912C0E0E946C3AA1
:10D3400090931C0E80931B0EFF90EF90DF90CF9078
:10D3500008958091320E81112CC080911A0E88237D
:10D3600041F08091210E811104C081E08093210E53
:10D37000AFDF8091190E882361F08091320E811108
:10D3800008C08091280E811104C081E08093280E8E
:10D390005EDF8091180E882361F08091320E81113A
:10D3A00008C08091310E811104C081E08093310E5C
:10D3B0000DCF08950F931F93CF93DF9320919D0F6F
:10D3C00021111BC0C091E605D091E70508811981A4
:10D3D0009C01AFEFB0E00E9449B22FEF33E040E094
:10D3E00050E00E94FBB1D801ED91FC91B901CE0152
:10D3F000DF91CF911F910F911994DF91CF911F91E0
:10D400000F9108950C94BD7F0E949D46809159060E
:10D4100090915A06DC01ED91FC9104A0F5A1E02D5C
:10D4200019940E9424458091590690915A06DC0176
:10D43000ED91FC9102A0F3A1E02D19940F931F939D
:10D44000CF93DF930091410E1091420EC091C5051C
:10D45000D091C605B801CE010E94053A882379F023
:10D46000B801CE010E941D3A8091C7059091C80570
:10D47000DC01ED91FC9100A0F1A1E02D1995009146
:10D480003F0E1091400EC091C505D091C605B80160
:10D49000CE010E94053A882321F0B801CE010E94F6
:10D4A0001D3A729880915F06882361F065EA75E104
:10D4B00080915D0690915E06DF91CF911F910F9153
:10D4C0000C943840DF91CF911F910F910895CF9325
:10D4D000DF93C091C505D091C6056091410E709152
:10D4E000420ECE010E94053A811129C040913D0EA5
:10D4F00050E060E070E020E231E7CE010E94863A21
:10D500009093420E8093410E8091C7059091C8057B
:10D51000DC01ED91FC91068CF78DE02D1995809141
:10D52000DE05882361F060913F0E7091400E80917E
:10D53000C5059091C6050E94053A882371F0809137
:10D540005F068823E9F06CE975E180915D069091B2
:10D550005E06DF91CF910C9438400E94107420E158
:10D5600034E744E650E060E070E08091C5059091BA
:10D57000C6050E94863A9093400E80933F0EDFCFFF
:10D58000DF91CF9108950E94F97580915F068823FD
:10D5900041F061E775E180915D0690915E060C9423
:10D5A00038400895E0913B0EF0913C0E82810E943C
:10D5B000AF8080915F06882341F063E575E180913B
:10D5C0005D0690915E060C943840089580914D0E52
:10D5D000882319F00E94637602C00E944D768091E4
:10D5E0005F06882379F020918F0F80915D069091DE
:10D5F0005E06222319F067E175E102C060E375E180
:10D600000C94384008950C94607DCF9380918E0ADD
:10D61000882309F468C015DC90918C0A882341F0B6
:10D62000911161C08091E905882309F445C05BC070
:10D63000911159C080915F06882341F068EF74E131
:10D6400080915D0690915E060E9438409ADC81E0F0
:10D650008093E40580910702813009F044C08091F5
:10D66000C90F882309F43FC080918F0F882379F078
:10D670002CE23DE742E350E060E070E087EB9AE0A7
:10D680000E94863A90933A0E8093390E2CC04091B6
:10D69000910F5091920F141615065CF4052E000C94
:10D6A000660B770B27E83CE787EB9AE0CF910C9469
:10D6B0006C3ACF910C94877C82E08093E90580914D
:10D6C0005F06882341F064E075E180915D069091EA
:10D6D0005E060E943840C1E0C093E8050E94607D6C
:10D6E00050DCC093E405CF9108950C94F97C8091AF
:10D6F000550681110C94607D0C94F97C0C94037E8A
:10D700000C94537E0E94D8898091BD0581110C94A0
:10D71000037E0C94537ECF939C01A4E6B0E00E945C
:10D7200049B22FEF33E040E050E00E94FBB1C22F3E
:10D7300030E080913E0E281B310937FF03C0319540
:10D74000219531092330310534F1C33020F0C23640
:10D7500018F0C4E601C0C0E08091590690915A06C5
:10D76000DC01ED91FC91E25BFF4F0190F081E02D37
:10D770006C2F1995C0933E0E80915F06882359F057
:10D780006FED74E180915D0690915E060E94C73E48
:10D790008C2FCF911FCACF9108959C010197849738
:10D7A00010F4822F0895C90184569109843893405A
:10D7B00040F4C90164E670E00E9471AC822F94E6E7
:10D7C0001BC0283E43E03407D8F0C90168EE73E07F
:10D7D0000E9471AC48E15CEF649FC001659F900DB1
:10D7E000749F900D1124280F391FC9016AE070E061
:10D7F0000E9485AC822F9AE0699F801911240895B8
:10D8000080E008956CEE74E180915D0690915E0673
:10D810000C94C73E8091590690915A06DC01ED9117
:10D82000FC910484F585E02D60E0199480915906FF
:10D8300090915A06DC01ED91FC910484F585E02D70
:10D8400061E01994CF93DF9380919D0F882349F174
:10D8500080910102882329F1C091E605D091E70566
:10D860008BA19CA1892B11F01CA21BA22D8D3E8D9A
:10D870008B8D9C8D9B878A873D872C879F878E8782
:10D88000E881F9810190F081E02D60E070E0CE0147
:10D8900019951F8A1E8A0E94ED436F8F78A389A372
:10D8A0009AA3DF91CF910895CF93DF9380919D0F3D
:10D8B000882349F180910102882329F1C091E6056E
:10D8C000D091E7058BA19CA1892B11F01CA21BA272
:10D8D0002D8D3E8D898D9A8D9B878A873D872C87DC
:10D8E0009F878E87E881F9810190F081E02D60E0CB
:10D8F00070E0CE0119951F8A1E8A0E94ED436F8F3A
:10D9000078A389A39AA3DF91CF9108951F93CF9312
:10D91000DF9390919D0F9923C9F0182FC091E605D0
:10D92000D091E705CE010E9427638E899F89892BBC
:10D9300049F4112319F0898D9A8D02C08B8D9C8D2D
:10D940009F8B8E8B81E090E09CA38BA3DF91CF9186
:10D950001F910895809101028823B9F0109201026D
:10D9600080915F06882341F06FEC74E180915D0641
:10D9700090915E060E9438400E94D8898091BD0532
:10D98000882319F080915506C1CF08958091010236
:10D9900081111AC081E08093010280915F06882383
:10D9A00041F060EC74E180915D0690915E060E940A
:10D9B00038400E94D8898091BD05882329F0809144
:10D9C0005506811171CF3ECF08950F931F930E948A
:10D9D000D2790E94117F87EB9AE00E948E3A0E94D2
:10D9E000FD830E94D8898091B2099091B309892B57
:10D9F00001F10E94ED430091AE091091AF09209111
:10DA0000B0093091B109AB01BC01401B510B620B55
:10DA1000730B8091B2099091B309A0E0B0E0841734
:10DA20009507A607B70728F40E94A7790E94BD7939
:10DA300022C08091B9099091BA09892BE1F00E9426
:10DA4000ED430091AA091091AB092091AC093091E6
:10DA5000AD09AB01BC01401B510B620B730B8091F4
:10DA6000B9099091BA09A0E0B0E084179507A6071C
:10DA7000B70708F45AC08091BC0F833041F12CF4F1
:10DA80008130A9F0823099F02DC086305CF580910C
:10DA90004E0690914F06DC01ED91FC910680F781D6
:10DAA000E02D199580914C0690914D0614C08091FF
:10DAB000520690915306DC01ED91FC910680F781AE
:10DAC000E02D1995809150069091510604C08091E7
:10DAD0004E0690914F06DC01ED91FC910680F78196
:10DAE000E02D19958091570690915806DC01ED9133
:10DAF000FC910680F781E02D199580915B0690914D
:10DB00005C06DC01ED91FC910680F781E02D199512
:10DB10008091E6059091E705DC01ED91FC9106808E
:10DB2000F781E02D1F910F9119948091B7098F5FB4
:10DB30008093B7099091B8098917E0F480FF03C07A
:10DB40000E94A77902C00E94B2798091BB0981111D
:10DB500022C0E091B709EB3008F066CFF0E0EE0F9D
:10DB6000FF1FE454F64F808191819093BA0980930E
:10DB7000B90911C08091D009882309F455CF80914B
:10DB8000BC099091BD099093BA098093B90910928C
:10DB9000B7090E94B2790E94ED436093AA0970937D
:10DBA000AB098093AC099093AD0965CF0C945245B5
:10DBB0000C9467458091480E882319F00E945245C5
:10DBC00002C00E9467459091480E81E089278093AA
:10DBD000480E08950C947D450C9492458091470E13
:10DBE000882319F00E947D4502C00E9492459091C1
:10DBF000470E81E089278093470E08950C949E4438
:10DC00000C94D7448091460E882319F00E949E44BC
:10DC100002C00E94D7449091460E81E089278093EC
:10DC2000460E089581E00C94D5479091CC0F81E089
:10DC300089270C94054880E00C94054881E00C94F9
:10DC400005488091F805882329F00E94524527E66F
:10DC500035E404C00E94674522E535E44CE251E01A
:10DC600060E070E087EB9AE00C946C3A8091F105EB
:10DC7000882329F00E947D4522E935E404C00E94F2
:10DC800092452DE735E44CE251E060E070E087EB2F
:10DC90009AE00C946C3A8091590690915A06DC01F6
:10DCA000ED91FC9104ACF5ADE02D66E01995809105
:10DCB0005F06882349F0A6DD64ED76E180915D067C
:10DCC00090915E060C943840089580915906909189
:10DCD0005A06DC01ED91FC9102ACF3ADE02D66E05B
:10DCE000199580915F06882349F08CDD60EC76E120
:10DCF00080915D0690915E060C9438400895809165
:10DD0000590690915A06DC01ED91FC9100ACF1AD01
:10DD1000E02D66E0199580915F06882349F072DD59
:10DD20006EEB76E180915D0690915E060C94384032
:10DD300008958091590690915A06DC01ED91FC916D
:10DD400004ACF5ADE02D65E0199580915F06882360
:10DD500049F058DD65EB76E180915D0690915E06B5
:10DD60000C94384008958091590690915A06DC0130
:10DD7000ED91FC9102ACF3ADE02D65E01995809139
:10DD80005F06882349F03EDD61EA76E180915D0619
:10DD900090915E060C9438400895809159069091B8
:10DDA0005A06DC01ED91FC9100ACF1ADE02D65E08F
:10DDB000199580915F06882349F024DD6FE976E1AB
:10DDC00080915D0690915E060C9438400895809194
:10DDD000590690915A06DC01ED91FC9104ACF5AD29
:10DDE000E02D64E0199580915F06882349F00ADDF3
:10DDF00066E976E180915D0690915E060C9438406C
:10DE000008958091590690915A06DC01ED91FC919C
:10DE100002ACF3ADE02D64E0199580915F06882394
:10DE200049F0F0DC62E876E180915D0690915E0653
:10DE30000C94384008958091590690915A06DC015F
:10DE4000ED91FC9100ACF1ADE02D64E0199580916D
:10DE50005F06882349F0D6DC60E876E180915D06B4
:10DE600090915E060C9438400895809159069091E7
:10DE70005A06DC01ED91FC9104ACF5ADE02D63E0B8
:10DE8000199580915F06882349F0BCDC67E776E14D
:10DE900080915D0690915E060C94384008958091C3
:10DEA000590690915A06DC01ED91FC9102ACF3AD5C
:10DEB000E02D63E0199580915F06882349F0A2DC8C
:10DEC00063E676E180915D0690915E060C943840A1
:10DED00008958091590690915A06DC01ED91FC91CC
:10DEE00000ACF1ADE02D63E0199580915F068823C9
:10DEF00049F088DC61E676E180915D0690915E06EE
:10DF00000C94384008958091590690915A06DC018E
:10DF1000ED91FC9104ACF5ADE02D62E01995809196
:10DF20005F06882349F06EDC68E576E180915D0646
:10DF300090915E060C943840089580915906909116
:10DF40005A06DC01ED91FC9102ACF3ADE02D62E0EC
:10DF5000199580915F06882349F054DC64E476E1EA
:10DF600080915D0690915E060C94384008958091F2
:10DF7000590690915A06DC01ED91FC9100ACF1AD8F
:10DF8000E02D62E0199580915F06882349F03ADC24
:10DF900062E476E180915D0690915E060C943840D3
:10DFA00008958091590690915A06DC01ED91FC91FB
:10DFB00004ACF5ADE02D61E0199580915F068823F2
:10DFC00049F020DC69E376E180915D0690915E0680
:10DFD0000C94384008958091590690915A06DC01BE
:10DFE000ED91FC9102ACF3ADE02D61E019958091CB
:10DFF0005F06882349F006DC65E276E180915D06E4
:10E0000090915E060C943840089580915906909145
:10E010005A06DC01ED91FC9100ACF1ADE02D61E020
:10E02000199580915F06882349F0ECDB63E276E185
:10E0300080915D0690915E060C94384008950E9490
:10E040009E4440911F105091201060E070E027ED39
:10E0500034E487EB9AE00E946C3A90937C128093B0
:10E060007B1280915F06882341F066ED75E1809117
:10E070005D0690915E060C94384008950E94D74446
:10E0800040911F105091201060E070E02EE934E4C0
:10E0900087EB9AE00E946C3A90937C1280937B12FB
:10E0A00080915F06882341F063EC75E180915D0605
:10E0B00090915E060C9438400895ACCBB7CBCF93CB
:10E0C000DF9380917A12882321F110927A1260E016
:10E0D00088E00E943F42C0917B12D0917C12BE0129
:10E0E00087EB9AE00E94053A882329F0BE0187EB6E
:10E0F0009AE00E941D3A80915F06882371F06AE0E1
:10E1000076E180915D0690915E06DF91CF910C944F
:10E110003840DF91CF910C94868ADF91CF9108959A
:10E1200080917A12811102C00C94868A0895CF934F
:10E13000DF9380917D12882311F10E949E441092FA
:10E140007D12C0917B12D0917C12BE0187EB9AE0C8
:10E150000E94053A882329F0BE0187EB9AE00E94CD
:10E160001D3A80915F06882371F061EF75E180911F
:10E170005D0690915E06DF91CF910C943840DF915F
:10E18000CF910C94EA44DF91CF9108950C94EA4426
:10E190006091251070E088E00E94AA4280915F069D
:10E1A000882341F06DEA75E180915D0690915E06ED
:10E1B0000C94384008950C9462460C9477468091F4
:10E1C000450E882319F00E94624602C00E947746DD
:10E1D0009091450E81E089278093450E08950C9417
:10E1E0009D460C94C9468091440E882319F00E94E4
:10E1F0009D4602C00E94C9469091440E81E0892745
:10E200008093440E08950C94D8460C94F246809165
:10E21000430E882319F00E94D84602C00E94F2469D
:10E220009091430E81E089278093430E0895809159
:10E230004C0E81110C94A77F0C94BD7F0C94A77F8A
:10E2400080911002882311F0729801C0729A909107
:10E25000100281E089278093100208951092E5054D
:10E260001092D1051092C4051092CD051092CE05E2
:10E270001092CF051092D00581E080938A0A4091D8
:10E28000D5055091D60560E070E02DE431E780912E
:10E29000C5059091C6050C946C3A80919D09811139
:10E2A0001CC01092D5091092D6091092D70910926D
:10E2B000D8091092D9091092DA091092DD098091DB
:10E2C000880A9091890ADC01ED91FC910190F0811E
:10E2D000E02D199510928A0A08952DE431E745E062
:10E2E00050E060E070E08091C5059091C6050C9407
:10E2F0006C3A6091580E7091590E8091C5059091BD
:10E30000C6050E94053A882319F081E08093570ED4
:10E31000089560E087E00E943F4210928B0A0895C2
:10E3200061E087E00E943F4281E080938B0A08957C
:10E33000CF93DF938091650E811110C084EF91E03F
:10E340009093640E8093630E8BE290E09093620E44
:10E350008093610E81E08093650E20C08091610EF4
:10E360009091620E8532910514F0049709C08331B3
:10E37000910514F0029704C0823091052CF00197AA
:10E380009093620E8093610E8091610E9091620E67
:10E3900097FF04C01092620E1092610EC091600E41
:10E3A000CC2311F0B6DF01C0BBDF81E08C27809366
:10E3B000600EC091630ED091640E1C161D0654F0C1
:10E3C0001092650EA6DF28E032E74AEF50E060E0E9
:10E3D00070E007C028E931E7AE010D2E000C660B96
:10E3E000770B8091C5059091C6050E946C3A909379
:10E3F0005F0E80935E0E8091610E9091620EC81B3D
:10E40000D90BD093640EC093630EDF91CF91089522
:10E410000F931F93CF93DF9380918C0A882329F069
:10E42000DF91CF911F910F9183CF00915E0E1091DC
:10E430005F0EC091C505D091C605B801CE010E94FE
:10E44000053A882321F0B801CE010E941D3ADF91E0
:10E45000CF911F910F915DCFCF92DF92EF92FF92FC
:10E4600010928C0A2091C9053091CA054091CB05C4
:10E470005091CC056091CD057091CE058091CF056E
:10E480009091D0050E94ACAC6B017C0120E030E0A3
:10E49000A9010E94B2B087FD09C0C092CD05D092FB
:10E4A000CE05E092CF05F092D00508C01092CD05C0
:10E4B0001092CE051092CF051092D005FF90EF90EC
:10E4C000DF90CF90A5CF0F931F93CF93DF938091D1
:10E4D0005D0E9091E50581112AC0992309F456C07B
:10E4E00000915B0E10915C0EC091C505D091C605E0
:10E4F000B801CE010E94053A882321F0B801CE016F
:10E500000E941D3A0DDF23E632E742EC51E060E065
:10E5100070E08091C5059091C6050E94863A90935F
:10E520005C0E80935B0E81E080935D0E5AC08091FB
:10E530008B0A992361F0882329F0DF91CF911F91F5
:10E540000F91E7CEDF91CF911F910F91E9CE8823F4
:10E55000C9F360915B0E70915C0E8091C50590913E
:10E56000C6050E941D3A23E632E744E150E060E030
:10E5700070E08091C5059091C6050E94863A9093FF
:10E580005C0E80935B0E10925D0E2BC0C091110249
:10E59000D09112022297D0931202C09311021C163E
:10E5A0001D0674F4BE01772787E00E94AA42CC239F
:10E5B00021F081E080938B0A14C010928B0A11C065
:10E5C00060915B0E70915C0E8091C5059091C605BF
:10E5D0000E941D3A9EDE8FEF90E09093120280938E
:10E5E0001102DF91CF911F910F9108950F931F9307
:10E5F000CF93DF930091530E1091540EC091550E9E
:10E60000D091560EC00FD11FD093560EC093550E09
:10E61000BE01772787E00E94AA42CC2321F081E047
:10E6200080938B0A02C010928B0A10161106ECF52B
:10E630008091510E9091520EC817D9070CF485C0E5
:10E640008091570E882371F01092520E1092510E45
:10E650008CEF9FEF9093540E8093530E81E0809344
:10E66000500E73C068E770E080E090E00E949C3E2E
:10E67000DC01CB010A96A11DB11D9093520E80932F
:10E68000510E68E270E080E090E00E949C3EDC0168
:10E69000CB010A96A11DB11D66277727681B790B50
:10E6A0007093540E6093530E50C0012B09F44DC06B
:10E6B0008091510E9091520E8C179D070CF445C01D
:10E6C0008091500E882311F10091580E1091590E2F
:10E6D000C091C505D091C605B801CE010E94053A8A
:10E6E000882399F1B801CE010E941D3A12DE1092E2
:10E6F000560E1092550E1092500E8091E50588230B
:10E7000021F1DF91CF911F910F91DDCE69E670E08D
:10E7100080E090E00E949C3EDC01CB018A569F4F36
:10E72000AF4FBF4F9093520E8093510E68E270E04E
:10E7300080E090E00E949C3EDC01CB010A96A11D86
:10E74000B11D9093540E8093530EDF91CF911F9182
:10E750000F910895EF92FF921F93CF93DF9300D014
:10E76000CDB7DEB784E689838CE38A8388E28B8326
:10E7700010915A0E1330E8F4E12EF12C10FF02C074
:10E78000C8DD01C0CDDDE1E0F0E0EC0FFD1FEE0DD6
:10E79000FF1D408150E060E070E02AEA33E780919D
:10E7A000C5059091C6050E946C3A1F5F10935A0EE2
:10E7B00003C0AFDD10925A0E0F900F900F90DF91B3
:10E7C000CF911F91FF90EF90089560E088E00C9446
:10E7D0003F4261E089E20C943F420F931F93CF9335
:10E7E000DF9360E08BE20E943F4200914E0E109159
:10E7F0004F0EC091C505D091C605B801CE010E944B
:10E80000053A882341F0B801CE01DF91CF911F91E5
:10E810000F910C941D3ADF91CF911F910F910895A4
:10E8200081E080938A0A8091DD0579D236CD1F92EE
:10E830000F920FB60F9211242F933F938F939F93B4
:10E84000AF93BF938091140D9091150DA091160D6B
:10E85000B091170D3091660E23E0230F2D3720F471
:10E860000196A11DB11D05C026E8230F0296A11D2A
:10E87000B11D2093660E8093140D9093150DA093F7
:10E88000160DB093170D8091180D9091190DA09150
:10E890001A0DB0911B0D0196A11DB11D8093180D8D
:10E8A0009093190DA0931A0DB0931B0DBF91AF91CA
:10E8B0009F918F913F912F910F900FBE0F901F90BE
:10E8C00018950F931F93CF93DF9300915E0E1091D5
:10E8D0005F0EC091C505D091C605B801CE010E945A
:10E8E000053A8823A1F0B801CE010E941D3A29E71C
:10E8F00031E748EB5BE060E070E08091C505909106
:10E90000C6050E946C3A90935F0E80935E0E6091F4
:10E91000580E7091590E8091C5059091C6050E94C0
:10E92000053A81114BC01092570E8FEF90E09093F3
:10E93000560E8093550EF4DC68E770E080E090E0BE
:10E940000E949C3EDC01CB010A96A11DB11D909353
:10E95000520E8093510E68E270E080E090E00E94D9
:10E960009C3EDC01CB010A96A11DB11D66277727CD
:10E97000681B790B7093540E6093530E26EF32E7A9
:10E9800044E150E060E070E08091C5059091C605DB
:10E990000E94863A9093590E8093580E29E731E7EA
:10E9A00048EB5BE060E070E08091C5059091C605A2
:10E9B0000E946C3A90935F0E80935E0EDF91CF9130
:10E9C0001F910F9108958F929F92AF92BF92CF9215
:10E9D000EF92FF920F931F93CF93DF932091E00567
:10E9E000223008F07AC07B018C018090CD05909098
:10E9F000CE05A090CF05B090D00520E030E0A90171
:10EA0000C501B4010E94B2B0181654F520E030E000
:10EA1000A901C501B4010E94AAAD181654F420E062
:10EA200030E048E452E4C501B4010E94B2B01816C7
:10EA3000D4F420E030E048E452E4C501B4010E947F
:10EA4000AAAD18169CF420E030E048EC52E4C50171
:10EA5000B4010E94B2B087FF09C0CBE4D0E008C087
:10EA6000C0E0D0E005C0C2E3D0E002C0C4E6D0E020
:10EA70008FEF8C0D823070F4209739F06C2FC80125
:10EA80000E94534A6C2FC7010DC0C8010E94276322
:10EA9000C70116C08DEF8C0D8230F8F4209779F005
:10EAA0006C2FC801DF91CF911F910F91FF90EF90D4
:10EAB000CF90BF90AF909F908F900C94534AC80115
:10EAC000DF91CF911F910F91FF90EF90CF90BF906A
:10EAD000AF909F908F900C942763DF91CF911F91FF
:10EAE0000F91FF90EF90CF90BF90AF909F908F903D
:10EAF00008958F929F92AF92BF92CF92DF92EF9242
:10EB0000FF92C090CD05D090CE05E090CF05F0905B
:10EB1000D00520E030E0A901C701B6010E94AAADEE
:10EB200020E030E040E05FE387FD0BC0C701B601A5
:10EB30000E94ADAC4B015C010E9479AD97FD27C0EE
:10EB400010C0C701B6010E94ACAC0E9479AD97FD20
:10EB50001EC06536710581059105DCF424E6822F1F
:10EB600014C0C501B4010E9479AD653671058105F7
:10EB700091057CF420E030E040E05FE3C701B6019E
:10EB80000E94ADAC0E9479AD84E6861B03C084E68A
:10EB900001C080E0FF90EF90DF90CF90BF90AF90EA
:10EBA0009F908F9008950F931F93CF93DF930091C1
:10EBB000BE051091BF05C091C505D091C605B8012D
:10EBC000CE010E94053A882321F0B801CE010E94AF
:10EBD0001D3A80918C0A882339F010928C0ADF91BB
:10EBE000CF911F910F9114CCDF91CF911F910F9175
:10EBF000089560E089E20E943F4229EE33E742E354
:10EC000050E060E070E08091C5059091C6050C94DD
:10EC10006C3A1F920F920FB60F9211240BB60F92FF
:10EC20002F933F934F935F936F937F938F939F9314
:10EC3000AF93BF93EF93FF9380914D0E8823B1F074
:10EC4000669918C0EE98C9DD80914C0E882391F02A
:10EC500080914B0E882339F0E091490EF0914A0ED5
:10EC600082810E94AF800E94776704C0669B02C0C9
:10EC7000EE98B3DDFF91EF91BF91AF919F918F918E
:10EC80007F916F915F914F913F912F910F900BBEAC
:10EC90000F900FBE0F901F90189561E08BE20E94BD
:10ECA0003F42EE9A2DEE33E748E853E160E070E032
:10ECB0008091C5059091C6050E946C3A90934F0EC5
:10ECC00080934E0E089561E08BE20E943F42EE9ADF
:10ECD0002DEE33E748E853E160E070E08091C50530
:10ECE0009091C6050E946C3A90934F0E80934E0E01
:10ECF00008950F931F93CF93DF93EC01AB0160E076
:10ED000070E02AE00E94003F8C01CE010E94254065
:10ED1000800F911FDF91CF911F910F9108958F92D6
:10ED20009F92AF92BF92CF92DF92EF92FF920F939A
:10ED30001F93CF93DF931F921F92CDB7DEB7082E9C
:10ED4000000C990BAA0BBB0BFC013197ED30F105C0
:10ED500008F033C28827EA5AFE4F8F4F0C9498ACC4
:10ED600084E0809399098AE080939A0986E28093EF
:10ED70009C0981E080939F098093A00980939E095C
:10ED800045E257E120E030E08091990990E02817B2
:10ED900039070CF059C1FA0185919491A0E0B0E0D7
:10EDA000880F991FAA1FBB1FF901EE0FFF1FEE0F5F
:10EDB000FF1FE05DF64F80839183A283B3832F5FB3
:10EDC0003F4F4E5F5F4FE0CF84E0809399098AE028
:10EDD00080939A0986E280939C0981E080939F0941
:10EDE0008093A00982E080939E094DE157E120E0E5
:10EDF00030E08091990990E0281739070CF024C180
:10EE0000FA0185919491A0E0B0E0880F991FAA1FA4
:10EE1000BB1FF901EE0FFF1FEE0FFF1FE05DF64F66
:10EE200080839183A283B3832F5F3F4F4E5F5F4FF9
:10EE3000E0CF84E080939A0985E280939C0981E089
:10EE400080939F0988E08093A00983E080939E09C6
:10EE500080E090E0FC01EB5EF84EE491DC01AF5500
:10EE6000B64FEC93019688309105A1F70E94264C8D
:10EE7000EBC088E08093990986E080939A0986E246
:10EE800080939C0981E080939F098093A00984E08E
:10EE900080939E0945E057E120E030E08091990998
:10EEA00090E0281739070CF0CFC0FA0185919491B2
:10EEB000A0E0B0E0880F991FAA1FBB1FF901EE0F59
:10EEC000FF1FEE0FFF1FE05DF64F80839183A2834B
:10EED000B3832F5F3F4F4E5F5F4FE0CF88E080935B
:10EEE000990986E080939A0986E280939C0981E0E3
:10EEF00080939F098093A00985E080939E0945EF48
:10EF000056E120E030E08091990990E02817390718
:10EF10000CF09AC0FA0185919491A0E0B0E0880FBE
:10EF2000991FAA1FBB1FF901EE0FFF1FEE0FFF1F56
:10EF3000E05DF64F80839183A283B3832F5F3F4FC1
:10EF40004E5F5F4FE0CFE091F809F091F9097297B9
:10EF50008081918140E550E060E070E08850964FFC
:10EF60000E947D4D2AC182E18093990985E08093BA
:10EF70009A0982E280939C0981E080939F098093A3
:10EF8000A00987E080939E0980E993E3A0E0B0E0C8
:10EF90008093300990933109A0933209B0933309DB
:10EFA000F2E08F2E912C01E010E080E090E0A0E0F4
:10EFB000BBE54CE454E060E070E024EEC22E2CE0AF
:10EFC000D22EE12CF12C9801220F331F220F331F78
:10EFD0005401AA0CBB1CAA0CBB1C205D364FF901C6
:10EFE000B7FF0DC0C082D182E282F3829501205D1D
:10EFF000364FF90140835183628373830CC0408391
:10F000005183628373839501205D364FF901C0827D
:10F01000D182E282F382880F991FAA1FBB1F0E5F65
:10F020001F4FF2E08F0E911C22E18216910459F6D7
:10F0300088E79FEFA0E0B0E0809374099093750992
:10F04000A0937609B09377090E94954CB6C0CE0183
:10F0500001960E94124C23E040E150E060E070E035
:10F0600072C084E08093990982E380939A0986E2D2
:10F0700080939C0981E080939F098093A0098AE096
:10F0800080939E094DEE56E120E030E08091990991
:10F0900090E028173907C4F6FA0185919491A0E011
:10F0A000B0E0880F991FAA1FBB1FF901EE0FFF1FC9
:10F0B000EE0FFF1FE05DF64F80839183A283B38341
:10F0C0002F5F3F4F4E5F5F4FE1CF84E08093990900
:10F0D00080E280939A0986E280939C0981E0809384
:10F0E0009F098093A0098BE080939E0945EE56E12D
:10F0F00020E030E08091990990E0281739070CF062
:10F10000A3CFFA0185919491A0E0B0E0880F991FF8
:10F11000AA1FBB1FF901EE0FFF1FEE0FFF1FE05DDF
:10F12000F64F80839183A283B3832F5F3F4F4E5F5F
:10F130005F4FE0CFCE0101960E94124C21E040E1EA
:10F1400054E060E070E0CE0101960E94F14C35C0C1
:10F1500084E08093990983E080939A0986E2809302
:10F160009C0981E080939F098093A0098DE08093A2
:10F170009E094DED56E120E030E08091990990E044
:10F18000281739070CF060CFFA0185919491A0E01F
:10F19000B0E0880F991FAA1FBB1FF901EE0FFF1FD8
:10F1A000EE0FFF1FE05DF64F80839183A283B38350
:10F1B0002F5F3F4F4E5F5F4FE0CF0F900F90DF917B
:10F1C000CF911F910F91FF90EF90DF90CF90BF9064
:10F1D000AF909F908F9008950F931F93CF93DF93DD
:10F1E000EC01462F50E060E070E02AE00E94003F12
:10F1F0008C01CE010E942540800F911FDF91CF919D
:10F200001F910F9108952FB7F894882381F0809172
:10F210009311909194119093A2118093A1118091D8
:10F22000A3119091A41118161906ACF00FC080918B
:10F230009511909196119093A2118093A1118091B4
:10F24000A3119091A411181619062CF48091A31102
:10F250009091A41107C08091A3119091A411919550
:10F26000819591099093A4118093A3112FBF0895C4
:10F27000AF92BF92CF92DF92EF92FF920F931F93C4
:10F28000CF93DF931F921F92CDB7DEB78C017A83A5
:10F290006983CE0101966C01580192E0A90EB11C60
:10F2A000E12CF12CC8010E94DBB1F60161916F01E4
:10F2B000861731F0C8010E94EDB1FFEFEF1AFF0A87
:10F2C0000F5F1F4F0A151B0569F781E0EF2809F44E
:10F2D00080E00F900F90DF91CF911F910F91FF90E1
:10F2E000EF90DF90CF90BF90AF900895EF92FF9294
:10F2F0000F931F93CF93DF931F921F92CDB7DEB76B
:10F300008C017B018AEA8A8341E050E0BE016E5F96
:10F310007F4FC8010E94E650D701ED91FC91028415
:10F32000F385E02DC701199582E8898341E050E01B
:10F33000BE016F5F7F4FC8010E94E6500F900F9093
:10F34000DF91CF911F910F91FF90EF9008958091E1
:10F35000B509882311F061E001C060E08091B40933
:10F360000C943F428091B509882311F060E001C000
:10F3700061E08091B4090C943F42CF93DF93CAEAD5
:10F38000D9E01C861D861E86188A1F860E94ED43C2
:10F39000688379838A839B83198618861C86DF910C
:10F3A000CF910895CF92DF92EF92FF920F931F9328
:10F3B0000E94ED436B017C0160930F127093101259
:10F3C00080931112909312128091A30A0E94174207
:10F3D00080930E129091A50A992329F091E0811152
:10F3E00090E090930E128091AD0A9091AE0AA09198
:10F3F000AF0AB091B00A97018601081B190B2A0BBE
:10F400003B0B4091B10A5091B20A6091B30A7091DE
:10F41000B40A9091A60A041715072607370760F467
:10F42000C092A90AD092AA0AE092AB0AF092AC0A62
:10F430001092A80A892F1EC09093A70A80910E12DD
:10F440008093A60AC092A90AD092AA0AE092AB0AB7
:10F45000F092AC0A891761F0C092AD0AD092AE0A60
:10F46000E092AF0AF092B00A91E09093A80A02C02D
:10F470001092A80A1F910F91FF90EF90DF90CF900C
:10F480000895462F50E060E070E02AE00C94003FC1
:10F490000F931F93CF93DF93EC012AE00E94003F6C
:10F4A0008C01CE010E942540800F911FDF91CF91EA
:10F4B0001F910F910895CF92DF92EF92FF920F93D9
:10F4C0001F93CF93DF936B01770FEE08FF08F7FED2
:10F4D0001BC0EC016DE20E94C03E8C014427552701
:10F4E000BA014C195D096E097F092AE0CE010E941C
:10F4F000003F800F911FDF91CF911F910F91FF90DF
:10F50000EF90DF90CF9008952AE0B701A601DF9138
:10F51000CF911F910F91FF90EF90DF90CF900C94BF
:10F52000003FCF92DF92EF92FF920F931F93CF9302
:10F53000DF938C016B01770FEE08FF08F7FE12C016
:10F540006DE20E94C03EEC0144275527BA014C19D8
:10F550005D096E097F092AE0C8010E94003FC80FBB
:10F56000D91F06C02AE0B701A6010E94003FEC01A6
:10F57000C8010E9425408C0F9D1FDF91CF911F91E4
:10F580000F91FF90EF90DF90CF9008950F931F930E
:10F59000CF93DF931F92CDB7DEB78C0169830E94B2
:10F5A000DBB16981861729F0C8010E94EDB181E0C5
:10F5B00001C080E00F90DF91CF911F910F910895CE
:10F5C000CF930E94148484E090E09093A00A8093EB
:10F5D0009F0A88E69EE09093321180933111109239
:10F5E0002C1180919E0A9091680E891718F091E075
:10F5F0009093291121E73EE030933C1120933B1179
:10F60000109236119091710E891718F091E0909335
:10F6100033112AE73EE030934611209345111092B2
:10F62000401190917A0E891718F091E090933D1156
:10F6300023E83EE03093501120934F1110924A116D
:10F640009091830E891718F091E0909347111092D2
:10F650009D0A20E030E0F901E85FF04F40815181E0
:10F66000415051094432510520F491E090939D0A94
:10F6700005C02D5F3F4F2837310569F790919D0AEE
:10F68000992341F120917B0E30917C0E2D5D3F4FEF
:10F6900030937C0E20937B0E20917D0E30917E0E58
:10F6A0002352310930937E0E20937D0E2091840EDB
:10F6B0003091850E2D5D3F4F3093850E2093840E43
:10F6C0002091860E3091870E235231093093870E98
:10F6D0002093860E9091810F9F3049F49091820F74
:10F6E0009F3029F4109228111092271108C0209100
:10F6F000D00F3091D10F309328112093271122E1A0
:10F7000030E0309325112093241120919F0A3091ED
:10F71000A00AACE8BEE0E0EDF0E141E0B683A583ED
:10F720009C91992329F0891718F040832F5F3F4F50
:10F730001A96379691E1E432F90781F73093A00ADF
:10F7400020939F0A2131310534F080E190E09093BD
:10F75000A00A80939F0A0E94FF838DE291E190931B
:10F760003310809332108091311190913211909327
:10F770003110809330108AE291E19093351080939C
:10F7800034108BE291E1909337108093361089E228
:10F7900091E1909339108093381087E391E1909331
:10F7A0003D1080933C1080913B1190913C119093BF
:10F7B0003B1080933A1084E391E190933F10809343
:10F7C0003E1085E391E1909341108093401083E3D4
:10F7D00091E1909343108093421081E491E19093E2
:10F7E0004710809346108091451190914611909357
:10F7F0004510809344108EE391E1909349108093DB
:10F8000048108FE391E190934B1080934A108DE361
:10F8100091E190934D1080934C108BE491E1909383
:10F8200051108093501080914F11909150119093EE
:10F830004F1080934E1088E491E190935310809381
:10F84000521089E491E1909355108093541087E40D
:10F8500091E1909357108093561020919F0A309118
:10F86000A00A2450310960E07AE0C7E0462F50E05A
:10F870004217530724F5CA010496789FF001799F37
:10F88000F00D1124E05DFF4EC49FC001C59F900D97
:10F890001124AC014E525F4E53834283DC01A053CE
:10F8A000BF4E15964D915C911697518340838F52B0
:10F8B0009F4E95838483B187A0876F5FD7CF81E008
:10F8C0008093A10ACF9108950F931F93CF93DF9355
:10F8D000FC01248135812115310519F4FB011082C9
:10F8E00011C0EA0121972C173D0708F4E9018B01AB
:10F8F000FC0160817181AE01C8010E94E2AFC00FBE
:10F90000D11F1882DF91CF911F910F91089580919F
:10F910000702813019F485E0809307020895109260
:10F92000540608958091BC05882371F01092BC059F
:10F9300080915F06882341F06CEB78E180915D0651
:10F9400090915E060C94384008958091BC0F8330EE
:10F9500099F08091BC0581110FC081E08093BC05B6
:10F9600080915F06882341F067EA78E180915D0627
:10F9700090915E060C94384008958091BB058330C9
:10F9800079F083E08093BB0580915F06882341F086
:10F9900066E978E180915D0690915E060C943840AE
:10F9A00008958091BB05823079F082E08093BB0599
:10F9B00080915F06882341F065E878E180915D06DB
:10F9C00090915E060C94384008958091BB0581307B
:10F9D00079F081E08093BB0580915F06882341F038
:10F9E00064E778E180915D0690915E060C94384062
:10F9F00008950E94D8898091BD05882361F1809186
:10FA00008C0A811128C080915506811124C081E0A3
:10FA1000809355060E94546C8091E805882319F064
:10FA20001092E8050CC08091590690915A06DC01AD
:10FA3000ED91FC910088F189E02D61E019958091AC
:10FA40005F06882341F069E478E180915D0690913A
:10FA50005E060C94384008958091870A8823C1F08F
:10FA60006091390E70913A0E87EB9AE00E941D3A30
:10FA700010923A0E1092390E1092870A8091070266
:10FA80008130D9F48091C90F8823B9F040DF15C0C7
:10FA9000809116128F5F80931612803580F06091EE
:10FAA000390E70913A0E87EB9AE00E941D3A10923F
:10FAB0003A0E1092390E1092870A1092161208957B
:10FAC0000E94D8898091BD05882341F18091550617
:10FAD000811101C00895109255060E94226C8091F8
:10FAE000E805882319F01092E8050CC080915906AA
:10FAF00090915A06DC01ED91FC910088F189E02D8E
:10FB000060E0199580915F06882341F06DE578E10A
:10FB100080915D0690915E060C9438400895CF93D5
:10FB2000DF93C0912312D0912412BE0187EB9AE09B
:10FB30000E94053A882329F0BE0187EB9AE00E94D3
:10FB40001D3A1092241210922312DF91CF91089542
:10FB50000F931F93CF93DF938091C10F9091C20FAA
:10FB6000A091C30FB091C40F181619061A061B06F0
:10FB70000CF044C00E94D8898091BD058823C9F14A
:10FB80000091231210912412B80187EB9AE00E9491
:10FB9000053A8823D9F0E5EBFCE0C0E0D0E08191A4
:10FBA00091918017910769F40E94ED43CC0FDD1FFE
:10FBB000CC0FDD1FC954D54F688379838A839B831B
:10FBC0001DC02196CE31D10551F718C04091C10F0B
:10FBD0005091C20F6091C30F7091C40F2FE33EE7A5
:10FBE00087EB9AE00E946C3A909324128093231240
:10FBF00005C0DF91CF911F910F9191CFDF91CF91F0
:10FC00001F910F91089580918C0A811137C00E9435
:10FC1000D889809180128823B1F08091BD05882316
:10FC200091F01092BD05109280120E94FF89809180
:10FC30001512882341F064E278E1809113129091CB
:10FC400014120E94384080915506882311F081E0FB
:10FC500001C080E00E94866C81E08093E80530DF7F
:10FC60008091590690915A06DC01ED91FC91048037
:10FC7000F581E02D19950E943A486ACF08950E94B7
:10FC8000D8898091BD05882369F0BDDF80915F062A
:10FC9000882341F064E378E180915D0690915E06EF
:10FCA0000C943840089580918C0A811155C0809140
:10FCB0005606823068F080915F06882309F44CC0B4
:10FCC00062EE77E180915D0690915E060C9438407B
:10FCD0000E94D88980918012882309F43DC08091C8
:10FCE000BD05811139C081E08093BD05109280125D
:10FCF0000E94FF8980911512882341F063ED77E11E
:10FD000080911312909114120E94384080915906EC
:10FD100090915A06DC01ED91FC910280F381E02D77
:10FD2000199580915606811116C04091B70F5091D8
:10FD3000B80F81E08093E8054115510559F060E066
:10FD400070E029EF3CE787EB9AE00E946C3A0E9452
:10FD5000226C01C04EDEFCCE0895CF93823069F450
:10FD60009091B00F2091AD0F3091B10F4091AE0F37
:10FD70005091AF0F6091AC0F0CC09091AA0F2091E1
:10FD8000A70F3091AB0F4091A80F5091A90F609130
:10FD9000A60F6093AC125093A9124093AA1230930D
:10FDA000A8122093AB129093AD1290910002891784
:10FDB000B1F08093000290915F06992381F0C82FE3
:10FDC0006AEB77E180915D0690915E060E94C73EE6
:10FDD0006C2F80915D0690915E06CF91FDC9CF9109
:10FDE0000895833079F030F4813051F0823091F40D
:10FDF0008BE30BC0843041F0853061F482E405C0B0
:10FE00008CE303C080E401C081E40E94174221E03A
:10FE1000892B09F420E0822F0895E3DF91E0892700
:10FE200008950F931F9380911B1281110DC00E94A2
:10FE3000ED436093171270931812809319129093E8
:10FE40001A1281E080931B12809113028A3AF1F416
:10FE500085E0C7DF882371F086EF97E09093C912A1
:10FE60008093C81290935E0680935D068FEF809317
:10FE700013020CC083E998E09093C9128093C812D2
:10FE800090935E0680935D06109213020E94ED43EC
:10FE900000911712109118122091191230911A1214
:10FEA000DC01CB01801B910BA20BB30BC397A10507
:10FEB000B10508F449C00E94ED4360931712709396
:10FEC00018128093191290931A1285E08ADF882302
:10FED00021F080911302882349F085E082DF8111AF
:10FEE00033C0809113028F3F79F518C086EF97E0F9
:10FEF0009093C9128093C81290935E0680935D061A
:10FF000080915F06882331F060EA77E186EF97E021
:10FF10000E9438408FEF8093130216C083E998E067
:10FF20009093C9128093C81290935E0680935D06E9
:10FF300080915F06882331F06BE877E183E998E0F0
:10FF40000E943840109213021F910F910895109251
:10FF50004C0E80915F06882379F020918F0F80915D
:10FF60005D0690915E06222319F06BE577E102C0F1
:10FF70006EE677E10C943840089581E080934C0E52
:10FF800080915F06882379F020918F0F80915D0624
:10FF900090915E06222319F06DE277E102C06FE3D3
:10FFA00077E10C9438400895482F50E095E1899FFF
:10FFB000F0011124EF5AFE4E218132818085918516
:10FFC000280F391F838194818217930728F0858138
:10FFD000968128173907E8F485E1849FF001859F11
:10FFE000F00D1124EF5AFE4E8581968128173907AE
:10FFF00028F52581368185E1849FF001859FF00DEC
:020000021000EC
:100000001124EF5AFE4E8285823019F41186108633
:10001000128685E1849FF001859FF00D1124EF5A2F
:10002000FE4E328321838091840090918500280FB9
:10003000391F30938900209388000895838194812B
:1000400082179307C0F623813481D5CF80919C0A13
:10005000811157C0E0913111F09132118581968163
:1000600090932E1180932D111092301110922F1118
:10007000E0913B11F0913C1185819681909338116C
:100080008093371110923A1110923911E091451175
:10009000F091461185819681909342118093411190
:1000A0001092441110924311E0914F11F0915011B0
:1000B0008581968190934C1180934B1110924E1133
:1000C00010924D1182E190E09093251180932411BC
:1000D00081E080932A118093341180933E118093A4
:1000E00048118093261180E090E021E0FC01E0536C
:1000F000FF4E2183079684359105C1F781E08093F7
:100100009C0A089510924A11089510924011089582
:10011000982F8FB7F89425E1929FF0011124EF5AA0
:10012000FE4E21E027838FBF41B121E030E0B901CD
:1001300002C0660F771F9A95E2F7CB01842B81B935
:1001400008958A3058F49FB7F89425E1829FF00112
:100150001124EF5AFE4E118610869FBF08951F93FB
:10016000CF93DF9325E1829FC0011124EC01CF5A88
:10017000DE4E8A8581110FC01FB7F89481E08A870F
:1001800089899A899A8389830E94ED436B877C874A
:100190008D879E871FBFDF91CF911F910895CF93C9
:1001A000DF938A30D0F56233710538F061369DE611
:1001B000790728F060E67DE602C062E370E0D42FA4
:1001C000C82F80E090E00E94B6B020E030E04AE71F
:1001D00054E40E9411AD20E030E04CE852E40E946B
:1001E00017B19B01AC0160E070E08AEF94E40E94DB
:1001F00011AD0E9479AD9B01DD2321F02227332729
:10020000261B370B8FB7F89495E1C99FF001112495
:10021000EF5AFE4E318720878FBFDF91CF9108952F
:100220008A3010F40C94693B08958A3010F40C94D1
:10023000843B08958A3058F495E1899FF001112498
:10024000EF5AFE4E8181928196958795089580E0C0
:1002500090E008958A3010F40C949F3B08951F920B
:100260000F920FB60F9211240BB60F920F931F939C
:100270002F933F934F935F936F937F938F939F93AE
:10028000AF93BF93CF93EF93FF938091791289300F
:1002900048F01092791280910012882399F0809191
:1002A000F9110DC0E0917912E15025E1E29FF001D2
:1002B0001124EF5AFE4E8781882321F0808192B16C
:1002C000892782B9E091791285E1E89FF001112434
:1002D000EF5AFE4E8781882321F0808192B1892BCD
:1002E00082B9E0917912C5E1CE9FF0011124EF5A55
:1002F000FE4E80859185892B09F04DC0E0917912E1
:10030000CE9FF0011124EF5AFE4E8285813009F014
:1003100060C00E94ED43E0917912CE9FF00111245C
:10032000EF5AFE4E0385148525853685E0917912B6
:10033000CE9FF0011124EF5AFE4E0784F089E02D84
:10034000AB01BC01401B510B620B730BCF01A0E052
:10035000B0E084179507A607B707D8F5E0917912A2
:10036000A0917912CA9FD0011124AF5ABE4E539664
:100370008D919C915497CE9FF0011124EF5AFE4E1F
:1003800091878087E0917912CE9FF0011124EF5A76
:10039000FE4E82E082878091791206DE809179128A
:1003A0008F5F80937912FF91EF91CF91BF91AF91C1
:1003B0009F918F917F916F915F914F913F912F917D
:1003C0001F910F910F900BBE0F900FBE0F901F90BB
:1003D0001895E0917912809184009091850025E133
:1003E000E29FF0011124EF5AFE4E21813281820FEB
:1003F000931F9093890080938800D0CF1F93CF9351
:10040000DF9380917812811173C0109279129FB797
:10041000F89485E128EB3BE04CED55E064E971E1AF
:10042000A1E0B0E0E0917912E93008F052C0E0912B
:1004300079128E9FF0011124EF5AFE4E32832183F0
:10044000E09179128E9FF0011124EF5AFE4E5683EF
:100450004583E09179128E9FF0011124EF5AFE4EF0
:1004600074836383E0917912F0917912ED0101C0F8
:10047000CC0FFA95EAF78E9FF0011124EF5AFE4E49
:10048000C083E09179128E9FF0011124EF5AFE4E45
:100490001782E09179128E9FF0011124EF5AFE4EDF
:1004A00011861086E09179128E9FF0011124EF5A87
:1004B000FE4E1286E09179128E9FF0011124EF5AC0
:1004C000FE4E148A138AE0917912EF5FE09379125D
:1004D000A9CF9FBF8FB7F89420EA3FE03093FB117C
:1004E0002093FA111092F9118FBF81E08093781256
:1004F000DF91CF911F9108950F931F93CF93DF93B7
:100500008C01C62FD42FDC0111968D919C911297EE
:10051000DC01ED91FC910190F081E02DD8016C910E
:100520001995F80181819281DC01ED91FC91019096
:10053000F081E02D6C2F1995F80181819281DC0109
:10054000ED91FC910190F081E02D6D2F1995F8014E
:1005500080816C2F70E0680F711D6D0F711D6F77BA
:10056000772781819281DF91CF911F910F910C9418
:10057000BF600F931F93CF93DF938C01C62FD42FAF
:10058000DC0111968D919C911297DC01ED91FC910B
:100590000190F081E02DD8016C911995F8018181CD
:1005A0009281DC01ED91FC910190F081E02D6C2FA6
:1005B0001995F80181819281DC01ED91FC91019006
:1005C000F081E02D6D2F1995F80180816C2F70E07E
:1005D000680F711D6D0F711D6F7777278181928173
:1005E000DF91CF911F910F910C94BF604F925F925A
:1005F0006F927F92AF92BF92CF92DF92EF92FF9273
:100600001F93CF93DF93DD24D39445E0C42E52E0B3
:10061000A52EB12CC3E0D0E0EE24E394F12C809120
:100620005C1290915D12DC01ED91FC910480F581EA
:10063000E02D1995892B09F4BEC0109130018091ED
:100640005C1290915D12DC01ED91FC910680F781C6
:10065000E02D199596B3B39A2091840030918500CE
:100660002059384E30938D0020938C00212F2C710F
:1006700039F010927712D0935B12C0935A12CFCFF9
:1006800093FB992790F9E0917712E11116C0992315
:1006900031F28F3021F6D092771280935E128091E2
:1006A0005A1290915B12892B09F0B9CFF0925B122C
:1006B000E0925A1210925912B2CF9111DACF91E012
:1006C0009E0F90937712F0E0E25AFD4E80839931AD
:1006D00009F0A5CF81116CC08091751282FF05C011
:1006E000D0935B12C0935A1263C083FDF9CF8091FF
:1006F0005A1290915B12019739F4809159128F5FD1
:1007000080935912843020F0B0925B12A0925A125A
:10071000809158128F5F80935812909157129817BA
:1007200008F044C0D0925612A6E3B2E1EFE5F2E140
:1007300040E050E0BA0110E0CF01FC011B3098F41A
:1007400001964080512C612C712C012E04C0440C68
:10075000551C661C771C0A94D2F744295529662932
:100760007729185FEACF9A013770205E3340C29E26
:10077000C001C39E900D112497FD079623E0959527
:1007800087952A95E1F784529A4F8D939D931B503C
:100790003BE076956795579547953A95D1F782E175
:1007A000A635B80749F61092581202C01092561298
:1007B0001092771234CFDF91CF911F91FF90EF907D
:1007C000DF90CF90BF90AF907F906F905F904F90F1
:1007D00008958091A20A833029F480913412909177
:1007E0003512E5C108958091A20A823029F48091E2
:1007F000321290913312FACE0895F5DFEACF1092BB
:100800002A111092341110923E1110924811109238
:10081000261180E090E0FC01E053FF4E1182079624
:1008200084359105C1F708958091A20A823039F08C
:10083000833049F0813049F480912F1201C080E16A
:1008400080939E0A04C08EE0FBCF10929E0A809196
:100850009E0A08958091A20A823039F0833049F0CF
:10086000813059F480912E120895BDDF8091561287
:100870000895AFDF80912D12089580E00895809152
:10088000A20A823049F0833069F0813089F4809186
:10089000291290912A120895A6DF80915A12909100
:1008A0005B12089596DF80912B1290912C1208957F
:1008B00081E090E008958F929F92AF92BF92CF9285
:1008C000DF92EF92FF921F93CF93DF93EC0111E041
:1008D0008E819F81892B09F410E02C813D81E88570
:1008E000F985C580D680878190E0A601480F591F01
:1008F0002417350764F180850D2C000CEE08FF08E5
:10090000A901330F660B770B0380F481E02D9A0168
:10091000AB012C193D094E095F09882329F0A1E09C
:10092000BFEF0E9423B204C0AFEFB0E00E9417B245
:100930004F01FF0FAA08BB08A50194012C193D091E
:100940004E095F090E94FBB13F832E834BC0A60175
:10095000481B590B421753070CF43FC080850D2CE0
:10096000000CEE08FF08A901330F660B770B81809E
:100970009280092C000CAA08BB089A01AB01281927
:1009800039094A095B09882399F0A1E0BFEF0E9469
:1009900023B2A7019601281939094A095B090E9467
:1009A000FBB1DA01C90181509F4FAF4FBF4F12C059
:1009B000AFEFB0E00E9417B2A701960128193909DC
:1009C0004A095B090E94FBB1DA01C9018F5F9109F5
:1009D000A109B1099F838E8305C01F821E82111158
:1009E00001C019828E819F81009789F08F3F910508
:1009F00019F014F08FEF90E081305FEF950714F459
:100A000081E09FEF9F838E8381E018271A83DF9117
:100A1000CF911F91FF90EF90DF90CF90BF90AF905C
:100A20009F908F900895CF93DF93C0912512D0911E
:100A300026126091271270912812CE010E94053A69
:100A400081110DC026E230E84CE251E060E070E038
:100A5000CE010E946C3A9093281280932712DF9166
:100A6000CF910895FC01128213821482158216829E
:100A700017821286089580E008950F931F93CF93F5
:100A80008C0162ED79E183E998E00E94C73ED801CC
:100A90001896ED91FC9119976081718183E998E036
:100AA0000E947976C1E0D8011A968C91C81710F58A
:100AB0006DEC79E183E998E00E94C73E6C2F83E9F1
:100AC00098E00E94417A6AEC79E183E998E00E941B
:100AD000C73EF80190858185E92FF82FEC0FF11DB5
:100AE000EC0FF11D6081718183E998E00E947976B5
:100AF000CF5FD9CFCF911F910F910895CF93DF93FF
:100B0000CDB7DEB76E970FB6F894DEBF0FBECDBF80
:100B10008F300CF080E022EC39E13A8329832BEB13
:100B200039E13C832B832DEA39E13E832D8321EA91
:100B300039E138872F8327E939E13A87298720E986
:100B400039E13C872B872CE839E13E872D8725E862
:100B500039E1388B2F872AE739E13A8B298B2DE64B
:100B600039E13C8B2B8B22E639E13E8B2D8B26E540
:100B700039E1388F2F8B24E439E13A8F298F23E331
:100B800039E13C8F2B8F2EE239E13E8F2D8FE82FFC
:100B9000EE0FFF0BEC0FFD1F818192816E960FB659
:100BA000F894DEBF0FBECDBFDF91CF910895AF9215
:100BB000BF92CF92DF92EF92FF920F931F93CF934A
:100BC000DF9387E892E17EE1D72ED80ECC24C39440
:100BD00002E010E0C3E0D0E0E2E0BE2EEE24E394B9
:100BE000F12C8091360D9091370DDC01ED91FC9147
:100BF0000480F581E02D1995892B09F4ADC0A090F2
:100C000030018091360D9091370DDC01ED91FC9112
:100C10000680F781E02D199596B3B39A2091840050
:100C200030918500285A344E30938D0020938C00EB
:100C30002A2D2C7119F01092330D4BC093FB99277C
:100C400090F9E091330DE11116C0992351F28032F1
:100C500041F6C092330D8093871280912B129091B0
:100C60002C12892B09F0BDCFF0922C12E0922B129E
:100C70001092350DB6CF9111DECFE13041F48034C2
:100C800009F0AFCFB092330D80938812E6CF91E098
:100C90009E0F9093330DF0E0E957FD4E8083903224
:100CA00009F09FCF1092330DE7E8F2E12FEF3FEF0D
:100CB0008191281B3109DE12FBCF4091A512809152
:100CC000A61290E0982F8827840F911D28173907C6
:100CD00029F0D0932C12C0932B1283CF80912B122A
:100CE00090912C12019739F48091350D8F5F80938C
:100CF000350D843020F010932C1200932B1280912C
:100D0000340D8F5F8093340D9091320D981708F554
:100D1000C0922D1220E030E0F901E957FD4E4281EA
:100D2000838190E0982F8827840F911DAC014F5E3E
:100D300052404B3D554028F4F901E85CF24F918355
:100D400080832E5F3F4F2C31310531F71092340DE7
:100D500048CF10922D1245CFDF91CF911F910F9167
:100D6000FF90EF90DF90CF90BF90AF900895EF92FB
:100D7000FF920F931F93CF93DF931092670E82E041
:100D80008093680E68EE73E070936A0E6093690E4C
:100D900040ED57E050936C0E40936B0E2CED35E018
:100DA00030936E0E20936D0E8FE080936F0E109235
:100DB000700E94E09093710E7093730E6093720EA8
:100DC0005093750E4093740E3093770E2093760EE9
:100DD0008093780E1092790E93E090937A0E709330
:100DE0007C0E60937B0E50937E0E40937D0E30936D
:100DF000800E20937F0E8093810E1092820E91E0E0
:100E00009093830E7093850E6093840E5093870E9B
:100E10004093860E3093890E2093880E80938A0E1D
:100E200010928B0EECE8FEE0A5E9BEE080E008EE53
:100E300013E060ED77E04CED55E031E022E095E025
:100E4000980F908312830183748363835683458351
:100E5000ED01229791E03883219628831C928F5FC1
:100E60003A961A968C3059F71092040F9093050F0A
:100E70001092060F9093070F80E090E09C01295993
:100E8000314FF901EF55FF4F1182108232961082D7
:100E900003968837910591F784E290E09093090FCB
:100EA0008093080F81E080930A0F2CE030E03093AC
:100EB0000C0F20930B0F94E090930D0F21E230E084
:100EC00030930F0F20930E0F27E02093100F29E08F
:100ED00030E03093120F2093110F20E12093130F75
:100EE0007AE07093800F2BE02093810F2093820F84
:100EF00048EE53E05093840F4093830F20ED37E08A
:100F00003093860F2093850F1092870F64E66093CD
:100F1000880F6093890F50938B0F40938A0F309303
:100F20008D0F20938C0F10928E0F10928F0F809345
:100F3000900F1092920F1092910F8093930F8093C5
:100F4000940FE8ECF0E0F093960FE093950FE0E259
:100F5000F3E0F093980FE093970F50939A0F40931C
:100F6000990F30939C0F20939B0F80939D0FE9E581
:100F7000F0E0F0939F0FE0939E0FE0E8F0E0F09335
:100F8000A10FE093A00FEFEFF0E0F093A30FE09339
:100F9000A20FF093A50FE093A40F8093A60F909358
:100FA000A70F1092A80F8093A90F9093AA0F1092E9
:100FB000AB0F1092AC0F8093AD0F1092AE0F10924A
:100FC000AF0F8093B00F1092B10F98E29093B20FD1
:100FD0005093B40F4093B30F5093B60F4093B50F97
:100FE0003093B80F2093B70F8093B90F92E390938B
:100FF000BA0FE2E0E093BB0F8093BC0F6093BD0F8C
:10100000E6E4E093BE0F9093BF0F1092C00F1092D2
:10101000C10F1092C20F1092C30F1092C40F109202
:10102000C50FEAEFF0E0F093C70FE093C60F109200
:10103000C80F1092C90F6093CA0F61E46093CB0F81
:101040001092CC0F9093CD0F1092CE0F9093CF0FA4
:10105000EEE5F1E0F093D10FE093D00F1092D20FB4
:10106000ACEDB5E0B093D40FA093D30F00EA1FE02E
:101070001093D60F0093D50F3093D80F2093D70F2E
:10108000C8E8D3E1D093DA0FC093D90F68EBE62E0E
:101090006BE0F62EF092DC0FE092DB0FE0E4FFE174
:1010A000F093DE0FE093DD0F1092DF0F1092E00F50
:1010B0001092E10F69E16093E20F8093E30F809358
:1010C000E40F8093E50F5093E70F4093E60F3093C2
:1010D000E90F2093E80FF092EB0FE092EA0F1093E4
:1010E000ED0F0093EC0FD093EF0FC093EE0F20E7BE
:1010F00037E13093F10F2093F00F1092F20F10921E
:10110000F30F1092F40F9093F50F9093F60F9093C6
:10111000F70F8093F80F109208101092F90F99E0D2
:101120009093FA0F1092FB0F1092FC0F1092FD0F8C
:101130001092FE0FB0930010A093FF0FF0930210D7
:10114000E093011080930310709304101092051027
:1011500021E030E0309307102093061040E052EC7D
:1011600061E070E04093091050930A1060930B10F7
:1011700070930C1040930D1050930E1060930F104D
:101180007093101040E056E960E070E04093111059
:101190005093121060931310709314104093151015
:1011A0005093161060931710709318101092191026
:1011B00020E039E130931B1020931A1010921C107C
:1011C0009EE190931D1010921E102EE130E030939E
:1011D000201020931F103093221020932110309361
:1011E0002410209323109093251090932610809321
:1011F0002710809328101092291090932A10809322
:101200002B108AE29FE4A0E0B0E080932C10909332
:101210002D10A0932E10B0932F1007E61EE0C0E013
:10122000D0E0CE010E94DBB1F80161918F018617F9
:1012300019F0CE010E94EDB12196C93CF1E0DF0723
:1012400081F7DF91CF911F910F91FF90EF9008955B
:101250004F925F926F927F928F929F92AF92BF92C6
:10126000CF92DF92EF92FF92CF93DF93EB01A091A9
:101270008512B09186129D012F5F3F4F45E0429F3E
:101280002001439F500C1124052C000C66087708A0
:10129000812C912C54012A33E1E03E07ECF449E61D
:1012A00059E761E0772775016401C40CD51CE61C81
:1012B000F71C4C0D5D1D6E1D7F1D6BBFFA01479124
:1012C000569165E0860E911CA11CB11CC417D50770
:1012D00029F12F5F3F4FDFCF25E0822E912CA12CEB
:1012E000B12C21E030E0A217B30708F44CC049E666
:1012F00059E761E07727480D591D6A1D7B1D6BBFBB
:10130000FA0147915691F5E08F0E911CA11CB11C7A
:10131000C417D50719F02F5F3F4FE5CF49E659E7CE
:1013200061E07727E5E0E29F6001E39FD00C1124A4
:101330000D2C000CEE08FF084E5F5F4F6F4F7F4F84
:101340004C0D5D1D6E1D7F1D6BBFFA0147915691BF
:10135000FC015383428349E659E761E077274C5FFC
:101360005F4F6F4F7F4FC40ED51EE61EF71EEBBEBC
:10137000F601C790FC01C482309386122093851237
:10138000C901019606C0109286121092851280E063
:1013900090E0DF91CF91FF90EF90DF90CF90BF90E2
:1013A000AF909F908F907F906F905F904F90089537
:1013B0000F931F938091801281111EC00E94ED43F4
:1013C0000091811210918212209183123091841227
:1013D000AB01BC01401B510B620B730B80917E1261
:1013E00090917F12A0E0B0E084179507A607B70799
:1013F00018F481E0809380121F910F9108958091DD
:101400007E1290917F12892B89F08091801288231F
:1014100081F00E94ED436093811270938212809359
:1014200083129093841210928012089581E0809329
:10143000801208951F920F920FB60F9211242F93CE
:101440008F939F9310929500109294008091960A2A
:101450008F5F8093960A9091A712891784F010925B
:10146000960A2091980A8091B2129091B312820F3D
:10147000911D27FD9A959093B3128093B21280919B
:10148000950A8F5F8093950A9091B712891784F01F
:101490001092950A2091970A8091B5129091B612F8
:1014A000820F911D27FD9A959093B6128093B512E5
:1014B0009F918F912F910F900FBE0F901F901895B5
:1014C0008091940A811104C08091930A882321F0AD
:1014D00080917100826003C0809171008D7F809344
:1014E000710008951F93CF93DF931F92CDB7DEB79E
:1014F00010E0181731F089830E9480661F5F898190
:10150000F8CF0F90DF91CF911F910895CF93DF9384
:1015100060E088E00E943F4210927D12C0917B12F1
:10152000D0917C12BE0187EB9AE00E94053A882395
:1015300029F0BE0187EB9AE00E941D3A81E080937A
:101540007A1280915F06882341F064E179E180910D
:101550005D0690915E060E943840DF91CF910C9419
:101560002E4460911A1070911B1080E090E00E9450
:10157000B6B020E030E04AE754E40E9411ADAB0180
:10158000BC0121E080915D0690915E060C94483F7D
:1015900065E079E180915D0690915E060E94C73E0C
:1015A0006091CF0F80915D0690915E060E94417A16
:1015B0009091CF0F8091B905981781F065EF78E190
:1015C00080915D0690915E060E94C73E6091B905CC
:1015D00080915D0690915E060E94417A63EF78E10A
:1015E00080915D0690915E060C94C73E64EE78E1B2
:1015F00080915D0690915E060E94C73E6091CD0F7E
:1016000080915D0690915E060E94417A9091CD0F87
:101610008091BA05981781F064ED78E180915D06BC
:1016200090915E060E94C73E6091BA0580915D066A
:1016300090915E060E94417A62ED78E180915D06AC
:1016400090915E060C94C73E4115510529F0611535
:10165000710511F00C94647C0895EF92FF920F9342
:101660001F93CF93DF931F921F92CDB7DEB78C01EC
:101670008CE789831A82F801E480F580FFEFEF1A86
:10168000FF0AB701C8010E94B73D882381F0F80125
:101690002081318184819581BE016F5F7F4F820FF0
:1016A000931F0E94DBAFF801F582E48281E00F9086
:1016B0000F90DF91CF911F910F91FF90EF900895C0
:1016C000AF92BF92CF92DF92EF92FF920F931F9350
:1016D000CF93DF9300D01F92CDB7DEB78C01498343
:1016E0005A836B837C83CE0101966C01580194E090
:1016F000A90EB11CE12CF12CC8010E94DBB1F6014E
:1017000061916F01861731F0C8010E94EDB1FFEFC2
:10171000EF1AFF0A0F5F1F4F0A151B0569F781E0DB
:10172000EF2809F480E00F900F900F900F90DF9159
:10173000CF911F910F91FF90EF90DF90CF90BF90CE
:10174000AF900895CF92DF92EF92FF920F931F9385
:10175000CF93DF93EC010091B812E0E0F0E020E0DD
:1017600030E0A90110E0CE17DF071CF1309711F42B
:101770000D32E1F0DF01A854BD4EFC9080ED8F0DDD
:101780008A30A8F4AAE0B0E00E9417B22F2DFF0C17
:10179000330B205331096901330FEE08FF089B0119
:1017A000AC012C0D3D1D4E1D5F1D01C011E0319699
:1017B000DACFCA01B901112339F09095809570955F
:1017C00061957F4F8F4F9F4FDF91CF911F910F9169
:1017D000FF90EF90DF90CF9008958091A60A81113D
:1017E00005C081E09091A80A911101C080E00895A0
:1017F000CF93DF932091D1093091D209E901269747
:10180000A881B981AF52B64F12961C92082E000CD7
:10181000990BAA0BBB0BFC013197EE30F10508F0D8
:1018200057C18827ED59FE4F8F4F0C9498ACF901A2
:101830003A97808191818F52964F0E9477AA882390
:1018400009F44BC1E091D109F091D209369701908A
:10185000F081E02DEF52F64F81E0A0C0F9013C97F6
:10186000808191818F52964F0E94B4A9882309F4F8
:1018700034C1E091D109F091D20936970190F081FD
:10188000E02DEF52F64F82E089C0F9013E9780814A
:1018900091818F52964F0E94F7A8882309F41DC1A9
:1018A000E091D109F091D20936970190F081E02DB5
:1018B000EF52F64F83E072C0F901709780819181F9
:1018C0008F52964F0E947AA8882309F406C1E091AE
:1018D000D109F091D20936970190F081E02DEF52B5
:1018E000F64F84E05BC0F9017297808191818F523D
:1018F000964F0E9435A8882309F4EFC0E091D109E2
:10190000F091D20936970190F081E02DEF52F64F19
:1019100085E044C0F9017497808191818F52964F80
:101920000E94BCA7882309F4D8C0E091D109F091A6
:10193000D20936970190F081E02DEF52F64F86E004
:101940002DC0F9017697808191818F52964F0E9428
:1019500036A7882309F4C1C0E091D109F091D209DA
:1019600036970190F081E02DEF52F64F87E016C0D8
:10197000F9017897808191818F52964F0E9428A714
:10198000882309F4AAC0E091D109F091D2093697D1
:101990000190F081E02DEF52F64F88E082839DC0E8
:1019A000F901B097808191818F52964F0E944AA48D
:1019B000882309F492C0E091D109F091D2093697B9
:1019C0000190F081E02DEF52F64F83819481A58143
:1019D000B6814097A105B10509F07FC08EC0F9011D
:1019E0007A97808191818F52964F0E945DA68823BD
:1019F00009F473C0E091D109F091D20936970190B2
:101A0000F081E02DEF52F64F8AE0C8CFF9017C97C4
:101A1000808191818F52964F0E9492A5882309F46C
:101A20005CC0E091D109F091D20936970190F08124
:101A3000E02DEF52F64F8BE0B1CFF901B0978081E6
:101A400091818F52964F0E944AA4882309F445C081
:101A5000E091D109F091D20936970190F081E02D03
:101A6000EF52F64F83819481A581B68180319440F5
:101A7000A105B10591F543C0F9017E97808191815F
:101A80008F52964F0E94C3A4882339F1E091D10967
:101A9000F091D20936970190F081E02DEF52F64F88
:101AA0008DE07CCFF901B097808191818F52964F64
:101AB0000E944AA4882389F0E091D109F091D209CB
:101AC00036970190F081E02DEF52F64F8EE066CF11
:101AD000E881F981EF52F64F1282E091D109F0913D
:101AE000D20936970190F081E02DEF52F64F81E058
:101AF0009281911106C080E004C089E04FCF8CE054
:101B00004DCFDF91CF910895EF92FF920F931F93E6
:101B1000CF93DF931F921F92CDB7DEB741110AC05A
:101B20007C0197FF03C0F194E194F108E616F706F3
:101B300064F402C0E12CF12C81E08093930A8FEFD2
:101B4000633371059CF425E012C06E157F0534F0F7
:101B50001092930A81E091E021E00AC06D33710593
:101B6000BCF381E08093930A23E001C024E092E07B
:101B70003091930A332379F03FB7F894899F902DE1
:101B800011249093970A2093B7120091B5121091E7
:101B9000B6123FBF0AC09FB7F8941092970AF0920E
:101BA000B612E092B5129FBF87014A83898388DC11
:101BB0004A818981442319F017FF19C014C081306C
:101BC00031F417FD10C0E016F1068CF40FC08F3F02
:101BD00071F40E151F0554F00F3F110541F03CF054
:101BE0000FEF10E004C000E010E001C08701C80161
:101BF0000F900F90DF91CF911F910F91FF90EF9079
:101C00000895CF92DF92EF92FF920F931F93CF939D
